:1000000000800010011B0000311B0000331B0000AA
:10001000351B0000371B0000391B000000000000EA
:10002000000000000000000000000000B1280000F7
:100030003D1B0000000000001F29000057290000A0
:10004000431B0000431B0000431B0000431B000038
:10005000431B0000431B0000431B0000431B000028
:10006000431B0000431B0000431B0000431B000018
:10007000431B0000431B0000431B0000431B000008
:10008000431B0000431B0000431B0000431B0000F8
:10009000431B0000431B0000431B0000431B0000E8
:1000A000431B0000431B0000431B0000431B0000D8
:1000B00091440000431B0000431B0000431B000051
:1000C000431B0000431B0000431B000010B5054C00
:1000D000237833B9044B13B10448AFF300800123F4
:1000E000237010BD2C020010000000000428010045
:1000F00008B5064B1BB106480649AFF30080064819
:10010000036813B1054B03B1984708BD0000000018
:1001100004280100300200102C0200100000000032
:10012000154B002B08BF134B9D46A3F5803A0021C9
:100130008B460F461348144A121A0CF08BFA0F4BD9
:10014000002B00D098470E4B002B00D09847002082
:10015000002104000D000D48002802D00C480BF0CF
:10016000E2FF0CF0C3F92000290000F09FFB0BF028
:10017000F7FF00BF00000800008000100000000032
:10018000092A00002C020010801C001027C100006A
:1001900085C40000436809B1C26800E002691360C9
:1001A000704743691A6843681A420CBF0020012057
:1001B0007047000013B50468A088A378217862789E
:1001C000009007480CF0E6FAA268E16805480CF0D8
:1001D000E1FA054B1A6801321A6002B010BD00BF87
:1001E000541E01008F1E0100A802001038B518220D
:1001F00004460D4600210CF02DFA2046294601F058
:10020000D0FD204638BD30B585B0044601F042FD32
:10021000684601F03FFD9DE80F0084E80F0020468E
:1002200005B030BD10B5044601F023FD23699842A6
:1002300034BF0020012010BD38B504460D4601F042
:1002400008FD2046256101F01CFD2046BDE8384030
:1002500001F0EABC7FB504460E4601F01BFD68467E
:1002600001F018FD9DE80F0084E80F00204631469C
:10027000FFF7E2FF204604B070BD10B5046901F03D
:10028000F8FC201A10BD2DE9F04705460E469046B1
:100290000024B44204DA4046FFF7C4FF814690B11F
:1002A000B4420CD1D5F8F83033B14FF47A7105F17E
:1002B000D0005943FFF7C0FF0020BDE8F0874FF0A2
:1002C000FF30BDE8F08740462F68FFF7D6FF04F106
:1002D000080A024649463846AA440BF02AFD384629
:1002E000514632460BF0D8FD0028E8DB0444D0E745
:1002F0002DE9F34705460446084655F86C7B0E4643
:10030000FFF7BBFF0021024638460BF012FD3846CE
:10031000294601220BF0E5FD0128074602D04FF0E7
:10032000FF354AE03046FFF7A8FF4FF00508824648
:100330000025B8F1010818D0D4F8009000214846F3
:1003400052460BF0F6FC48460DF1070101220BF076
:10035000C8FD012809D19DF8073003F07F021B0674
:1003600007FB02554FEAC717E3D404F16D00294695
:1003700002F066F8002D13DD04EB00083046276814
:10038000FFF77BFF08F16D080246002138460BF0AD
:10039000D0FC384641462A460BF0A3FDA842BED108
:1003A00094F86C50D4F8F8302D0933B14FF47A71C9
:1003B00004F1E4005943FFF73FFF284602B0BDE8CF
:1003C000F08710B50446D0F8F80086B018B304F1F1
:1003D000D000FFF727FF20B904F1E400FFF722FF68
:1003E000B8B194F8FC30A3B94FF47A7101A8FFF7C3
:1003F00031FF642104F1080001F0A3FF011E08DDB4
:10040000204601AAFFF73FFF28B9012384F8FC30FA
:1004100001E04FF0FF3006B010BD10B543687BB16E
:1004200004685CB1806810F0010F4FEA600018BFEB
:100430002258204418BFD358984710BD0846984703
:1004400010BD2DE9F74307460D46904604464FF090
:1004500000094FF0FF36D4F8041189B3284602F0A2
:10046000CDF828BBAB686868D4F804211844013A79
:1004700012F8011FD1B1834222D293F800C0BCF11F
:100480002F0F01D12F2904E02B2908D023290AD0CE
:10049000614509D014E009782F2905D00133591C92
:1004A0008142F8D300E0431E0133E1E7834207D1E4
:1004B000D4F8083104F584708BB9D4F80C3173B9D1
:1004C00009F10109B9F1050F04F11004C3D1B6B166
:1004D000D7F854315BB9D7F8583143B910E06946C1
:1004E000CDF8008001950026FFF797FFE8E707F5B4
:1004F000AA706946CDF800800195FFF78EFF0026AF
:10050000304603B0BDE8F0832DE9F0418EB00546DA
:100510008846FFF7EDFE86B2B31E0B2B49D8DFE805
:1005200003F04806484848484848484848440CAB07
:1005300001930DAB029307AC05F16C0364270393A1
:10054000009404970DF12A000AA90DF129020BABC2
:1005500001F0FAFE012836D1214628460AAAFFF703
:1005600070FF9DF828402CB3012C07D1BDF82C302A
:1005700005F1080000933946042208E0022C1FD13F
:10058000BDF82C3005F10800009339460522002300
:1005900002F0AAF80028014612DD28464246FFF77D
:1005A00072FE431C044605D108E0002485F8FC4097
:1005B00000E000242846FFF704FF24B1264602E0AD
:1005C0004FF0FF34FAE730460EB0BDE8F081F8B5E1
:1005D00007460E4615464FF0FF342846FFF722FE29
:1005E00030B938462946FFF78FFFB0420446F4D1B0
:1005F0002046F8BDF0B585B0044616461F46FFF705
:1006000042FE054600BB012F21D12046042132467F
:10061000FFF7DDFF042815D1642300930DF10D00D1
:1006200003A90DF10E0204F16C0301F0D3FE0128C1
:1006300008D1B4F8CC21BDF80E309A4207D1A4F805
:10064000CC5104E04FF0FF35002384F86031284698
:1006500005B0F0BD2DE9F047044690B089460BA8DF
:100660006168D2F80880D768157892F801A0FFF782
:10067000F1FD94F86031002609960A9613B94FF0FF
:10068000FF3039E06B1E012BCDF820900AD8D4F84A
:1006900000614FF6FF739E4214BF01360126C4F875
:1006A0000061B6B2CDF800A0019602AB04F10809D2
:1006B00008AA07CA83E807000697CDF814804846C1
:1006C000642100222B4601F0C7FF071ED7DD94F8F6
:1006D000FD305BB904F2611049463A460BF096FFD3
:1006E000A4F8CC61C4F8C87184F8CE5120463946CC
:1006F0000BAA2B46FFF77EFF10B0BDE8F08770B560
:10070000044686B00D4601A86168FFF7A3FD94F882
:100710006031002B53D12B8B04F10806C4F8F8305C
:10072000AB7E6421003318BF012384F8FD303046CE
:100730002A4601F045FD011E41DD204601AAFFF7D2
:10074000A2FD00283DD1D4F8F83033B14FF47A71CE
:1007500004F1E4005943FFF76FFD2046022101AA8E
:10076000FFF735FF022812D1FF2306A800228DF8DB
:10077000023000F8152D0DF1020104F16C02642322
:1007800001F0A0FD012802D19DF8020001E04FF028
:10079000FF30B4F8CC316BB104F261116422304601
:1007A0000BF034FF2046D4F8C81101AA94F8CE31DA
:1007B000FFF720FF28B9012384F8603101E04FF0F2
:1007C000FF3006B070BD2DE9F041044692B00E46F0
:1007D0000DA861680AAF98468DF81720FFF73AFD1B
:1007E000384600210C220BF035FF94F860310A9650
:1007F000002B54D0D4F800514FF6FF739D424FF0B8
:10080000010314BFED181D46C4F800518DE888009F
:100810000DF117030293642104F108000022ABB22A
:1008200001F098FF011E3ADD20460DAAFFF72BFDCF
:100830000546002835D1204609210DAAFFF7C7FE3D
:1008400009282CD14FF0FF33099304F16C03009376
:10085000642301930DF11E00012108AA09AB08953C
:1008600001F0BDFF012803D10998802813D000E0D2
:100870002846002204EB0213D3F804313BB91032AE
:1008800004EB02146660C4F80C8018460BE00132D9
:10089000052AEFD138B1002384F8603103E04FF02E
:1008A000FF352846F7E712B0BDE8F0812DE9F043A7
:1008B000ADF2045D0DF13C08824F40460BF0BAFAF0
:1008C0000BF0CEFB43F698200BF0DAFBFB687A685E
:1008D0007D4E1A60F36872687C4D1A60EB686A6836
:1008E0007B4C1A60E36862684FF07C501A6001F03C
:1008F00017FC3846FFF755FCD0F1010138BF002145
:100900003846FFF747FC3046FFF74BFCD0F10101BA
:1009100038BF00213046FFF73DFC2846FFF741FC79
:10092000D0F1010138BF00212846FFF733FC2046F3
:10093000FFF737FCD0F1010138BF00212046FFF757
:1009400029FC4FF07C5001F0EBFB3846FFF729FC07
:10095000D0F1010138BF00213846FFF71BFC3046BB
:10096000FFF71FFCD0F1010138BF00213046FFF72F
:1009700011FC2846FFF715FCD0F1010138BF00211A
:100980002846FFF707FC2046FFF70BFCD0F10101DA
:1009900038BF00212046FFF7FDFB4E4B00224E489A
:1009A0000BF0F8FE80A8CDF83081FFF72CFC85A86D
:1009B000FFF729FC00238C934CAA1A44103300241F
:1009C000502BC2F80841C2F80C41F5D1C0AE3046F8
:1009D00080AF3546A194A294FFF715FC0FCD0FC749
:1009E0002B6830463B60FFF70EFC85AFB646BEE88D
:1009F0000F000FC72B6839493B6040F25B7247F22A
:100A0000305337484D938DF82C428D9491949594A2
:100A100099949D948DF89042ADF8FC428DF8FE4279
:100A20000BF0B8FE214640464FF47A720BF081F984
:100A300040462A4940F25B720BF009FA044610B1B5
:100A4000284821463AE01F48FFF7ABFBD0F10101EF
:100A500038BF00211B48FFF79DFB4FF07E5001F08F
:100A60005FFB1848FFF79DFBD0F1010138BF002163
:100A70001448FFF78FFB4FF07E5001F051FB1148F7
:100A8000FFF78FFBD0F1010138BF00210D48FFF7C0
:100A900081FB154958221DA80BF0B8FD03238DF8E2
:100AA0007C30124B1DA94CA820932D943094FFF755
:100AB00026FE0146002800F087800D480BF06AFEF4
:100AC00077E000BF900200104802001060020010A2
:100AD000780200100000E03F9D1E0100CC1E0100C6
:100AE000B71E0100DA1E0100FC1D01005A1F0100A3
:100AF000F51E01006048FFF754FBD0F1010138BF3B
:100B000000215D48FFF746FB4FF07E5001F008FBE7
:100B10005948FFF746FBD0F1010138BF0021564884
:100B2000FFF738FB4FF07E5001F0FAFA5248FFF71A
:100B300038FBD0F1010138BF00214F48FFF72AFBF5
:100B40004E4900224E4B33A80BF020FF4FF40073A8
:100B50004C49324600974C488DF818708DF8197042
:100B60008DF81A7000F054FB4849099006AA4CA869
:100B70000896FFF76FFD00244FF4007300250393E0
:100B80004349444A444B8146CDE9004502960497C7
:100B90003D4800F07BFB3A4B0990404933A80022C6
:100BA00008960BF0F3FE01238DF81830B9F1000F11
:100BB00059D012A80BF076F840460BF026F9002029
:100BC0000DF2045DBDE8F0833548FFF7EAFAD0F195
:100BD000010138BF00213248FFF7DCFA4FF07E50A8
:100BE00001F09EFA2E48FFF7DCFAD0F1010138BF80
:100BF00000212B48FFF7CEFA4FF07E5001F090FA1B
:100C00002748FFF7CEFAD0F1010138BF0021244870
:100C1000FFF7C0FA4CA823490222234BFFF7D3FD6C
:100C2000074600283FF466AF2048394646E70AA841
:100C3000FFF7F8FA28B94CA80AA9FFF765FC0130BC
:100C4000F5D1124906AA4CA8FFF704FD18480BF08D
:100C500019FE1848FFF7A5FAD0F1010138BF0021AD
:100C60001448FFF797FA0AA8FFF7CDFA0AA84FF43D
:100C70007A71FFF7E1FADAE760020010831F0100E2
:100C80000000E03FCA1F0100B41F01002F1F010038
:100C900052B8DC419A19AD42B8310A46EF1F010043
:100CA00048020010661F0100B5010000111F01007D
:100CB000481F01007802001008B508490848FFF7EE
:100CC00095FA08490848FFF791FA08490848FFF7DC
:100CD0008DFA08490848FFF789FA08BD32C0092093
:100CE0009002001034C009204802001035C00920CD
:100CF0006002001037C0092078020010F0B5C0F380
:100D0000C7567F3EB6B233B2802B4FEAD0774FF052
:100D10000001C0F316001BD07F331ED150EA01033F
:100D200019D0001841EB01014FF4000200230240EA
:100D30000B4052EA030406D1001806F1FF3641EBDE
:100D40000101B6B2F0E70E4A00231040194004E05A
:100D50004FF4806601E04FF601464B0743EAD003AB
:100D6000FD073605002443EA0501420706F17F53DB
:100D700042EA040003F5401320431943F0BD00BFCD
:100D8000FFFF7F0010B54468A3184360002393421F
:100D900003D0C85CE0540133F9E7012010BD000026
:100DA00010B5034C8260002204604160C26010BD37
:100DB000850D0000F8B503680446154623B9E368BD
:100DC00001201D44E560F8BDC66897198668B742E2
:100DD00001D90020F8BD98470028F0D1F9E7F0B517
:100DE00052EA030187B08646CDE9002303D01646B8
:100DF0001F46002202E0694601221BE0F40966F06A
:100E00007F0303A944EA4764FD09535454EA0503E8
:100E100002F1010202D026462F46EFE706A8531E34
:100E2000034413F80C0CCDE9004500F07F0003F8F3
:100E30000C0C7046FFF7BEFF07B0F0BD0B79042B1A
:100E400003D0082B05D10CCA01E012680023FFF77C
:100E5000C6BF002070470B79013B072B11D8DFE894
:100E600003F00407100B1010100D92F9002001E0A0
:100E7000B2F90020D31702E01268FBE70CCAFFF7B3
:100E8000AEBF00207047002A73F1000105DA921806
:100E900043EB0303D243DB4302E0921843EB03032B
:100EA000FFF79DBF0B79042B03D0082B05D10CCA8B
:100EB00001E01268D317FFF7E6BF00207047042255
:100EC000FFF778BF1146FFF7FABF0822FFF772BF9E
:100ED0001146FFF7FABF41EAC2020023FFF77FBFC6
:100EE0004B780A4603F00F03072B0FD8DFE803F017
:100EF0000404040A06080808002104E0012102E0B5
:100F0000022100E005211278FFF7E5BF00207047BD
:100F10002DE9F04715464A7886B002F0C003402B11
:100F200006460C4676D0802B02D0002B40F09C80E9
:100F300001218DF80710514902F00F0051F820806F
:100F4000E17811B149B2294401E00DF10701802B8C
:100F500005D12D682F1C18BF01278DF8077002F0EE
:100F60003002102A05D0202A11D0002A7CD11DB9C8
:100F70007AE00B78002B5FD030462146FFF7B0FFB8
:100F8000002871D0304621462A46C04773E00F68DA
:100F9000002F51D0802B02D063799F4264D804285F
:100FA00064DC304602212278FFF795FF00285BD0F1
:100FB000637803F00F03032B02D14FEA87091AE08D
:100FC000042B02D14FEAC70915E002A80021102224
:100FD0000BF040FBAA464FF0000902A821465246FA
:100FE000C047002840D0237909F10109B9459A4446
:100FF000F3D1DDF8149030464A460023FFF7EFFEA8
:10100000002831D0316851B930464A46FFF7D2FE48
:1010100050B311E02B682A1D73B198472BE04FF0B5
:101020000009304621462A46C047E8B1237909F134
:101030000109B9451D44F4D101201CE06378304614
:1010400003F0CF03862B214613D12A68C04758B13D
:10105000237909F10109B9451D44EDD030462146F7
:10106000FFF73EFF0028E9D1002004E04FF000091F
:10107000F4E72A46EAE706B0BDE8F0872020010041
:101080002DE9F0418046174601F10A04002614F8C4
:101090000A3CA4F10A01002B33D014F8083C1E448A
:1010A00014F8093C374403F0C002802A03F0F00230
:1010B0000CBF042614F8066C202A08BF14F8052C6F
:1010C00003F00F0308BF5643082B12D13D68B5B19A
:1010D0002A684046536813B12946984703E091684F
:1010E0006A68FFF715FF10B90020BDE8F081AD6810
:1010F000EDE740463A46FFF70BFF0028F4D00A34EC
:10110000C5E70120BDE8F08170B5144622460023F2
:1011100005460E46FFF763FE30B1284631462246AB
:10112000BDE87040FFF746BE70BD10B54B780C7936
:1011300003F0C003802B08BF4FF0FF340023A3420D
:1011400005D11146BDE810401A46FFF7DDBFD15C5E
:101150000029F6D00133F2E710B513464A7802F0C1
:10116000C002802A02D159681A6805E01A68097914
:10117000141D8C4204D8191DBDE81040FFF7C4BFF0
:10118000002010BDF0B585B00F4616460021102294
:10119000044668460BF05EFA684639463246FFF769
:1011A0006FFF08B9002027E0039D20462A46002350
:1011B000FFF715FE0028F5D023682BB92046194605
:1011C0002A46FFF7F7FD17E0E268A918A2689142E6
:1011D000E8D8009363683246019368460023394695
:1011E00003930295FFF74CFF039BE268AB421A445E
:1011F000E260019A6260D5D105B0F0BDD1F8061069
:1012000009B1FFF7BFBF08467047FFF7BBBF00003B
:1012100070B5A0B006460D46684611461A46249C95
:10122000FFF7BEFD04A8002120220BF013FA0123D2
:101230008DF8103034B10DF1120021468DF81130C7
:101240000BF041FC68460F4904AAFFF7DEFF08B91E
:10125000002014E0502200210CA80BF0FBF93146CD
:101260000CA80BF030FC294616A80BF02CFC6846A5
:1012700005490CAAFFF7C9FF0028E9D0039820B060
:1012800070BD00BF442001009E2001002DE9F04701
:10129000A2B08246894668462C9990462D9A1F46F0
:1012A000DDE92A452E9EFFF77BFD04A800212022C0
:1012B0000BF0D0F903238DF810303EB101230DF16E
:1012C000120031468DF811300BF0FDFB68461949CC
:1012D00004AAFFF79AFF08B9002027E0582200214E
:1012E0000CA80BF0B7F951460CA80BF0ECFB4846E4
:1012F000FFF704FDCDE916014046FFF7FFFCCDE9FD
:1013000018013846FFF7FAFC0123CDE91C018DF8DE
:1013100068301CB1CDE920458DF878306846064923
:101320000CAAFFF772FF0028D6D0039822B0BDE8C0
:10133000F08700BF442001006220010010B50021A9
:10134000044604F01F0400F02DF80120A04010BD59
:1013500038B504464B1C0D4621600FD00846FFF7F8
:10136000EDFF25F01F0505F11803E36005F11C03EF
:10137000236105F1140360606361A56038BD0068F6
:1013800000F029B811B1012906D07047836841687F
:101390001A6822EA010203E08368426819680A4376
:1013A0001A60704700F16040A0F51C2000F00F02A9
:1013B0005200030903209040914010B59B0003F1B7
:1013C000804303F530331C6824EA00001860186875
:1013D0000843186010BD00F16040A0F51C2030B536
:1013E000C1F3800200F01F0402FA04F443099B00D9
:1013F00003F1804303F530339D6E25EA04059D66B5
:101400009D6E2C439C669AB900F00F0252000309AE
:101410000320904001FA02F29B0003F1804303F5A0
:1014200030331C6C24EA00001864186C02431A6400
:1014300030BD0000012810B50C4602D002280FD0A4
:1014400010BD014638225443104B18591A19D8B10F
:1014500011B992F83630BBB10D4B1B68984710BDDF
:101460000A4B382101FB04335968013105D09968D2
:101470001869016093F8361009B10021E2E753685A
:1014800023F001035360DDE710BD00BFB40200107C
:10149000B0020010034A00219068C0F34200FFF739
:1014A000C9BF00BF00C00040034A01219068C0F3DB
:1014B0004200FFF7BFBF00BF00000140034A022106
:1014C0009068C0F34200FFF7B5BF00BF008009403D
:1014D000034A03219068C0F34200FFF7ABBF00BF8F
:1014E00000C0094070B5294C0368A34211D006DC46
:1014F000A4F58044A34212D1254C052511E0254CCA
:10150000A34209D004F58044A34208D1224C082507
:1015100007E0224C062504E0214C072501E00024C9
:1015200025467AB1012606FA01F16DB2284606FA7F
:1015300005F55A6811435960214600F003FB194B29
:101540001D6070BD01290AD04468174A382606FB81
:10155000042292F8354030329279E24215D10122CC
:1015600002FA01F6D1F1010138BF002102FA01F1BE
:101570005C6824EA06045C6003685B68194204D175
:1015800002FA05F5074BC3F8805070BD000001401A
:101590009514000000800940D1140000A914000037
:1015A000BD14000000E100E0B40200102DE9F04F8E
:1015B0000368634A87B0934223D00FDCA2F58042D0
:1015C000934239D15F4BD3F8A82122F0C002C3F86F
:1015D000A821D3F8A82142F040021DE05A4A9342C4
:1015E0001DD002F58042934226D1564BD3F8AC2150
:1015F00022F44022C3F8AC21D3F8AC2142F480227B
:1016000018E0504BD3F8A82122F44072C3F8A82167
:10161000D3F8A82142F48072C3F8A8210CE0494B0A
:10162000D3F8AC2122F44032C3F8AC21D3F8AC217A
:1016300042F48032C3F8AC21444B0F01D3F8009040
:10164000B9FBF7F307FB13971FFA83FC002F58D061
:10165000012400238DE818008A464E460291770047
:101660004FEA860BE2B20497CDF814B0D0460025BD
:10167000049BEFB2002B039703DAB3FBF8F31B09CB
:1016800003E0059FB7FBF8F35B090133C3F34F0396
:10169000039F002B08BF012317B1012B98BF022322
:1016A00005EB040B0BFB03FB4FEACB0BB6FBFBFB81
:1016B0000BF1010BC1EB5B0B029FBBF1000FB8BF3D
:1016C000CBF1000BBB4507DA8B450DD0039FCDF85E
:1016D00008B0019200979C460135EBB293428844D2
:1016E000C6D3019A002304E0039D9C460291009515
:1016F00001230F2C07D001344E448A441BB90192B8
:10170000ADE7012200970368197B41F0800119734E
:101710000368CCF30721197103685FFA8CFC009908
:1017200083F800C0036841EA0212D2B283F828208D
:1017300003681A7B02F07F021A7307B0BDE8F08FCE
:101740000000014000C00F4000800940CC000010A4
:1017500010B502680346117DC907FCD51078596899
:10176000084A382404FB01225168C0B2013108D074
:101770005169043252680A601B685A6842F00102DB
:101780005A6010BDB402001010B5436838225A43A5
:1017900010498B18DC6901340AD01A6B1C331268AB
:1017A0005B681A4214D10368187DC0F3801010BD25
:1017B00002683033127D12F0200F03D000221A711C
:1017C000012010BD18790F288CBF0020012010BD0A
:1017D000002010BDB402001038B504460D46204666
:1017E000FFF7D2FF0028FAD02368EDB21D706368BE
:1017F000044A382101FB032393F83420013283F893
:10180000342038BDB40200102DE9F84F98463A4C08
:1018100003680546A34218BF00240E461746D0F8B9
:1018200004901CB1237C03F03F032374DFF8D4A0A1
:10183000382303FB09A24FF0FF31D16151606A6880
:10184000002103FB02A3284683F835100A46FFF760
:1018500049FE002E4ED02949384600F00BFB28499E
:101860008346404600F006FBB31E012B17D8B8F1A3
:10187000FF3F3DD0204B984209D144B1237C4046E4
:1018800043F0800323741E4900F0C6FA30E038208C
:1018900000FB09A041461C3000F067FA28E0012E49
:1018A00028D17B1C26D02B6807221A72124B9B452D
:1018B0000AD14CB1237C384643F0400323740F49CE
:1018C000BDE8F84F00F0A8BA382404FB09A0394657
:1018D0000430002200F04CFA6B68012204FB03A4E0
:1018E00084F8352028460021BDE8F84FFFF7FABDFF
:1018F000032ED5E7BDE8F88F00000140BC200100B1
:10190000E0200100B40200102DE9F04104460F462A
:1019100008464749164600F0B9FA4649054630469A
:1019200000F0B4FA0146284600F092FA424B054610
:101930009842206017D009D8A3F5804398421FD160
:101940003E4BD3F8C42042F0080217E03C4B9842CB
:101950000FD003F58043984212D1384BD3F8C420FE
:1019600042F000720AE0354BD3F8C42042F0100276
:1019700004E0324BD3F8C42042F08072C3F8C42094
:10198000236801221A7223684FF00008C3F804800C
:1019900020464FF41651FFF709FE236803221A73FD
:1019A0003846234900F038FA3046224900F034FA2C
:1019B0007A1C03D038464146FFF70DFD731C03D057
:1019C00030460021FFF707FD1B4B9D420FD005D885
:1019D000A3F580439D420ED100230BE0184B9D429E
:1019E00007D003F580439D4205D1032302E0012384
:1019F00000E0022363606268124B382101FB023071
:101A00004FF0FF324260606801FB00332046DA612C
:101A100000211346FFF7F8FE0B4B9D4206D10B4BFE
:101A200001221A6020680A4B616803C3BDE8F08197
:101A300070210100042101000000014000C00F409E
:101A400000800940B402001000C00040AC02001049
:101A50009403001008B5114B1A68EAB90121196006
:101A60000F4BD3F8C40040F40000C3F8C400A3F542
:101A7000D0231A670B4A0220126858600A4892085D
:101A8000B2FBF0F2013ADA6004205960074900F035
:101A900059F8074B10221A6008BD00BF9C030010C4
:101AA00000C00F40CC00001040420F00FD2000009D
:101AB00000E100E008B5044B1B680BB9FFF7CAFF53
:101AC000024B986808BD00BF9C030010004009400D
:101AD000034B98615A6942F001025A61704700BF96
:101AE00000400940024B5A6922F001025A617047D6
:101AF00000400940014B01221A6070470040094034
:101B00000649074A074B9A42BEBF51F8040B42F8F8
:101B1000040BF8E7044880470448004710280100F8
:101B2000C80000102C020010851B000021010000DD
:101B3000FEE7FEE7FEE7FEE7FEE7FEE7FEE7FEE77D
:101B4000FEE7FEE710B50C4A946892682346B2F1AE
:101B5000805F0DD2094B04F170420432D25843F831
:101B6000042F074A9342F6D1034A4FF08053936003
:101B7000103043F8201010BD00ED00E0FCFFFF0F17
:101B8000C0000010264B2022C3F8A021D3F8A021CA
:101B9000910603D5D3F8A0215206FBD50222C3F843
:101BA00004210022C3F8A8210120C3F8AC210B2294
:101BB000C3F80C01AA21C3F884205522C3F88C1065
:101BC000C3F88C20C3F88000C3F88C10C3F88C20B5
:101BD000134AD2F888305B01FAD50323C2F880306B
:101BE000AA23C2F88C305523C2F88C30D2F8881062
:101BF0000B4B11F0407FF9D00522C3F80821094AA8
:101C0000C3F8C4200022C3F8C8211A6822F4704225
:101C100022F03A0242F4405242F03A021A6070470F
:101C200000C00F40DE87280410B5036804462BB9B6
:101C3000C06800F05AFA01236060236010BD10B53F
:101C40000446006820B1E06800F04FFA6368C01AEB
:101C500010BD10B50446FFF7F2FFA3681844002337
:101C6000A060236010BD10B58468FFF7E8FF204432
:101C700010BD08B5FFF7F7FF4FF47A7390FBF3F050
:101C800008BD10B50446C06800F02FFA002360605C
:101C9000A36010BD002310B5036043608360044659
:101CA00000F028FAE0602046FFF7EBFF204610BD69
:101CB00000B599B072B61749684600F072F806A8E8
:101CC000154900F06EF80CA8144900F06AF812A843
:101CD000134900F066F8019A039B96201A60079A50
:101CE0000A9B1A600D9A109B1A60139A159B1A6032
:101CF00000F022FA019A049B96201A60079A099B29
:101D00001A600D9A0F9B1A60139A169B1A6000F0C6
:101D100013FAE0E732C0092034C0092035C0092099
:101D200037C009200FB407B5054B04AA1B6852F849
:101D3000041BD86801920BF0C5FB01200AF010FAD1
:101D4000DC01001070B50E4604461546FFF700FB97
:101D5000013609D020460021FFF714FB2046294612
:101D6000BDE87040FFF70BBB70BD0322FFF7EABF71
:101D700070B50E4604461546FFF7EAFA01360FD055
:101D800063680DB1E26800E022692046012113601A
:101D9000FFF7F8FA20460221BDE87040FFF7EFBADE
:101DA00070BD0022FFF7E4BF00F074B910B504461F
:101DB00000F070F920B12046BDE8104000F05BB99A
:101DC00020704FF0FF3010BD30B58BB0044601A835
:101DD000FFF7ECFF002388B9054606AB03EB45008F
:101DE0000C496A460AF0F6FD009B63550135062D45
:101DF000F3D1237823F00103237008E002226270FC
:101E0000F722A270F0222370E270237163710BB08D
:101E100030BD00BFDC21010010B50446013001D106
:101E200010BD0C310B685A1C0BD0A342F9D12046CF
:101E30008968FFF7B7FA20460221BDE81040FFF796
:101E4000CABA0248BDE81040FFF76CBFE0210100AC
:101E5000884208B50AD0431C07D0013106D0044897
:101E6000FFF760FF4FF0FF3008BD084608BD00BF18
:101E7000F12101000B685A1C05D0834201D148684A
:101E800070470C31F6E7184670470000421C10B549
:101E9000044607D0FFF7EEFF431C044602D1024878
:101EA000FFF740FF204610BD02220100044B1B68D3
:101EB00023B904480449054AFFF726BD704700BF0F
:101EC000AC0200109403001002C0092003C00920D6
:101ED000022808B54FF000030ADD084AC11E52F877
:101EE000210042F8213028B103685B68984708BD9B
:101EF000184608BD4FF0FF3008BD00BFA00300101A
:101F0000022870B50C4615460FDC0E4B1B680BB94A
:101F1000FFF7CCFF6619B44205D00B4814F8011B3B
:101F2000FFF75AFCF7E7284670BD084B033853F813
:101F3000200018B103681B68984770BD4FF0FF3050
:101F400070BD00BFAC02001094030010A00300108D
:101F5000022810B50C460ADC0B4B1B680BB9FFF7C7
:101F6000A5FF0A48FFF7F4FB2070012010BD084BC5
:101F7000033853F8200018B103689B68984710BDD8
:101F80004FF0FF3010BD00BFAC02001094030010F2
:101F9000A0030010022808B508DD074B033853F8EA
:101FA000200028B10368DB68984708BD012008BD00
:101FB0004FF0FF3008BD00BFA0030010022808B595
:101FC00008DD074B033853F8200028B103681B696C
:101FD000984708BD002008BD4FF0FF3008BD00BF86
:101FE000A0030010022808B504D84FF400534B603A
:101FF000002008BD0AF0AEF8092303604FF0FF305F
:1020000008BD0000084B1B681844EFF3088290429B
:1020100005D3064B0C221A604FF0FF307047024A7E
:1020200010601846704700BFD00000107C1C0010E4
:1020300008B50A4C0546236898680AF053F92368E6
:10204000D8680AF04FF9FFF7AFFE08B100F008F8C2
:1020500005B9FEE7FFF72CFEFBE700BFDC0100102F
:1020600030B585B06D46182420462946ABBE0446DF
:10207000204605B030BD37B52123009001936D4651
:1020800040F2011420462946ABBE0446204603B068
:1020900030BD0000024B186800F00100704700BF1F
:1020A000F0ED00E038B503680446DB6898476368E4
:1020B0005A68236812B99B68984738BD5B681568F1
:1020C0009847281A0028636809DC5A6891685960A3
:1020D00063681B68002BEAD050689847E7E75A68A6
:1020E000216810680B69984738BD08B503685B68BC
:1020F000984708BD00487047542201000148FFF787
:10210000D1BF00BF5422010038B50446FFF7D2FC0E
:102110000546FFF7CFFC401BA042FAD338BD0000B4
:1021200008B504490FF0E8FC0FF036FEBDE80840A2
:10213000FFF7EABF002474494FF47A735843FFF75E
:10214000E3BF70B5037A0446032B04D0042B0CBF05
:102150000A25002500E00C2504F10C0393E8070094
:1021600000F040FAE37E023005447BB104F1240321
:1021700093E8070000F036FA04F13003064693E8CE
:10218000070000F02FFA3044061D3544236C0BB9CC
:10219000A36C3BB104F1400393E8070000F022FA7E
:1021A00002300544E36C0BB9636D33B14C3494E8F1
:1021B000070000F017FA02300544284670BD000001
:1021C000F7B50646019010460D461446FFF7B9FFD5
:1021D000074600F06FF9A8426BDC01A8102100F05F
:1021E00093F9019D3946284600F02AF92844257ABA
:1021F0000190042D01A805D1304900F0A3F901A8F0
:10220000294604E02E4900F09DF901A8032100F0C1
:102210007BF90025A37E6FF3070563F34105E37E99
:10222000003318BF012363F382053BB194F83D30BE
:1022300063F3C40594F83C3063F34515236C0BB984
:10224000A36C0BB145F08005E36C0BB9636D0BB16A
:1022500045F0400501A8E9B200F056F901A8218B2C
:1022600000F058F904F10C030ECB01A800F07EF940
:10227000E37E5BB104F124030ECB01A800F076F9F4
:1022800004F1300301A80ECB00F070F92A0605D541
:1022900004F1400301A80ECB00F068F96B0605D5E8
:1022A0004C3401A894E80E0000F060F90198801BFE
:1022B00001E06FF0010003B0F0BD00BF5C2201003F
:1022C00061220100F7B5074602AC68460E4644F8A5
:1022D000082D00F013F9C0F30310022815D1009D5A
:1022E00001A9284600F0F8F8019B0544012B009550
:1022F0000CDD684600F002F9C0F3C0103870684683
:1023000000F0FCF83070012000E0002003B0F0BDC8
:1023100037B5012904464FF0000301900DDD62F34B
:102320000713194601A800F0EFF8019D0021284687
:1023300000F086F82844001B01E06FF0010003B0B4
:1023400030BD0C22FFF7E4BF2DE9F7431F460D9B7C
:1023500000258046684600930E469146019500F0A0
:10236000CDF82C4660F307042309032B2DD1C4F3C9
:10237000C003009D88F80030C4F34103C4F3000497
:102380003360284689F8004001A900F0A5F8019BB8
:10239000054400951D44044669460A982A4600F003
:1023A00007F998B1009BEB1A002B0FDB3368002B69
:1023B00003DD684600F09AF83880009B0C9AED1A0D
:1023C00015600B9A0124136000E02C46204603B0F0
:1023D000BDE8F083F7B5054602AC68460F461646E1
:1023E00044F8083D00F08AF8002360F30703C3F3C4
:1023F000C002C3F303133A702B70009D01A9284655
:1024000000F06AF8019B0544012B009504DD684645
:1024100000F06CF83080012003B0F0BD30B5074CFF
:10242000002322688B4203DAD55C01330570F9E79B
:102430000029A8BF52182260084630BDA804001029
:1024400010B500220B4B0B40002B03DA013B63F06D
:102450007F030133802491FBF4F1DBB2002902F108
:102460000102C8BF23438418002904F8013CE9DCB9
:10247000104610BD7F000080F7B5002407460E46C9
:102480000C6001250134052C11D00DF1070001214C
:10249000B84701280BD19DF80730326803F07F015F
:1024A00005FB01221B0632604FEAC515EAD420461F
:1024B00003B0F0BD431C7F2B01DC02307047B3F545
:1024C000804F01DA03307047024A9342D4BF043090
:1024D00005307047FEFF1F00024B18600248FFF7EF
:1024E000CBBF00BFA80400101D24000003681978AA
:1024F0005A780233036002EB0120704703680246FA
:1025000013F8010B136070470368197003680133F7
:102510000360704703684FF4807291FBF2F21A7007
:102520000268531C0360064B0B40002B03DA013B8F
:1025300063F0FF0301335370036801330360704796
:10254000FF00008070B5044608460E460AF0C3FA44
:10255000054629462046FFF7DDFF2A46206831461A
:102560000AF054F823681D44256070BD30B585B06D
:1025700004AC04E90E00029C0546002C01990CDD18
:102580002146FFF7C7FF2246286803990AF03EF864
:102590002B681C442C6005B030BD21B105B0BDE8EE
:1025A0003040FFF7CFBF05B0BDE83040FFF7B2BF06
:1025B0000B6870B5D31A012B05460C46164601DC94
:1025C00000200CE00846FFF791FF686023681A18A6
:1025D0009642F5D3AB6023681844206001200023A5
:1025E0002B6070BD84B004AB03E90700019810B103
:1025F00004B00AF070BA029804B0704770B504686D
:102600000E4624B120460AF066FA054601E08468C9
:10261000456830460AF05FFA854209D120463146C6
:102620002A460AF060FAD0F1010038BF002070BDE0
:10263000002070BD30B585B001AC84E80E000546C1
:1026400094E80700FFF7CEFF089B02301844002DE6
:10265000C8BF023005B030BD2DE9F04F85B0149EE3
:1026600010AC00968B4603908046924618461F4653
:1026700094E80E00FFF7DEFF8146FFF71BFF584589
:102680004FF000052BDC032363F307156AF3C30542
:102690009DF8383067F3420563F30005E9B203A8FB
:1026A000FFF732FF039D49462846FFF7C9FE94E82D
:1026B0000E002844039003A8FFF758FF002F04DD05
:1026C00003A8BDF83C10FFF725FF03981399324685
:1026D00009F09CFF03983044C8EB000001E06FF064
:1026E000010005B0BDE8F08F37B5032905464FF06E
:1026F0000004019016DD62F3071463F3C304E1B232
:1027000001A8FFF701FF019C02212046FFF798FE78
:1027100020440190BDF8181001A8FFF7FBFE0198B6
:10272000401B01E06FF0010003B030BDF8B5064674
:102730000F4602250024B4420ADA0C2303FB04737B
:1027400093E80700FFF74EFF033005440134F2E73A
:102750002846F8BD2DE9F74F0C9F0D9D8B46019043
:1027600029460646384690469946FFF7DFFF8246DF
:10277000FFF7A0FE58454FF000042BDC082363F35D
:10278000071468F3C304012363F34204E1B201A810
:10279000FFF7BAFE019C51462046FFF751FE204448
:1027A0000190494601A8FFF7B5FE0024BC420EDAAD
:1027B0000C2303FB045301A80ECBFFF7D7FE0E9B9F
:1027C00001A813F82410FFF79FFE0134EEE70198EB
:1027D000801B01E06FF0010003B0BDE8F08F2DE930
:1027E000F34799460A9B824602AC684688461546DE
:1027F00044F8083DFFF782FEC0F30310092822D1F8
:10280000009E01A93046FFF767FE019B0644012B9D
:10281000009606EB03071ADD6846FFF767FE002304
:10282000AAF800002B60009BBB420AD22E684645E6
:102830000BDC731C2B606846FFF760FE49F826002E
:10284000F1E7012003E0002001E04FF0FF3002B08B
:10285000BDE8F08780F309887047EFF3098070477F
:10286000684680F3098841480078C00714BF0220F9
:10287000032080F314887047DFF8F4C0EFF305837A
:102880001B0618BF6047EFF31483DB0708BF6047E0
:1028900000DF7047DFF8DCC0EFF305831B0618BFCD
:1028A0006047EFF31483DB0708BF604700DF704722
:1028B000EFF30980816911F8021CF9B990E80F1053
:1028C000E047EFF3098C8CE807002B4B93E80600F8
:1028D000914200F0108039B12CE9F00FC1F828C006
:1028E0000CB401F021FA0CBC1A60D2F828C0BCE884
:1028F000F00F8CF309886FF0020E704710B51F4A75
:102900001268914200F20A801D4C54F8214090E870
:102910000F10A047EFF3098C8CE80F0010BD01F0F9
:1029200091F9154B93E80600914200F01180EFF306
:10293000098C2CE9F00FC1F828C00CB401F0F4F9AF
:102940000CBC1A60D2F828C0BCE8F00F8CF30988E0
:102950006FF0020E704701F0C7F9FFF7E2BF01F018
:10296000C1F901F0C1F9FFF7DCBF00006A220100E4
:102970004D39000067390000E00F00100000000032
:10298000FCFFFFFF436AC26A23F0030313445A07A4
:1029900048BF043B4FF0807270B503E90600A3F115
:1029A0004004A3F14402A3F10C05002642F8046F91
:1029B000AA42FAD1C26943F8202CC3788462012B61
:1029C000016302D0C36A014A1A6070BDA52E5AE2A3
:1029D000836A19627047836A19625A627047FEE718
:1029E000FFF766B908B1FFF763B970470449054AB4
:1029F000C1F1805303F5F8439360D160704700BF85
:102A0000801C0010D40000100020002104460D4658
:102A1000094809F088FB09F069FD2046294600F0C5
:102A200091F8FFF7E3FF0548002100F029F900F0D5
:102A30009DF809F095FB000085C40000D40000104B
:102A400038B1830704D10378002B18BF00207047EA
:102A50000020704700B5DFF80CC000DFDFF808C0C9
:102A600000DFFEE74D2C0000652C000030B50C4C5B
:102A700000222368254633B11C89A14203D31A469C
:102A8000091B1B68F7E789B20360018113B11C8938
:102A9000611A19810AB1106030BD286030BD00BFD5
:102AA000980F00100C4900220B6823B1834205D017
:102AB0001A461B68F9E74FF0FF30704703680AB108
:102AC000136000E00B6003681BB101891A890A4496
:102AD0001A810020704700BF980F0010431C11D0CE
:102AE0000B4B984211D80B4B4FF47A711B685A1E4E
:102AF00001FB0020B0FBF3F04FF6FE73984228BFB5
:102B0000184670474FF6FF7070474FF6FE707047DB
:102B100000093D006C22010038B5084C257855B9F4
:102B200001F00EFA064BFF221B6828469A70FFF749
:102B300059FF01232370002038BD00BF940F0010FF
:102B4000E00F001010B5EFF305845CB9EFF31484C7
:102B5000E40703D4BDE81040FFF7DEBFDFF808C08C
:102B600000DF10BD822010BD192B000010B588B009
:102B7000EFF3058434BBEFF3148404F00304022C58
:102B80000CD0032C16D0012C1ED008AC84F309887D
:102B90000F4C2478E40705D5022404E00C4C24787B
:102BA000E4070BD4032484F31488BFF34F8FBFF3DF
:102BB0006F8F03E0064C2478E40705D4DFF814C0D7
:102BC00000DF02E0822000E0FF2008B010BD00BF5F
:102BD0006A220100B13100002DE9F843894604461C
:102BE00060B1036853B1B0F8048008F103039BB2ED
:102BF000062B03D883680BB1C2682AB98020FFF77F
:102C0000F1FE0020BDE8F8834363C26300F11005C4
:102C100001F0AEF80B4E471E46F8275008F10401AC
:102C20002268E074C9B22846C4F82C9001F0B4F8C8
:102C3000284601F0CFF856F82700034A836A5A6302
:102C4000BDE8F883300D0010552A000008B501F0EA
:102C5000FDF818B1024B013853F8200008BD00BF41
:102C6000300D001008B5FFF7EBFE38B1C07801F069
:102C70002FF9FF2814BF0020812008BD802008BD47
:102C800010B5EFF3058474B9EFF31484E40706D4A8
:102C9000064C24781CB9BDE81040FFF79DBFDFF853
:102CA00010C000DF10BD002010BD00BF9C0F001041
:102CB000D92B000008B530B1FFF710FF80B201F04A
:102CC000CBF9402008BD08BD10B5EFF305841CB951
:102CD000DFF808C000DF10BD822010BDB52C000059
:102CE00010B508B103680BB980200AE04368002BD7
:102CF000FAD0012988BF862003D8094C246824B95A
:102D00008120FFF76FFE002010BD1C79002CF7D149
:102D1000012418611C715971DA60184610BD00BF9A
:102D20008C0F001038B58307044618D1B8B1084697
:102D3000FFF7D4FE0546A0B12379012B06D0022B64
:102D400011D12046FFF7AEFE68B902E002232371DD
:102D5000608120462946FFF789FE002038BD80208B
:102D600038BD862038BD812038BD830706D128B103
:102D70000169C3680A68194610467047002000219F
:102D800070470000F8B5134B1C681F460CB323892D
:102D9000013B23812389E3B90F4B26681D683E6000
:102DA00055B12B78012B07D1284600F02FFD18B123
:102DB0002846214600F02EFD6379012B04D12046E0
:102DC0006189FFF753FE01E0012323710EB1344600
:102DD000E0E7F8BD980F0010900F001010B5EFF36A
:102DE000058474B9EFF31484E40706D4064C247800
:102DF0001CB9BDE81040FFF773BFDFF810C000DF5B
:102E000010BD002010BD00BF9C0F0010E12C000081
:102E100010B5EFF305841CB9DFF808C000DF10BD62
:102E2000822010BD252D000010B504460846DFF8AD
:102E30000CC000DF84E80300204610BD6B2D0000AD
:102E400038B50C46FFF7FCFD034648B1220C1204CE
:102E500032B9058BD978A0B200F0CAFA284638BD3D
:102E60004FF0004038BD00002DE9F74F020C12046E
:102E700003460C46002A2DD1084601935BB1FFF7AB
:102E80002DFE019B81B2012298B200F08BFA02283C
:102E9000019B0FD112E0FFF721FE019B81B21A4680
:102EA0004FF6FF7000F07EFA022803D10F4B1B682B
:102EB0005B8B03E024B10023402203E0082201E001
:102EC000234622464FF00008C14614461D464E4692
:102ED0004F4603E0002586242E462F4620462946ED
:102EE00032463B4603B0BDE8F08F00BFE00F001054
:102EF00038B50C46EFF3058181B1FFF7A1FD03461C
:102F000048B1220C120432B9058BD978A0B200F076
:102F10009DFA284638BD4FF0004038BD2146DFF805
:102F200008C000DF38BD0000412E000030B5044667
:102F300008461146EFF3058515B18223236004E0AE
:102F4000DFF80CC000DF84E80700204630BD000039
:102F5000692E000010B520B98020FFF743FD002046
:102F600010BD0468002CF7D02378002BF4D1204644
:102F700000F00DFD204610BD70B510F003060446AC
:102F80000D4611D180B10378032B0DD10846FFF710
:102F9000A5FD81B2204600F059FD012806D1002D83
:102FA0000CBF8120C12070BD802070BD304670BD37
:102FB000820708B50AD148B10378032B06D100F087
:102FC000EFFCFF2814BF0020812008BD802008BD31
:102FD00010B5EFF3058474B9EFF31484E40706D455
:102FE000064C24781CB9BDE81040FFF7B3BFDFF8EA
:102FF00010C000DF10BD002010BD00BF9C0F0010EE
:10300000552F000010B5EFF305841CB9DFF808C098
:1030100000DF10BD822010BD792F000010B5EFF346
:1030200005841CB9DFF808C000DF10BD822010BD88
:10303000B12F000038B520B98020FFF7D3FC002065
:1030400038BD0468002CF7D02578002DF4D1B1F5F7
:10305000803FA8BF8620F0DA204689B200F058FDF4
:10306000204638BD38B510F0030504460FD170B1C5
:103070000378022B0BD10846FFF730FD81B22046C2
:1030800000F090FD012805D06088013038BD4FF078
:10309000FF3038BD284638BD10B510F003040CD100
:1030A00058B10278022A08D142884FF6FF739A423B
:1030B00005D000F061FD204610BD802010BD8120AC
:1030C00010BD10B510F0030407D130B10378022B06
:1030D00003D100F023FD204610BD802010BD00006C
:1030E00010B5EFF3058474B9EFF31484E40706D444
:1030F000064C24781CB9BDE81040FFF79BBFDFF8F1
:1031000010C000DF10BD002010BD00BF9C0F0010DC
:103110003530000010B5EFF305841CB9DFF80CC0A2
:1031200000DF10BD4FF0FF3010BD00006530000023
:1031300010B5EFF305849CB110F003040CD158B125
:103140000378022B08D142884FF6FF739A4205D0CC
:1031500000F044FD204610BD802010BD812010BD30
:10316000DFF804C000DF10BD9930000010B5EFF3A8
:1031700005841CB9DFF808C000DF10BD822010BD37
:10318000C330000010B5044618B1016809B14068A9
:1031900020B98020FFF726FC002010BD0378002B0B
:1031A000F7D10431890089B200F086FA606810BD59
:1031B00038B5114B1C781D46E4B921460F48FFF77E
:1031C000E1FF0F4B214618600E48FFF705FD0E4B3F
:1031D00021461860204600F041FE0C4B1B689B6A9C
:1031E000203383F30988094B00221A6000F016FF90
:1031F00001232B70002038BD9C0F00101801001017
:10320000900F0010200100108C0F0010E00F001034
:1032100070B50E461546044688B10378012B0ED1D1
:103220001046FFF75BFC314682B2204600F052FAAE
:10323000012806D1002D0CBF8120C12070BD802047
:1032400070BD002070BD2DE9F04F0C4685B0804662
:10325000E8B10378012B1FD10846FFF73FFC02A914
:1032600082B2404600F07EFA012806D10020002CF0
:103270000246034618BF402003E0002002460346F2
:103280001020029904460D4616461F4608E0802489
:1032900005460646074603E0002580242E462F46B5
:1032A0002046294632463B4605B0BDE8F08F000077
:1032B00010B5EFF3058474B9EFF31484E40706D472
:1032C000064C24781CB9BDE81040FFF75BBFDFF85F
:1032D00010C000DF10BD002010BD00BF9C0F00100B
:1032E0008531000070B504460E461546EFF30582A1
:1032F0008AB170B16DB90378012B0AD100F086FA5A
:1033000028B12046314600F085FA284670BD81205C
:1033100070BD802070BD2A46DFF804C000DF70BD9C
:10332000113200007FB5044616460846EFF30581CA
:10333000A9B101AD00B10AB180230AE00378012BE5
:10334000FAD102A900F06DFA042801D0019601E03B
:103350001023019395E8070084E8070005E0114673
:10336000DFF80CC000DF84E80700204604B070BD21
:10337000473200007FB50A4B03A819684FF0FF32AF
:10338000FFF7D0FF039B102BF5D101A80499FFF79D
:103390004BFD019B002BEED002989847EBE700BF56
:1033A000900F001070B50346104C4AB12268158B7F
:1033B00000EA050686420DD125EA0605158307E0D9
:1033C0002268158B284007D025EA03035083138316
:1033D000022070BD062200E00522206843830846D3
:1033E000114600F019FD012070BD00BFE00F001074
:1033F00010B5154B013953F821401CB3238B62786B
:103400001843062A2083638B04D100EA03029A4200
:1034100018D105E0052A15D110EA030212D0628303
:1034200020EA03002083204600F010F90123204603
:103430006370628B0821FFF7CEFA2046BDE810408A
:1034400000F0C8BC10BD00BF300D001008B5074B20
:103450000139024653F8210030B1114600F00AF953
:10346000BDE8084000F0DCBB08BD00BF300D001017
:1034700010B5038B42781943062A04460183438B17
:1034800004D101EA03029A4219D105E0052A16D1B6
:1034900011EA030213D0428321EA0301218320466B
:1034A00000F0D4F80123204663700821628BFFF7F7
:1034B00092FA21460248BDE8104000F003B810BD62
:1034C000B80F001030B502788C78013A4368D2B258
:1034D0002BB19D78A54202D318465B68F8E7022A13
:1034E0004B60416003D803B19960886030BD002310
:1034F0008B6030BD43685A6842600278013A022A04
:103500004FF0000205D8596809B188605A609A6086
:1035100000E05A6018467047034B5A684260002228
:1035200082605860704700BFB80F001010B5114B93
:10353000DA680AB19A8A0CE000248A1AC460D8605A
:1035400003619A82848210BD002CF5D0A38A1A44AC
:1035500023468A42DC68F7D3C460D860C46803613C
:1035600004B12061521A92B28282998A8A1A9A828E
:1035700010BD00BFA00F001038B5194DEB68002B2F
:103580002DD0AB8A013BAB82AB8A002B27D1144AEA
:10359000D46824B3A26842B161685160626812B114
:1035A000A168916063600023A3600E482146FFF785
:1035B00089FFA38AAB826378042B04D10A4B1A6873
:1035C000E38A1344A38201236370E368EB60E2683B
:1035D000002312B102491161E3602361D4E738BDD1
:1035E000A00F0010B80F00101C100010836833B13A
:1035F00042685A60436863B182689A607047054BBD
:103600005A68824202D142685A6070470AB1134632
:10361000F6E77047B80F001038B58468054624B93E
:103620004378012B0ED1084C03E023780BB9A46832
:10363000FBE72846FFF7DAFF20462946BDE8384079
:10364000FFF740BF38BD00BFB80F001003697BB162
:10365000C268DA60C26842B19A8A818A0A449A8250
:10366000C26813610023C36000E09A8200230361F3
:103670007047000030B50F4BDD78EFF3108372B662
:103680000C4A9378AB4207D20133937013785C1CD9
:10369000AC4208BF0024147062B6AB4204D202EB05
:1036A000C3035860996030BD0220BDE83040FFF789
:1036B00097B900BFAC0C00100123103903708908C2
:1036C0000023437083704360038143818381C18100
:1036D00070470000F8B50C4641680346174689B1AB
:1036E0004278012A0ED1FFF705FF10210546224638
:1036F000FFF771F92846FFF7A9FF284600F06AFB9B
:103700000020F8BD9D89D889854214D137B3144D66
:1037100021B118462968FFF7D5FE05E02E68022280
:103720005E607160B3605A702B683846DC610821B6
:1037300000F072FB12E01A89111D43F82140EFF3EB
:10374000108172B601359D8162B6013292B2824219
:103750004FF0000014BF1A811881F8BD0120F8BD98
:10376000E00F001038B5838904461546002B36D08B
:103770004389043350F823300B604389C2890133F5
:103780009BB29A42438104BF002343814368EBB15B
:103790004378022B1AD1FFF7ADFE00210546FFF753
:1037A00017F92389EA69191D44F82120E2890133B8
:1037B0009BB29A42238108BF0023284608BF238179
:1037C000FFF744FF284600F005FB06E0EFF3108307
:1037D00072B6A389013BA38162B6002038BD82B1D5
:1037E0004268094B1AB11968FFF76CFE05E01B68C7
:1037F00043605A609860012343702846082100F016
:103800000BFB012038BD00BFE00F0010C28980898A
:10381000101A704708B5FFF72DFFBDE8084000F00B
:10382000FFB910B583890446EBB14389043350F8DE
:1038300023300B604378022B04D10021FFF71AFFDD
:1038400000F0EEF9EFF3108372B6A389013BA38178
:1038500062B66389E28901339BB29A42638104D1E3
:103860000023638101E0184610BD042010BD000054
:1038700070B5436804460E46002B4AD04578022DA9
:103880001CD0032D0AD0012D5DD1FFF733FE10218E
:1038900004463246FFF79FF8657034E0084600F0B2
:1038A00055F8054600284ED02046FFF723FE29464E
:1038B0000446FFF78DF80123637024E0FFF71AFE3A
:1038C00000210546FFF784F82389EA69191D44F8A9
:1038D0002120EFF3108272B6A2890132A28162B672
:1038E000E28901339BB29A42238104BF00232381E2
:1038F000012328466B70FFF7A9FE13482946BDE84F
:103900007040FFF7DFBD2046FFF7A0FE0E482146BE
:10391000F5E78189C289914210D20389181D44F8C4
:103920002060EFF3108072B60131A18162B60133DD
:103930009BB2934208BF0023238170BD0320BDE8E2
:103940007040FFF74DB870BDB80F0010EFF3108155
:1039500072B6036801F001010BB11A68026001B987
:1039600062B61846704781420DD3436899420AD225
:10397000EFF3108272B603680B601346DB07016039
:1039800003D462B601E00120704700207047032392
:1039900003700023437043804360836070470000DE
:1039A0002DE9F84345880446002D48D0254F82680C
:1039B0003B689A4243D1013DADB2458015B100202C
:1039C000BDE8F8833B684278DFF87C809A704668EF
:1039D00026B3FFF78FFD294606464FF00109FEF793
:1039E000F7FF3046FFF732FEA4F80290A660B378E6
:1039F00063703968D8F804308A789B789A421AD272
:103A00004046FFF75FFD40463146FFF75BFD3B68F0
:103A1000284683F8019086F801900DE0D8F804302C
:103A200039689A788B789A42C9D94046FFF74AFD9F
:103A30003B6801225A70304600F0CCF9BFE7FF2006
:103A4000BDE8F883E00F0010B80F001070B50E4607
:103A500041880446144D21B92B6883609B784370DC
:103A600003E083682A68934203D10131618000201A
:103A700070BDB6B192784178914203D29A70806855
:103A8000FFF7CAFD626822B120462968FFF71AFDD8
:103A900003E02B6863605A609C603046092100F0A7
:103AA000BBF9012070BD00BFE00F0010034B0022E6
:103AB0001A60034A1268DA80704700BFD00F001006
:103AC0007822010008B50F4B59680F4B1A688A42DB
:103AD0000E4A05D0D88819601168013801449980D0
:103AE0009988138899420BD1074B002205481A6028
:103AF000FFF700FDBDE8084001460248FFF7E2BCC1
:103B000008BD00BFB80F0010D00F00101C1000102F
:103B100002230370002343604180704770B5044660
:103B2000656885B12046FFF7E5FC00210546FEF7F4
:103B30004FFF2846FFF78AFD01236B700C4829468A
:103B4000FFF7C0FCECE70A4843686BB1094E9A786E
:103B500031688B789A4207D9FFF7B4FC33680122A9
:103B60005A70284600F036F90020207070BD00BF62
:103B7000B80F0010E00F001010B5426862B1FFF7F7
:103B8000B9FC01210446FEF723FF2046FFF75EFD46
:103B9000204600F01FF902E04288013242800020F6
:103BA00010BD000010B542880C461AB1013A42809F
:103BB000002010BD71B14168074A19B11168FFF7C3
:103BC00081FC03E01268426051609060204607214A
:103BD00000F022F9012010BDE00F001008B500210F
:103BE000FFF748FDBDE8084000F01AB810B542687C
:103BF0007AB1FFF77FFC0446FFF728FD01216170D1
:103C00002046FEF7E5FE21460448BDE81040FFF7D8
:103C100059BC42880132428010BD00BFB80F00106D
:103C2000054B1B7823B9054B4FF080521A60704743
:103C3000034B01221A707047DD0F001004ED00E005
:103C4000DC0F001038B5194B01211A68184D51705E
:103C50001868FFF761FC6C78AA78154BEAB103EBA2
:103C6000C403586802781AB91989FFF701FC07E004
:103C7000012A03D19968FFF7FBFD01E0FFF7B6FFCA
:103C8000EB7801349C4208BF0024EFF3108372B636
:103C9000AB78013BAB7062B6DEE75C700548FFF7BE
:103CA00029FCBDE8384000F08DB800BFE00F0010DF
:103CB000AC0C0010B80F0010084B4FF0FF301A6822
:103CC000074B1A6000225A60072243F8042CD3F8ED
:103CD0000C2D42F07F42C3F80C2D70477422010076
:103CE00014E000E07047000008B50C4B01211A6891
:103CF00051701868FFF710FCFFF7E4FE084B1A68D4
:103D000001321A60FFF738FCFFF73CF80548FFF76F
:103D1000F1FBBDE8084000F055B800BFE00F00100F
:103D20001C100010B80F0010084B1B68DA78012A2D
:103D30000AD0DA6A9B6A9A4203D81268044B9A4204
:103D400002D00120FEF74CBE704700BFE00F00100C
:103D5000A52E5AE208B50448FFF7CCFB034B586088
:103D60000223437008BD00BFB80F0010E00F001021
:103D7000074B01201B88984207D8064A02EB8002B5
:103D800052F8042C12B10130F5E70020704700BF53
:103D900068220100300D001030B5002401250470A8
:103DA0004570817044608460C46004618482C48210
:103DB0000483448380F820401146BDE83040FEF77C
:103DC000E1BD0000024B586002234370704700BF02
:103DD000E00F001070B5044618B9BDE87040FFF759
:103DE000B9BF0B4DA2782868012683789A4207D97B
:103DF000FFF792FB2B685E7002236C60637070BDEE
:103E0000667021460348BDE87040FFF75BBB00BF0A
:103E1000E00F0010B80F001038B50D46014678B11C
:103E20004FF6FF729042074C02D02068FFF77EFBEE
:103E3000236805485D70FFF75DFB022360604370F7
:103E400038BD00BFE00F0010B80F0010024B18681B
:103E500000B1C078704700BFE00F001010B588B9FE
:103E6000174B1B689970174843689B788B4222D97F
:103E7000134C2168FFF726FB236801225A70FFF7D5
:103E800069FF18E0104B1B88984216D80F4B013879
:103E900053F820408CB10A4BA1701B689C42E2D0C1
:103EA0002046FFF7B9FB6378012B04D10548FFF7E3
:103EB00021FBFFF78FFF002010BDFF2010BD00BFCA
:103EC000E00F0010B80F001068220100300D001044
:103ED00070B5184D18B12B68DB78984214D12B6857
:103EE00000245C702E68FEF7B8FCB062FFF71CFF80
:103EF0002B68114AD9782C60013942F82140DC62E4
:103F0000FFF728FF204670BD0C4B1B8898420FD846
:103F1000094C461E54F8265055B12846FFF766FB5B
:103F20002846FFF793FB002044F82600E86270BDA6
:103F3000FF2070BDE00F0010300D0010682201005E
:103F400010B5284B1A880023934205D22649002039
:103F500041F823000133F7E7244CFF23E370244B9F
:103F600020461B8800216362224B234AE362FFF74D
:103F700013FF224A0023042111705360204A11705C
:103F8000D360136193821F4A1460022262701E4A3A
:103F9000137053701D4B1B78D370FFF787FD1C4BBC
:103FA0001A6842F47F021A601B681B0203F07F4309
:103FB000DB43B3FA83F3174ADBB21268C3F1080399
:103FC000C2F302229A42A8BF531C6FF0807000FA1D
:103FD00003F3114A03F07F43116821F07F410B4343
:103FE000136010BD68220100300D0010E80F0010B2
:103FF000702201008C0D0010DF290000B80F0010A6
:10400000A00F0010E00F0010AC0C00107222010095
:1040100020ED00E00CED00E01CED00E008B5FFF73E
:104020004BFE0C4B0028186012DB00F16040FF22B1
:1040300000F5644002701A680121531102F01F025A
:1040400001FA02F29B0003F1604303F561431A6039
:1040500008BD00BFD80F00100321FFF7DDBE70B50B
:1040600000F1080504460E4608222846002108F003
:10407000F1FA204640F8045F3146FFF731F820603E
:10408000204670BD0068FFF745B80068FFF750B8DC
:1040900010B504460068FFF769F8204610BD10B55A
:1040A0004C89D0F89030013C00EBC30244F000444E
:1040B00014674C68D4664FF0FF3440F833405460C6
:1040C00000EB8302C2F88410D0F89420013322441C
:1040D000032B28BF0023C0F894204FF0A042C0F863
:1040E0009030C2F8183110BD90F83930DB0601D598
:1040F00000F0FABD6FF00C00704700F0ADBB38B5B2
:10410000456A0024D5F8943063B14FF4C0610320B0
:10411000002203F088FB014620B12846FFF7BFFFCD
:104120000134EFE7204638BD2DE9F0414FF0A043C0
:10413000D3F8E02F0646446A12F0010031D01A6825
:10414000002522F001021A601A6842F480621A60A7
:104150000122C3F8E82F6619D6F8840020B103F0D5
:1041600035FB0023C6F8843004350C2DF3D14FF015
:10417000A04504F16C03C5F808310223C5F80C41D1
:10418000C5F810310323C4F894300023C4F89030EC
:10419000A069FFF7B4FF2B6843F001032B60BDE873
:1041A000F081D3F81821D3F81431934245D054F854
:1041B000323013F038614FEA82030BD0D4F89420E8
:1041C00023440132C4F89420D3F88410C3F8840047
:1041D000204619E054F832702344D3F88450C7F3D2
:1041E0000A070137B5F80A806F81C3F88410D4F844
:1041F0009430A0690133C4F89430FFF780FF38B9D8
:10420000A5F80A8020462946BDE8F041FFF747BFE0
:104210006B682F819B895BBAB3F5006F03D040F6C2
:104220000602934204D1336928463146984720B1AB
:104230002846BDE8F04103F0C9BABDE8F0811FB5DA
:104240000446684601214FF0FF32FEF76FFE4FF043
:10425000A043D3F81821D3F814319A42F1D0A069C1
:10426000FFF762FFF3E770B5446A4FF0A04304F133
:10427000C4052846D3F82C6107F084FCD4F8AC3090
:104280009E421AD0263354F8230038B103F09EFA28
:10429000D4F8AC300022263344F82320D4F8D800D8
:1042A000FEF746FFD4F8AC300133042BC4F8AC3031
:1042B00084BF0023C4F8AC30E0E72846BDE8704076
:1042C00007F070BCF8B5044604F1B40000214FF0CB
:1042D000A04507F01BFCD5F8E03FDB0636D504F11E
:1042E000C406304607F04EFC2B6843F480732B6005
:1042F0001023C5F8E83F00256719D7F8980020B1CA
:1043000003F064FA0023C7F898300435142DF3D174
:10431000304607F047FC002304EBC30101330022C1
:104320004FF0FF30052B0A624864F5D14FF0A043EF
:1043300004F11C01C3F81C1104F14401C3F820115D
:104340000421C3F82411C4F8AC20BDE7024B9869DE
:10435000FFF789FFB8E700BF000008204FF0A04238
:10436000D2F82C31D2F82801984209D0834287BF75
:1043700003F1FF33C0EB03000430C3EB00007047D0
:10438000052070472DE9F0470C46466A81460846ED
:1043900003F0F5FA4FF00008224662B1536847F681
:1043A000FE7103F16043A3F5F8238B4288BF08F147
:1043B00001081268F1E7B8F1000F01D1074617E0D4
:1043C0000320218903F02FFA074600285CD0D0F89B
:1043D00004A02546504669686A8907F0DAFA6B89B5
:1043E0002D689A44002DF5D123893C467B81012715
:1043F0004846FFF7B3FF874206DDD6F8D8004FF0F6
:10440000FF31FEF787FEF3E706F1C4094FF0A04342
:104410004846D3F8285107F0B5FBB8F1000F02D198
:10442000204603F0B4FA2346002F24DD5889013FCB
:1044300005F1030205F1260100F1FF3008D140F03B
:10444000404E06EBC200C0F808E046F8214008E004
:1044500040F0004E06EBC200C0F808E0002046F82D
:1044600021005968013506EBC2025160052D1B6819
:1044700028BF0025D8E74FF0A0434846C3F828518D
:1044800007F090FB002000E0FF2040B2BDE8F0877D
:1044900010B54FF0A043D3F8E04F14F00B0F06D047
:1044A000084B0121D3F8B0301868FEF721FD14F055
:1044B000B00F02D0044807F044FB4FF0A043C3F80C
:1044C000E84F10BD00000820B40008204FF0A043C2
:1044D0005A6850B142F001025A60D3F8002142F408
:1044E0008062C3F80021152209E022F001025A601F
:1044F000D3F8002122F48062C3F8002112229A60CE
:1045000070474FF0A04318B14FF480729A61704722
:10451000986170472DE9F743754E0446B06133301A
:10452000FDF752FC062384F8323040F2DC53238638
:10453000E22384F839306F4B6662D3F8C4204FF021
:10454000A04542F08042C3F8C4206B4AA3F5502333
:104550009A60DA680A2022F00F0242F00502DA605F
:104560004FF44F432B607823C5F80031FEF7ACFBC6
:1045700002232B6070236B604FF4C0636B6148F2C1
:104580002C032B622B6A204623F400432B6243F258
:104590000F732B6140F61243EB604FF41073C5F8B4
:1045A0000031012100F002F98146002840F09A8094
:1045B00094F8342094F83330804643EA0223AB6405
:1045C00094F8362094F8353043EA02236B6494F86B
:1045D000382094F8373043EA02232B6408F10303B0
:1045E00006EBC30300279F6008F1080308F10108E8
:1045F00006EBC3034FF0FF32B8F1050F3C4D5A6094
:10460000ECD14FF0A04605F11C03C6F81C3105F1B2
:104610004403C6F820310423C6F8243105F16C03A5
:10462000C5F8AC70C6F808310223C6F80C51C6F8BC
:104630001031A8690323C5F89430C5F89070FFF7CE
:104640005EFD2623C6F800324FF6FF73C6F8E83F3A
:10465000BB23C6F8E43FD6F80031284643F00303F5
:10466000C6F800313368414643F001033360234B01
:10467000E362652384F83A306E2384F83B30204BA4
:104680006361204BA36105F1E00340F8DC3FC5F80E
:10469000E070C5F8E470FEF723FDC5F8D80005F119
:1046A000C40007F059FA626A4FF400731649009784
:1046B000164807F0BDFA3946C5F8B00005F1B40058
:1046C00007F00AFA1249626A4FF400730097114822
:1046D00007F0AEFA012110482246FEF77FFBFA21CF
:1046E000FEF796FB4FFA89F003B0BDE8F08300BFF8
:1046F0000000082000C00F40050115507C22010079
:10470000E9400000854300003F4200008422010090
:10471000C54200009322010064010010034B4822AF
:1047200083F81C234FF080521A60704700E100E0CC
:1047300038B540F480704FF0A0439862FA25D962F2
:104740004FF0A0435C6BE4B2E30704D50120FEF711
:10475000BBFA013DF4D1002C0CBF2046FD2040B235
:1047600038BD4FF0A04340F48070012298625A6235
:10477000704770B50E46FFF7F4FFFA254FF0A043DF
:104780005C6B04F0F704E20702D41B6B336004E0B7
:104790000120FEF799FA013DF0D100224FF0A0432D
:1047A000944218BFFD245A6260B270BD73B5264BA7
:1047B0000E4626491A78087802F0FC026FF382024E
:1047C00000F0FC001A706FF38200214B087000208B
:1047D0004FF400411860FFF7ABFF4FF4C87538B1D4
:1047E000FD242EE0019B13F4084F0CD0013DF7D0BF
:1047F0000120FEF769FA002001A9FFF7BAFF04467D
:104800000028EFD0ECE701A90220FFF7B2FF019BDF
:10481000104D1B0401A903202B60FFF7AAFF019A8A
:104820004FF6F07313402A684FF444511343204667
:104830002B600191FFF77CFF1EB117202021FFF7AD
:1048400077FF60B202B070BD401000103C10001045
:104850003410001038100010F8B5664A064610688B
:10486000174601281CD002283AD0634B63491B68C5
:104870008B4208D14FF0A0434FF488719962012117
:10488000596202230AE05E498B4240F0AF804FF04C
:10489000A04140F21F138B6201234B621360A5E01D
:1048A000554B1968564B99424FF0000340F09F80DA
:1048B0004FF0A0410C6B4B6214F0100F0CBF1D4663
:1048C000022514F0080F0CBF04241C4625434D4C50
:1048D000256040F201148C6248620221116086E07A
:1048E0004FF0A0414B6B13F001037FD10A6B4B6279
:1048F00041494248096881420FD112F0040F02F089
:1049000001030CBF0021022112F0020F41EA030350
:104910000CBF00220422134308E03948814205D12C
:104920003849C2F38003086803430B60364C13F028
:1049300001012278354D14BF42F0040261F3820276
:104940002270227813F0020114BF42F0020261F3D8
:104950004102227013F0040F237814BF6FF3000399
:1049600043F00103237020782B7800F0010003F05E
:10497000010383420AD000B10120FFF7C2FD2B786A
:10498000227862F300032B70012300E000232078DB
:104990002A78C0F34000C2F3400282420BD000B13B
:1049A0000120FFF793FD22782B78C2F3400262F3D7
:1049B00041032B70012322782978C2F38002C1F3CE
:1049C000800191420FD00AB1114800E01148012244
:1049D000314606F03BFF22782B78C2F3800262F367
:1049E00082032B70012300223A6000E00023184666
:1049F000F8BD00BF3410001038100010905C00208B
:104A0000F0C0070044100010401000103C100010CF
:104A1000B7760000FF7600002DE9F74F00230A2447
:104A2000384A054600919A469B4601932746A04680
:104A3000A4460A2F5FFA83F9907B02D110B94F4642
:104A400023E010B335B129685668B14202D15FFA4C
:104A500089F052E0012810D1106892F80F9020B12F
:104A6000D14512D3DCB2CA460FE0019989450CD377
:104A70005FFA83FCCDF8049007E0022805D1D07BD3
:104A8000584524BF5FFA83F8834601330A2B02F1AD
:104A90001002CED1009A91072ED40A2F02D1D3074B
:104AA00002D429E0FCB21BE0B8F10A0F02D05FFA91
:104AB00088F408E0BCF10A0F02D05FFA8CF402E03F
:104AC0000A2C19D0E4B20F4B2701D85920B102F0BB
:104AD0007DFE0C4B0022DA510A4E00233744BB7393
:104AE00023011DB1074A29681A4451600549002273
:104AF0000B44DA73E0B200E0FF2040B203B0BDE83F
:104B0000F08F00BF4C10001038B51D684C68256050
:104B10009B88A3801368C4F80630938863810823B8
:104B20002373002363738369984738BD38B50D4CF0
:104B300004F1A005A27B8AB1E37B0133DBB2EF2B4A
:104B4000E37303D8012A09D1012B07D9206818B1D2
:104B500002F03CFE002323600023A3731034AC4218
:104B6000E8D138BD4C1000102DE9F0410022044678
:104B70000F4600F1330500F104082A21032002F05A
:104B800052FE0646A0B34368012252BA9A822A68AE
:104B90000420C3F81620AA885A83174A11689288FD
:104BA00019629A84154A1168928819609A802A6855
:104BB0000121C3F80620AA885A81D8F80020DA61BA
:104BC0003A68D973C3F8262000229A7308215A74D0
:104BD000062219749A74D87419735A73A3692046FB
:104BE000314698470446304602F0F0FD204600E08A
:104BF000FF2040B2BDE8F081A8220100A2220100FE
:104C00002DE9F04780460F4608684146144600F0FB
:104C100038FE00283ED13B6803F0F002E02A39D08C
:104C2000002B37D038460121FFF7F6FEB0F100091E
:104C300032DB2B4E4FEA091573199A7B08330AB9F8
:104C400001229A7173199B7B012B00D034B9404625
:104C50003946FFF789FF03460CB920E0FF2372199C
:104C6000927B022A0DD11F4B083583F800901C4B14
:104C70004046214608F133022B44BDE8F047FFF7D8
:104C800043BF012A0AD1234663B11A7B012A14D1FA
:104C90001B68F9E7F22002E0484600E0184640B2FF
:104CA000BDE8F087204602F072FEBCB1705908B131
:104CB00002F08CFD74510020F1E7032019890022D5
:104CC00002F0B1FD074648B1214602F087FE18B157
:104CD000384602F07BFD01E03C46E7E7FF20DEE7D7
:104CE0004C10001048100010F7B504460E46084658
:104CF0000E21154602F03EFD00284FD128682146BE
:104D000000F0BFFD002841D12B6803F0F002E02A3B
:104D100014D101238DF800305E238DF802306B78BA
:104D20008DF8010003F07F038DF80330AB788DF828
:104D30000430EB788DF805306B4628E0626883EA32
:104D40000201A268114208D09BB24FF6A9629342B9
:104D500003D0E36804F10C0513B3134B134F1B7816
:104D60001B01FA18917B02290AD1296852689142E5
:104D700006D108332046314604F133023B440AE0B1
:104D8000204629463246FFF73BFF0AE0084B204603
:104D9000314604F13302FFF7B7FE02E0FE2000E0E7
:104DA000FC2040B203B0F0BD481000104C100010C1
:104DB000A22201002DE9F04F438985B00E2B074652
:104DC0000D4640F2B3804468A289082A03D0B2F5A8
:104DD000C16F11D0AAE091F83930990640F1A68050
:104DE0006FF00D0102F0C6FC002840F09F803846AD
:104DF000294600F093FB9CE091F83920920640F19F
:104E00009580292B40F29280E389B3F5807F40F0B2
:104E10008D80A37C062B40F08980E37C042B40F03E
:104E20008580238A082B40F08180A14659F81C0F09
:104E30004B680290D4F82600039033B1039AD31A3A
:104E4000D3F1000A5AEB030A01E04FF0000A02987E
:104E5000BAF1000F04F116060CBF4FF0020B4FF031
:104E6000010B05F1330878B3294600F00AFD03462B
:104E700050BB029A02F0F002E02A25D002A859465F
:104E80000193FFF7C9FD0028019B1DDB2B4902019F
:104E900001EB020C02208CF80E003068CCF8080000
:104EA000B0888CF80F30ACF80C0051F802B0BBF1B0
:104EB000000F09D08B502846594642463346FFF72B
:104EC00023FE584602F082FCA38AB3F5807F07D008
:104ED000B3F5007F2AD1284602A901F073FD25E031
:104EE000BAF1000F22D002235BBAA382D9F80030B6
:104EF0002846C4F826306B683946E361336823627C
:104F0000B388A38433682360B388A380D8F80030C3
:104F1000C4F81630B8F80430B380D8F80030C4F8BC
:104F20000630B8F804306381AB699847384602F020
:104F30004DFC002005B0BDE8F08F00BF4C10001004
:104F40002DE9F043064685B089469046012024218C
:104F5000002202F068FC054660B34468002337680D
:104F600084F8009084F8018023716371A371E37168
:104F700042683368083203F11C0153F8040B8B427A
:104F800042F8040BF9D10026A670E6706989204624
:104F900000F078FA6080FB6804AA42F8043D01231F
:104FA0000193009628463146FF2300F04EFC284628
:104FB00002F00CFC05B0BDE8F08300002DE9FF47CE
:104FC000456804460F462E8876BAC6F30326B60017
:104FD000C6F1000A514602F0CDFB98B92389032B94
:104FE00010D962681278082A0CD1364A11689146A5
:104FF00001F0F001E02905D0072B03D9204600F08D
:1050000047FA28B1204604B0BDE8F04702F0DEBB05
:10501000204622211FFA86F802F0ACFBF0B12046B0
:10502000414602F0A7FB02460028EBD1022021896D
:1050300002F0F9FB06460028E4D0214602F0CEFC3F
:105040000028DFD130465146756802F093FB0028F6
:10505000D8D1204602F0BAFB344606E020466FF075
:10506000210102F087FB0028CCD1D9F80020636829
:10507000EA60154A4FF6F6711268FF262A6100228F
:105080001A705A8828468A428CBF093208325A80E0
:105090000023AB72EB7214212E7200F0F3F941463B
:1050A0006881204602F066FB02460028AAD101234F
:1050B00000900193029720460249334600F0B4FB6A
:1050C000A0E700BF04110010001100100A460430D0
:1050D0000321FFF735BF0A4604300B21FFF730BF2D
:1050E0002DE9F041254B05461B68002088B00E468F
:1050F00002460821069302F096FB074600283AD0A4
:105100006B68162E5B684468069306D1AB6805F1A0
:105110000808636001232B7307E0172E03BFAB68F9
:10512000DFF85C8063604FF00008A6F11603012BE6
:105130001ED82670002608216670A670E6702046EC
:1051400000F0A0F960806B6840F29442029307ABD4
:10515000ADF81C20039302220423019204930096CD
:10516000384606A942460123ADF81E6000F0B0FAA9
:10517000384602F02BFB08B0BDE8F081B4220100F4
:10518000F010001038B505460A200C4602F0BCF9B4
:1051900070B1456000230CB1226800E01A46C3815B
:1051A000437303730374034B82601A6818600260D0
:1051B00038BD00BFF410001038B5437B0546022B04
:1051C0000C4605D0012B11D1C3890BB199420DD2E8
:1051D000002C08BF012407F05DFB013C90FBF4F3B9
:1051E00003FB14000123441CEC816B7338BD0000E9
:1051F000034A044B1A60044B02F180721A60704734
:10520000E0000001EC100010F010001038B5074B62
:1052100005461C6844B16368AB4203D120460521B2
:10522000FFF7CAFF2468F5E738BD00BFF41000108F
:1052300010B5064B1B6833B15A688242FAD19C689C
:105240000A689442F6D1184610BD00BFF410001051
:1052500010B50E490446FFF7EBFF20B920460B4975
:10526000FFF790FF60B102224273027C01320274A8
:10527000236C3BB12046054901229847002002E0FB
:10528000FF2000E0184640B210BD00BFEC10001037
:105290002DE9F34143680F4605469046198849BAFF
:1052A000C1F303218900494202F064FA00284BD17E
:1052B0006989072948D96C68204600F0E3F806465A
:1052C000002841D138464146FFF7B2FF0346002887
:1052D0003AD02278112A02D0162A2ED034E01D4A64
:1052E000D8F80000116890468842626815D1A2B9CA
:1052F00063780BB90A236370174B1E6826B3736873
:10530000BB4208D1B168D8F80030994203D030468A
:105310006178FFF751FF3668F0E7AAB1884207D1FC
:1053200002A941F8042D3846FFF782FF034658B121
:1053300018466178FFF740FF06E0427B012A03D15F
:105340000222C68142730673284602F03FFA02B079
:10535000BDE8F081EC100010F410001010B5094BFE
:105360001C6874B1E38953B1013B9BB2E38133B94B
:10537000637B012B03D120461621FFF7B1FE246881
:10538000EFE710BDF41000102DE9F84300260546A4
:105390000F4690469946344685B16868698906F09B
:1053A000BBFA6B89204484B2DB0704EB104403D5BD
:1053B000C6F10106F6B264BA2D68EDE706B164BA2B
:1053C0003968D8F800208BB203EB114193B219442D
:1053D00001EB1242144499FA99F94C44BDF820307B
:1053E0005BBA1C44A3B203EB1444A0B200EB144418
:1053F000E04380B2BDE8F8832DE9F84F0026BDF800
:105400002C700546894692469B46344615B9E6B14E
:1054100064BA1AE0002FFAD0B5F80A8068684745E8
:1054200038BFB846414606F077FA6B892044C8EB8E
:10543000070784B2DB07BFB204EB104403D5C6F103
:105440000106F6B264BA2D68E0E7D9F80010DAF880
:1054500000208BB203EB114193B2194401EB1242CD
:1054600014449BFA9BFB5C44BDF828305BBA1C4497
:10547000A3B203EB1444A0B200EB1444E04380B2A7
:10548000BDE8F88F08B506F047FAC04380B208BD02
:1054900070B500260546344685B16868698906F00E
:1054A0003BFA6B89204484B2DB0704EB104403D53C
:1054B000C6F10106F6B264BA2D68EDE706B164BA2A
:1054C000E04380B270BD38B50546144606F061FA77
:1054D00028462146BDE8384006F01EBA0D4B1B6831
:1054E00053B193F83920D207F9D502685968514071
:1054F0009A681142F3D10AE0074A12683AB192F869
:10550000393013F0010F14BF1046002070471846C1
:10551000704700BF281800102C1800102DE9F84F14
:10552000476804460E46B7F800A09AFA9AF31B0B98
:10553000042B03D0204602F049F9BBE09AFA9AFA0C
:10554000CAF3032A4FEA8A0A7D886DBA4389ADB24D
:105550005345EFD30389AB42ECD338465146FFF7AE
:1055600091FF0028E6D12046294602F0E2F9396988
:10557000524A534B1160F86801F0F001E0291860BD
:10558000904699460AD196F93930002B28DA3046F0
:105590001146FFF74DFE18B335467AE035464FF019
:1055A000010B95F83930DB0705D4BBF1000F0FD0A4
:1055B000444B1D680DE06B68002BF6D0D8F8000056
:1055C000984266D0294600F05CF90028EDD060E0F2
:1055D0002D68B54208BF2D6815B14FF0000BE0E70C
:1055E0007B7A112B54D107EB0A035B88B3F5884F04
:1055F0004ED13546002D9DD0FB8823F0C00333B13A
:10560000204600F0D5FA0446002853D047687B7A3C
:105610002D4A2E4D022B16602F60924615D006D8CB
:10562000012B18D120463146FFF7C8FC27E0062B96
:1056300006D0112B0FD12046314604F0EDFA1EE0C2
:105640002046314603F0E0F819E0204631461B4A77
:10565000FFF71EFE13E0D8F80000314600F011F904
:1056600050B9164B1B6803F0F003E02B04D06760C1
:1056700020460221FFF72AFD204602F0A7F800236A
:10568000CAF800302B60C9F80030C8F8003011E0CB
:105690000025D9F800000028ACD0314600F0F1F820
:1056A00000287FF447AF064B1B6803F0F003E02BA4
:1056B000A0D13FE70020BDE8F88F00BF0411001023
:1056C000001100102818001008110010F810001028
:1056D0002DE9F04F85B0054601919A469DF83CB002
:1056E000109FBDF848401646002A00F0818064B340
:1056F000E31C23F003031FFA83F80FFA88F102F08A
:1057000039F808F114091FFA89F9034608B1FE2097
:1057100083E0686811992246009306F03AF94445FF
:10572000009B06D2686819462044C4EB080206F0C4
:1057300091FF00224FEA580394469A4208DA6968BA
:1057400031F8121001328C44F7E74FF01409A446E7
:1057500028461421CDF800C002F00CF8DDF800C096
:105760000028D4D16C689DF8382084F808A084F80B
:1057700009B0336842F480424AEA0B2A23611FFAD7
:1057800083FB42EA89191B0C99FA99F9A4F8009055
:10579000B5F808E01FFA89F99EFA9EFE0022A27170
:1057A000E271204AA4F802E012881FFA8EFE50BA75
:1057B0001C4901320A800199A08080B209B10A68AF
:1057C00012B97968E16000E0E260E2685B4491B29E
:1057D0000B4403EB1243534463444B44734403446C
:1057E0009AB202EB134303EB1343DB43638104E000
:1057F000436804AE1B6946F8043D3B8E43B12A89D9
:105800009A4205D928463946324600F025FB04E085
:105810007B69384629463246984740B205B0BDE814
:10582000F08F00BFFC10001010B586B09DF820402E
:1058300000949DF8244001940A9C0294002403944F
:105840000494FFF745FF06B010BDF0B5054685B0DE
:1058500010460F4614461E46FFF740FE68B19DF8FD
:105860002830029000939DF82C3028460193394649
:1058700022463346FFF7D8FF00E0FC2040B205B0D7
:10588000F0BD421E0332034614D891F8392002F0CD
:10589000020202F0FF0082B1486883420CD08A689D
:1058A0005840104208D1D24303EA0200831A5842FA
:1058B0005841704701207047002070472DE9FF4193
:1058C00003780025A3F130026F46092A05EB070C87
:1058D0006BD8302B0BD1437803F0DF02582A02D06B
:1058E0000130082604E083781026023000E00A2602
:1058F00004460022A3F13000092803D806FB023237
:10590000303A16E0102E17D123F02008A8F14108F4
:105910005FFA88F8A3F16100B8F1050FC0B20BD8A7
:10592000192803F10A038CBF412061201B1A43EAA6
:10593000021263780134DDE72E2B06D10C2D34D012
:105940007A51601C63780435BCE713F0DF0F02D096
:10595000093B042B29D8C7EB0C0080100130042828
:105960001FD8DFE800F0251E030A1300B2F1807F84
:105970001BD2009B42EA036213E0B2F5803F14D2CF
:10598000009B1806019B40EA034309E0FF2A0CD85C
:10599000009B1806019B40EA0340029B40EA032358
:1059A0001A4321B112BA0A6001E0002000E0012090
:1059B00004B0BDE8F08107B501A9FFF77FFF08B18A
:1059C000019801E04FF0FF3003B05DF804FB2DE9D2
:1059D000F34703680DF1030401930DF107008C46B2
:1059E0000025677800234FF00A09B7FBF9F809FB97
:1059F00018770DF1080A5E1C3037534403F8087C11
:105A000018F0FF07F6B205D1013E04F8017FF6B2A7
:105A10002B460FE03346E6E7771E9342FFB21EDACD
:105A20000DF108094E4416F8086CE04408F80360CC
:105A300001333E46C5EB0C07FF2EC5F100081F449D
:105A4000EAD1934203F1010509DA2E23844207F1DA
:105A5000010C3B70C5D100233B70084600E00020DC
:105A600002B0BDE8F087000001491022FFF7AFBF88
:105A70000C11001010B50446406908B101F0A6FEF3
:105A800021460520BDE8104001F054BD2DE9F0414C
:105A90004668044673680F469A88C2B91B6800F1CD
:105AA0001C014360726800F1080353F8040B8B4239
:105AB00042F8040BF9D130460121FFF70CFB3046C8
:105AC00001F05DFF0546304601F080FE00E0002554
:105AD000666866B173683046D3F8008001F04FFF06
:105AE000284485B2304601F071FE4646F1E7094B85
:105AF00004201A682146A24215BF236822683B6031
:105B00001A6001F017FD044B28461A88521B1A80B0
:105B1000BDE8F0811C11001020110010F8B50646F8
:105B20000F460025174B00241B6821462246F3B17F
:105B3000D6F80CC05869604509D1D6F810C09869EC
:105B4000604504D1B3F80CC0B088844509D0013455
:105B500032B193F81FC0D07F844598BF1A4600E049
:105B60001A461868002818BF19460346DFE71AB11D
:105B70001046FFF78BFF0544BD4201DA012CD1DC52
:105B80002846F8BD1C11001038B5084B00241868D1
:105B900058B1C37F05681BB1013BC377044602E0DF
:105BA0002146FFF773FF2846F2E738BD1C110010AD
:105BB0002DE9F74FD0F804900546B9F800B09BFAEC
:105BC0009BF2C2F30322052A44D1B9F806305ABA2F
:105BD0000192B9F802A09AFA9AFA9BFA9BFB01F09B
:105BE000CEFE9B4E0746328802440A2A05DC994ABB
:105BF000002314680093904610E048463946FFF7AA
:105C00008DFF38B332883A440A2AF0DD22E0D9F811
:105C10000C1062698A4204D000942468002CF6D1EA
:105C20000AE0D9F81010A2698A42F5D1A189B9F821
:105C300004209142F0D111E0042001F065FC0446FB
:105C4000002840F0E08048463946FFF767FFB84239
:105C500080F2D280284601F0B9FDF5E0B9F80620BF
:105C600052BAC2F30C027AB9E28952BAC2F30C02F8
:105C700052B14A4604F1080109F1140052F804CB6C
:105C8000824241F804CBF9D132881744BFB2378041
:105C9000B9F8063099060ED4A37FCBF3032B43F05B
:105CA0000103A377019BC3F30C090AEBC90AAAEB12
:105CB0008B0AA4F81CA06B68B3F802A09AFA9AFAAF
:105CC000198849BAD88840BAC0F30C00C000C1F3A3
:105CD00003218244AAEB810A00221FFA8AFA1A7071
:105CE0005A709A70DA709880A3F806A0D4F80490DD
:105CF0000121B9F1000F00F09E80D9F804C0BCF872
:105D000004B058450CD2C3F80090BAB1B2F806906E
:105D1000814529D8BCF80400504525D315600EE014
:105D200022D0BCF8069081451ED81AB1D2885A45B7
:105D300018BF0021DCF800906246DAE76560A27FB8
:105D4000D20740F1818000297ED060684268928845
:105D5000002A79D11A686AB15168DA888B889A4228
:105D600072D10A680B46F6E7284601F008FE381A99
:105D700030806FE7A38B04F11C011433A3834568C3
:105D800004F108032F682A4653F8040B8B4242F8AB
:105D9000040BF9D1A38B5BBA6B800023AB71EB7161
:105DA000AB72EB7228461421FFF76CFB68816568C3
:105DB0006FB1D7F8049038466FF0130101F0DAFCA8
:105DC0003946284601F0F0FDD9F80070F0E7D8F820
:105DD00000302146A34208BF1E4A236818BF009A1C
:105DE0000420136001F0A6FB2846348801F0C7FDAB
:105DF000201A3080284628E0042001F085FB044664
:105E000000283FF427AF00212022204606F022FC84
:105E10000322E277D8F8002004F108012260C8F8D4
:105E200000404A4609F1140052F804CB824241F87E
:105E300004CBF9D128E7002A80D01560D0889A8851
:105E4000904218BF00217AE7002003B0BDE8F08F30
:105E5000201100101C1100102DE9F04F044640687D
:105E60008DB00B9205908B46C3885BBA9BB2C3F38F
:105E70000C01BBF8302003F400539BB20993079246
:105E80000823143A92FBF3F39BB227890893DB00B3
:105E90009BB2143F0A930491BFB200231425002F34
:105EA00000F0988004980999C0F30C0207980A43FF
:105EB0000692A0F11302BA4206DC0699DDF828A08A
:105EC00041F40051069100E0BA460220142100225C
:105ED000039301F0A8FC039B064600287CD0059A9A
:105EE000416802F1140C52F804EB624541F804EBEE
:105EF000F9D16268D6F804802A4462606289D1468A
:105F0000551B65811D46B9F1000F3CD06589A94537
:105F100038BF4D46ADB2002D33D0052001F0F4FA64
:105F2000844690B1636829468DE8280003206346C3
:105F30000222CDF808C001F0F2FBDDF808C00146EE
:105F400038B90520614601F0F5FA304601F03EFC13
:105F500042E020460391CDF808C001F018FDDDF8BD
:105F600008C0204BCCF81440CCF81030C5EB090920
:105F7000304603991FFA89F901F016FDB9F1000FB7
:105F800001D02468BFE7069A53BAA8F806300AF190
:105F900014035BBAA8F80230002388F80A3088F8A6
:105FA0000B3014214046FFF76DFAA8F80A00DBF821
:105FB000143031460B9A58469847304601F006FC9B
:105FC000049B0898CAEB070703449BB20493BFB233
:105FD0002B4664E7384600E0FF2040B20DB0BDE834
:105FE000F08F00BF755A0000037B8B4203D0002363
:105FF0000173437343837047038B30B544695D1C61
:106000002344058383F8F010038B41695C1C0B4427
:10601000048383F8F02030BD10B5038B42695C1C0B
:106020001344048383F8F01010BD038B426910B54C
:106030005C1C13440A0A048383F8F020038B426932
:106040005C1C1344048383F8F01010BD038B426979
:1060500010B55C1C13440A0E048383F8F020038BF4
:1060600042695C1C1344C1F30742048383F8F020A7
:10607000038B42695C1C1344C1F30722048383F839
:10608000F020038B42695C1C1344048383F8F010F6
:1060900010BD90B1038B4269591C01831344FF2248
:1060A00083F8F020038B432B05D84269591C0183E8
:1060B00013440022F4E79A07F7D17047F8B50C466D
:1060C00017460646002800F09880002900F09780C7
:1060D00000204FF49A71024601F0A5FB20610028D0
:1060E00000F08F80627B484B12B91A6801321A6047
:1060F0001B68082F236042684FF001036261137030
:1061000062695370636996F832209A7062694FF041
:106110000003D3702168626909BA51606269137221
:10612000537262699372D372626913735373937378
:10613000D37307D0042F05D0032F06D1237B043B54
:10614000012B02D863697268DA60626900231374F4
:1061500053749374D3746269137553759375D375BF
:106160006269137653769376D37696F832209DB291
:10617000AA4203F1010306D96269711991F833103B
:1061800015442977F1E70F2D4FF0000305D8626918
:106190002A4401351377ADB2F5E76269D1180133AE
:1061A0000022402B81F82C20F7D163699918013225
:1061B0000023802A81F86C30F7D162696FF07D008E
:1061C000632182F8ED00532082F8EC1082F8EE0093
:1061D00082F8EF10238362691A4482F8F0300133A9
:1061E000442BF8D1204635210122FFF705FF204638
:1061F0003946FFF711FF002004E0F22002E0FA2008
:1062000000E0FF2040B2F8BD6C01001010B504465C
:1062100030B1006908B101F0D9FA0023236163614C
:1062200010BD0000F7B5846A054604212046FFF73B
:10623000DBFE284621460322FFF740FF07460028E1
:1062400031D1204639210222FFF7D6FE2046298E81
:10625000FFF7EBFEEE6A9EB92046FFF71AFF218B8F
:106260002069F03189B201F064FB00956068216912
:10627000194A432303F0A8FE2046FFF7C7FF12E0A8
:10628000304606F028FCC2B2002AE5D020460C2198
:10629000FFF7B2FE013E16F8011F0029DCD02046B0
:1062A000FFF7BAFEF7E7637B0133DBB2092B6373B9
:1062B00006D8C3EB431203EB8203DB009BB201E081
:1062C00042F210734FF4FA7203F2F31393FBF2F3FA
:1062D0003846638303B0F0BDB0220100F7B5846A8D
:1062E000054601212046FFF77FFE2846214603226E
:1062F000FFF7E4FE074600285AD102222046392142
:10630000FFF77AFE2046298EFFF78FFE04222046F3
:106310003221FFF771FE616A204609BAFFF796FE47
:10632000042220463621FFF767FE216A204609BA7B
:10633000FFF78CFE042220463721FFF75DFE204642
:106340000121FFF769FE20460321FFF765FE204685
:106350001C21FFF761FE20460621FFF75DFEEE6A75
:106360009EB92046FFF795FE218B2069F03189B256
:1063700001F0DFFA009560682169194A432303F0B0
:1063800023FE2046FFF742FF12E0304606F0A3FB53
:10639000C2B2002AE5D020460C21FFF72DFE013EB7
:1063A00016F8011F0029DCD02046FFF735FEF7E77D
:1063B000637B38460133DBB2052B98BF4FF47A720A
:1063C00063739ABF02FA03F39BB24EF660234FF455
:1063D000FA7203F2F31393FBF2F3638303B0F0BD9D
:1063E000B022010073B5846A054603212046FFF7F9
:1063F000FBFD284621460322FFF760FE064630BB20
:10640000022220463921FFF7F7FD20464FF4107194
:10641000FFF70BFE042220463221FFF7EDFD616AF3
:10642000204609BAFFF712FE2046FFF732FE218B05
:106430002069F03189B201F07CFA00956068216929
:106440000F4A432303F0C0FD2046FFF7DFFE637BC6
:106450000133DBB2092B637306D8C3EB431203EBA2
:106460008203DB009BB201E042F210734FF4FA7238
:1064700003F2F31393FBF2F33046638302B070BD73
:10648000B022010073B5846A00230546636220468A
:106490000621FFF7A9FD284621460122FFF70EFE3F
:1064A0000646002830D1022220463921FFF7A4FDFC
:1064B0002046298EFFF7B9FD042220463721FFF739
:1064C0009BFD20460121FFF7A7FD20460321FFF792
:1064D000A3FD20461C21FFF79FFD06212046FFF764
:1064E0009BFD2046FFF7D5FD218B2069F03189B255
:1064F00001F01FFA0095606821690F4A432303F0F9
:1065000063FD2046FFF782FE637B30460133DBB23A
:10651000052B98BF4FF47A7263739ABF02FA03F3A4
:106520009BB24EF660234FF4FA7203F2F31393FB1F
:10653000F2F3638302B070BDB022010038B5846A03
:10654000054608212046FFF74FFD284604F12401A7
:106550000022FEF755FB637B0133637301236383E2
:1065600038BD37B50546002850D0846A002C4DD080
:10657000636B581C0CD03C221E33B3FBF2F34FF676
:10658000FF72934228BF13469BB203B90123A38332
:10659000A36B591C0CD03C221E33B3FBF2F34FF615
:1065A000FF72934228BF13469BB203B90123E383D2
:1065B000A37B0BB1A36A0BE094F824301A0601D434
:1065C000FF2305E0BF2B8CBF6FF07F434FF6FF73B7
:1065D0000093E36A01932BB9636A009A134043F076
:1065E00080730193284604F1240100F0B9FF284686
:1065F000694601F025F801A9284601F01DF8284652
:1066000001F028F820460A21FFF7EEFC03B030BD68
:106610002DE9F04F9246BAF80A3089B02B2B044688
:10662000D0F82880526840F23D811378022B40F068
:10663000398190F832100023D8B2884208D2E0188D
:106640000133D51890F83300ED7E8542F4D029E16E
:106650005268D8F8003012BA9A4240F023819A4822
:1066600000210A2205F0F6FFDAF804304FF0000BA3
:10667000C8F80830BAF80890F02357467A89934250
:1066800009D33F689B1AC2EB09099BB21FFA89F92B
:10669000002FF3D106E179680391039AD15CFF29B9
:1066A00000F0B4804B4580F0B1807A89581C90424C
:1066B00003DA039A1A44527803E03A680AB152683E
:1066C000127833292DD00ED801291FD022D30329C7
:1066D0003CD0062935D1082A34BF15460825EDB22D
:1066E0001946082635E0362923D007D834291CD08E
:1066F000352926D11546194601262AE03A291CD00B
:106700003B291ED115461946052622E01546194695
:1067100006261EE0591E002289B24FF0FF361546AC
:1067200017E015461946032613E0154619460026BC
:106730000FE01546194602260BE0154619460426B9
:1067400007E019464FF0FF36002502E019460726FC
:10675000042502310A4492B20292002D46D002333F
:106760005A4A9BB2049302EB8602002307930592D8
:10677000AC460193049A0199BCF1030F02EB81032B
:106780009BB294BF62460422384607A9CDF800C0E8
:1067900001F06DF9DDF800C04B4BBCF1040F0FD9CF
:1067A0000199334401225A54079B059A1BBA42F8B7
:1067B0002130ACF1040C01315FFA8CFC0191D9E776
:1067C0006A1EC2F385021644A5EB820202F0FF02A4
:1067D000042A02D1079A12BA01E09DF81C20079200
:1067E00001229A55079B394A42F826307B89029943
:1067F000994209D3CA1A3F6892B202927A68C3EBEF
:1068000009091FFA89F90392029B46E72E490B7882
:106810000A4693B12D4B00201B680870012B4AD00B
:10682000022B05D14FF0000B4FF06C092C2324E70D
:10683000032B02D14FF0010B3DE0BBF1000FF1D172
:106840005378214D002B2DD0204803790146052B8C
:106850005BD198F80C30012B50D1A36AE878C3F8CB
:1068600028B0C3F82CB008B1C8681863107930B3E9
:1068700008695863507928B3486998639868006933
:106880005862907918B1886900BA986201209873AB
:10689000D07910B1C86900BAD862137AC3B920465A
:1068A000FFF74CFE0023C8F80830504600F08EFF7A
:1068B00009B0BDE8F08F4FF0EC096C23DDE6186BF2
:1068C0004008D6E7186BD8E7221100102C110010F1
:1068D0000B6A08AD1BBA45F8043D0020294600F0BC
:1068E0009FFB254B5B7A002BD9D0244B01205B6AA0
:1068F00029461BBA079300F093FBD0E7033B022B1A
:10690000D0D82046FFF72DFECCE7062B1ED198F8F5
:106910000C30DA1E022A01D9012BC3D12046A56A08
:1069200000F0B9FE2046164900F01AFE2046144930
:1069300000F082FE2046124900F082FE28460C211B
:10694000FFF752FB2046FFF79DFDABE7022BA9D1D5
:1069500098F80C30062BA5D1AA78A8F81AB0A36A2B
:10696000002A9FD08268204612BA1A629A68126979
:106970005A62FFF7B3FC95E7221100102C110010AA
:10698000B422010038B5856A0446CDB12B7B0A2BB1
:1069900010D8DFE803F0150F0F0606060F0F0F0FD4
:1069A000060000F078FE00236B732046BDE83840F7
:1069B000FFF718BD00236B73BDE83840FFF762BDD9
:1069C00038BD000037B50546002835D0846A002C54
:1069D00032D0237B082B2FD10A68636A9A422BD1CD
:1069E00020460C21FFF700FB284621460422FFF732
:1069F00065FBE0B9042220463221FFF7FDFA616A07
:106A0000204609BAFFF722FB2046FFF742FB218B05
:106A10002069F03189B200F08CFF0095606821692F
:106A2000064A432303F0D0FA2046FFF7EFFB637BCF
:106A3000013363731423638303B030BDB0220100BC
:106A4000F7B5846A054605212046FFF7CDFA2846AA
:106A500021460322FFF732FB0746002832D12046A9
:106A600039210222FFF7C8FA2046298EFFF7DDFA06
:106A7000EE6AA6B92046FFF70CFB218B2069F031A6
:106A800089B200F056FF00956068216904F1200288
:106A9000432303F099FA2046FFF7B8FB12E0304693
:106AA00006F019F8C2B2002AE4D020460C21FFF704
:106AB000A3FA013E16F8011F0029DBD02046FFF79C
:106AC000ABFAF7E7637B0133DBB2092B637306D8BC
:106AD000C3EB431203EB82031B019BB201E044F6BC
:106AE00020634FF4FA7203F2F31393FBF2F3384688
:106AF000638303B0F0BD000010B5144B1C6824B3D1
:106B0000A36A03B3DA8B511ED983012AA36A0AD17F
:106B10001B7B03F0FB02012A01D00A2B13D1204674
:106B2000FFF780FB0FE09A8B511E012A99830AD14F
:106B3000A36A1B7B03F0FB02012A01D00A2B02D1BE
:106B40002046FFF77DFF2468D9E710BD2818001004
:106B500073B5846A054600212046FFF745FA0023F5
:106B600023626362A362E362A363636323632846D1
:106B700021460722FFF7A2FA064698B92046FFF7FA
:106B800088FA218B2069F03189B200F0D2FE00959D
:106B90006068216904F12002432303F015FA2046BE
:106BA000FFF734FB637B0133DBB2092B637306D839
:106BB000C3EB431203EB8203DB009BB201E042F222
:106BC00010734FF4FA7203F2F31393FBF2F363833F
:106BD000284600F060FD2846064900F0C1FC284622
:106BE000044900F029FD2846024900F029FD3046FD
:106BF00002B070BDB422010010B5264B1C68002CF9
:106C000046D0A36A002B41D05A8B012A02D9013AFF
:106C10005A833BE03AD100225A83A26A137B0C2BA1
:106C200027D0062B25D0012B06D1537B2046052BE0
:106C30001DD8FFF753FB29E0082B09D1537B2046D1
:106C4000012B02D8FFF77AFC20E0FFF78AFC1DE059
:106C5000052B03D12046FFF7F3FE17E0042B0AD1E2
:106C6000537B2046082B02D8FFF7DCFA0EE0FFF733
:106C70006FFF204608E0032B08D1537B2046012BF1
:106C800002D8FFF7AFFB01E0FFF7FCFB2468B6E793
:106C900010BD00BF2818001010B598B190F8393019
:106CA000846A23F0080380F839305CB1606818B159
:106CB00003F0BEF90023636020460021BDE81040C8
:106CC000FFF792B910BD000038B5044608B9F220AC
:106CD00043E090F83930856A23F008029B0680F87B
:106CE0003920F4D5038EB3F5107F2ED335B93C206F
:106CF00000F07EFB054640B3A06203E0686808B17F
:106D000003F096F900213C22284605F0A3FC03F08D
:106D1000A5F96860C8B1037A114943F020030372F2
:106D20004422686803F04AF80D494322686803F07A
:106D300055F968680B49224603F076F92046FFF7BB
:106D4000A1FB20B12046FFF7A7FFFF2005E094F844
:106D5000393043F0080384F8393040B238BD00BF01
:106D6000B4220100116600000278431C02F0C00149
:106D7000C02904D013441A780AB11846F4E7581C05
:106D8000704700002DE9FF4715461289A2F11A034A
:106D9000B3F5F37F58D84B4C00232846216800F008
:106DA00066FE2B8983424FD123681F887FBABFB20A
:106DB000032F49D84FF48C725743434EF25DF419B8
:106DC000022A41D10322F255DA7802F00F026271F1
:106DD000998849BAB3F8069099FA99F993F902009B
:106DE000002809DBD4F8103153B304F10C00002162
:106DF000D4F81421984723E0002AF3D18AB2012A5B
:106E0000F0D104F10C0803F10C000346414603F1F4
:106E1000010C1B7803F0C002C02A1BD0CA186346BD
:106E2000914208D091F800A093F800C0E245D9D172
:106E300001330131F4E71A780131002AE7D109E082
:106E40000023F355C4F81031284604B0BDE8F047DC
:106E500000F0BCBCFFF788FF1FFA89F90430B9F1D4
:106E6000000FBFD0FFF780FF03465968006801AAF2
:106E700003C219891180019ABDF80C00B2F1012FEB
:106E800018D1B0F5806F15D10299104A09BA914214
:106E9000A16088BFA260D3F80A00D4F8103104F5CD
:106EA0008671C4F80C01002BCED04046D4F81421D2
:106EB0009847C9E740BA0A3009F1FF3918441FFA68
:106EC00089F9CCE7C817001058110010803A090062
:106ED0002DE9F341074600200E4690464FF4887195
:106EE000024600F0A0FC0446002848D04568002176
:106EF00028460C2205F0AEFB98FA98F801230022F0
:106F0000A5F80080AB702A716B71711E0C356A1C7C
:106F1000013113460E78981A2E2EC0B204D1287073
:106F20000A783AB11D46F2E7002EF8D003F8016B5B
:106F30000131EFE71A704FF48072ADF80420ADF81C
:106F400006200198053343F8040C62680E4D991A27
:106F50000E4E05EB8705204689B200F0EAFC294673
:106F60003068352203F03AF82A4630682146352346
:106F700003F022F80546204600F028FC00E0FF253B
:106F800068B202B0BDE8F081B8150010C417001057
:106F900070B54FF48C7545431F4E0246735D7419EE
:106FA000022B0AD0032B2FD0012B34D10020022139
:106FB00071556070A370E07020E0A378013BDBB2F4
:106FC000A37043BBE37860780133DBB2042BE3703A
:106FD00013D138B9114B5B6823B101236370A370DF
:106FE000E07070BDD4F810312BB104F10C00002119
:106FF000D4F81421984700230AE0A37004F10C018F
:10700000BDE87040FFF764BFA368013BA36013B9FC
:107010007355C4F8103170BD58110010B815001028
:10702000012808D8044B1B682BB121B10B6813B1A0
:10703000024A42F820307047C4170010B8150010FB
:1070400037B50F4A0F4B22F003020F481A60FEF7C4
:10705000B2FC0E4D01902C6884B902F0FFFF28604D
:1070600060B10B49224602F0A9FE28680949224670
:1070700002F0DAFF204601A9FFF7D2FF03B030BDCE
:10708000C3150010C8170010B8220100C417001063
:10709000B4220100856D000008B5094B1B686BB177
:1070A0000020FFF775FF0120FFF772FF0220FFF7B6
:1070B0006FFFBDE808400320FFF76ABF08BD00BFAF
:1070C000C41700102DE9F84F9846424B05461B683F
:1070D00089461746002B77D0002975D0002873D039
:1070E0000378002B70D005F0F6FCFF286CD82846FA
:1070F000FEF761FC421C1AD1374E002416F80C3CF6
:10710000032B0ED12846314605F0D3FC48B9334B4A
:107110004FF48C7202FB0434D4F80C01431C06D1EA
:1071200009E00134042C06F58C76E7D103E0C9F8B8
:107130000000002049E02A48284E002190F800A0D5
:107140000B468C46324696F800B05FFA81F9344619
:10715000BBF1000F19D0BBF1030F07D13479C4EB99
:107160000A046445C4BF5FFA84FC4B46013104291C
:1071700006F58C76E7D1032B2AD84FF48C7159434E
:107180005418525C032A23D19946012323700378B3
:10719000C4F810715A1C23710270C4F81481284677
:1071A00005F099FCFF2834BF0646FF26294604F166
:1071B0000C00324604F0EDFB3444002348462373B0
:1071C000FFF7E6FEFB2000E0F22040B2BDE8F88FBA
:1071D000FF20FAE7C41700106411001058110010C6
:1071E0005411001008B504F0EBFC00F00FF800F0AB
:1071F00067F900F0B3F903F067FFFDF7F9FFFFF758
:107200001FFFBDE8084002F031BC00000B4B0C4AE8
:1072100023F00303002113600A4843F6EC725980FF
:1072200019719918016001201A8008719A524A80D8
:10723000054A0648136004F08FBC00BF03C0072056
:10724000E8170010D0170010CC170010D41700104A
:10725000F8B5044600284DD0274B1A681D469042C9
:1072600004D3264B1A681E46904205D304F0BEFC98
:10727000BDE8F84004F0CCBC214804F083FC214870
:107280000023016804F8043C2B6834F8085CA4F17E
:1072900008028A4203EB050138BF02608A4210D01F
:1072A0000F7977B93668B1420BD006688E4204BFB9
:1072B00014490A60595B24F8081C595BD51A194413
:1072C0004D8034F8065C591991420ED00E7966B99A
:1072D0000068904204BF0B4A116034F8082C5A53DE
:1072E00034F8082C1A44CB1A53800548BDE8F840FE
:1072F00004F058BCF8BD00BFE8170010D01700100C
:10730000D4170010CC1700102DE9F04103314FF6CF
:10731000FC750D400B2D044604D943F6EC739D42D9
:1073200001D956E00C25DFF8C480D8F800309C4223
:1073300003D32B4A1268944204D304F057FC04F0A0
:1073400067FC49E0A4F1080634F8087CF61AB6B2E6
:10735000083FBF1BBFB2BD423BD83DD0214804F01F
:1073600011FCD8F8003034F8081C5A18107978B994
:107370005F5A06F108010D441B49ADB208689042FE
:1073800003EB050208BF0A60002111715F5312E090
:1073900005F11402BA4218D8134906F1080215443F
:1073A0000868ADB25A19824238BF0A6000211171D3
:1073B00034F8081C5953568024F8085C5A5B43F68D
:1073C000EC718A421CBF9B185D80064804F0EAFB02
:1073D00002E00020BDE8F0812046BDE8F08100BF5A
:1073E000D0170010D4170010CC170010E8170010A9
:1073F000F8B500285AD003304FF6FC7404400B2C2B
:1074000004D943F6EC739C4201D94EE00C24284881
:1074100004F0B8FB274928480A6806688C46B31A66
:107420009BB2C4F57F512C318B423BDAD5182F79B2
:10743000D15A002F34D1A1F1080EC3EB0E0EA64590
:107440002ED304F114018E4512D308341C44A4B287
:1074500011190F712F8817534B8001232C802B712A
:10746000135B43F6EC718B4204D01A44548001E064
:1074700001232B71B54205D00D4804F093FB05F1B3
:107480000800F8BD0D4BDCF800101A6803681C7981
:1074900024B1934202D01B880B44F8E70360EBE76A
:1074A0000B46BEE7024804F07DFB0020F8BD00BF9C
:1074B000D4170010E8170010CC170010D0170010D8
:1074C00030B50D4A0D4922F0030200230C4C002078
:1074D0001D5B41F8040B84B2AC4209D251F8044C54
:1074E00001301460074C41F8042C1C5B2244F2E785
:1074F00002331E2BEAD130BDEB000820EC17001040
:10750000C8220100E62201000E2838B505460CD835
:1075100004F06CFB064B53F8254014B1226843F885
:10752000252004F075FB204638BD002038BD00BF83
:10753000EC17001038B505460C4659B104F056FB5F
:10754000054B53F82520226043F82540BDE838401C
:1075500004F05EBB38BD00BFEC17001070470000A0
:1075600070B5124D4368002918BF0D462A680446BD
:107570009A4202D12B68636070BD0D4B186840B110
:1075800001686268C668914201D100F0E5FD3046AD
:10759000F5E7084B1B68002BECD01A6822B1616834
:1075A0008A4204BF2A681A60DB68F4E7B42201004B
:1075B000401800103C18001070B5144606461D46D1
:1075C000FFF7CEFF04B12468B46005B12D68F56003
:1075D00070BD0000F8B5069E154F46623E78002546
:1075E00006F1010E80F83C60089E04464560856007
:1075F000C56080F839508562C56105620564066121
:1076000087F800E0FFF7D8FF2046079B984760B94E
:10761000084B20461A6822601C6094F93930AB424E
:1076200005DAFDF715FE2046F8BD2846F8BDF8BD81
:10763000301800102818001001B10968C1607047A7
:1076400001B1096881607047014B1860704700BF45
:107650002C18001010B590F839300446D90719D409
:1076600043F0010380F83930C36903B1984794F8B7
:107670003930DA060ED59B0603D52046211DFDF7CD
:1076800073FA94F93930002B04DA2046BDE8104033
:10769000FDF7BCBD10BD90F8392008B5D10706D55F
:1076A000C36922F0010280F8392003B1984708BD70
:1076B00000B1C161704710B590F839300446D90661
:1076C0001CD443F0100380F83930836A0BB1FFF704
:1076D00059F994F83930DA070CD59B0603D52046C2
:1076E000211DFDF741FA94F93930002B02DA2046CA
:1076F000FDF78CFD236A0BB12046984710BD90F82A
:10770000392008B5D10606D5036A22F0100280F8A8
:10771000392003B1984708BD00B10162704770B5C8
:10772000049C032824D8DFE800F00402070B00259E
:1077300000E01425143500E000250E35ADB200E060
:107740000025EE1CBDF8140026F003060E44864208
:107750004FF000000DDB186004B12C4402201A73B6
:10776000012258735C6019815981DA81184670BD15
:10777000002070BD10B529B338B3002905DA4B429B
:1077800042899BB29A4201D21EE08BB2027B4468CE
:107790000AB1032A05D1641A00F110039C4209D2F0
:1077A00012E0013A012A0FD800290DDA42899A42E3
:1077B0000AD3641A438989B20B4443810389446024
:1077C00019440181002010BD012010BDF8B5044608
:1077D00030B30025EEB224B304F008FAE789013F84
:1077E000BFB2E78104F014FADFB9627B2668920722
:1077F000237B03D52369204698470EE0032B01D154
:107800000E2003E0013B012B04D80D202146FFF799
:1078100091FE02E02046FFF71BFD01353446D9E713
:10782000F8BD3046F8BDF8B50D46174603287ED89A
:10783000DFE800F00402070B002600E014261436EF
:1078400000E000260E36B6B200E00026032F6ED808
:10785000DFE807F0445C5C020E20FFF755FE0446AB
:10786000002864D0032303730023036083190336C5
:1078700026F003061333C6F5BD6623F00303043672
:10788000AE42A8BF2E464360012346810581C381D5
:10789000AE1B0746002E44DD0E20FFF735FE002309
:1078A000054620B92046FFF791FF2846F8BD032280
:1078B00002734373036040F2EC52B3B240F2EB51F7
:1078C000386003818B4288BF134600F1100242608A
:1078D00001224381C281F61A0746DBE706F1130055
:1078E000EB1C23F0030320F00300184480B2FFF7E1
:1078F0007FFD0446D8B106441336002326F0030664
:10790000466005814581036003730AE00D20FFF79F
:10791000FBFD044658B100234360058145810360A7
:1079200007730123E381002363732046F8BD002021
:10793000F8BD38B50389044699420D461ED2CA1ACD
:1079400063899D4206D9ED1A2389ADB21344238180
:107950002468F5E7227B4AB99D4207D06368204638
:107960001B1BE91889B2FFF7CFFC0446206865812C
:10797000258108B1FFF72AFF0023236038BD0346A5
:107980000022D0B201320BB11B68FAE7704710B584
:10799000044640B104F02AF9E3890133E381BDE8EC
:1079A000104004F035B910BD10B568B101B910BD73
:1079B00002680B8922B10489234403811046F7E74A
:1079C000028901601344038110BD10B50C46FFF716
:1079D000EBFF2046BDE81040FFF7D9BF2DE9F0418D
:1079E0000C46054600283CD000293AD002890B8974
:1079F0009A4236D3002637466B89B4F80A80DB1BDF
:107A0000C6EB0808434568686168B4BF1FFA83F88D
:107A10001FFA88F838443144424603F0BAFF47441D
:107A20006B89BFB2BB4246446389B6B204BF2D68BE
:107A30000027B34202D824683CB10026628923891A
:107A40009A4203D123680BB10DE026462DB16A8915
:107A50002B899A4201D12B682BB9002CCCD120461E
:107A600002E0F22000E0FA2040B2BDE8F0812DE90A
:107A7000F84388461646044610B319B30025A946B4
:107A80001EB314B32BB16289934202D39B1A9BB2EB
:107A900014E067896168FF1ABFB2B74228BF374652
:107AA00008EB090019443A463D44B944F61B03F07B
:107AB00070FFADB21FFA89F9B6B200232468DFE780
:107AC000BDE8F8830846BDE8F8832846BDE8F8839A
:107AD00010B50D4B188819464FF6FF7398421ABF20
:107AE000013080B24FF440400023084A9A5812688F
:107AF00022B1948B8442EFD0D268F9E70433102B83
:107B0000F3D1088010BD00BF7401001004230100F0
:107B100030B5048DC16A058F426A034640F2B45005
:107B2000854228BF0546601A1044451B002D01DB25
:107B30005C8530BD501A0028D8BFC2EB01024FF05F
:107B40000000CCBF58855A8530BD10B5038D044662
:107B5000194489B240F6683399428CBF0385018588
:107B6000FFF7D6FF40F2D92398420ADD94F820307F
:107B7000204643F0020384F82030BDE8104001F0B5
:107B8000C5BC10BD10B5044648B1406808B1FFF748
:107B90001DFE21460320BDE81040FFF7CBBC10BD01
:107BA00010B520B10468FFF7EDFF2046F9E710BDDE
:107BB00041617047C0F884107047C0F8801070476A
:107BC000C0F89010704781617047C0F88C1080F841
:107BD0003520704710B5037C0446012B13D90A2BBE
:107BE00011D0C06F18B1FFF7F1FD0023E3674FF626
:107BF000FF73E386606FFFF7D3FFA06FFFF7D0FF3F
:107C000000236367A36710BD2DE9F743894E4FF04A
:107C10000008336801333360874B1C689946002C99
:107C200000F0E880217C94F84A20022901D1062A3C
:107C300051D00C2A4FD094F8A430C3B17F49D4F866
:107C4000A020194411F8011C01328A42C4F8A02076
:107C50003FD3062B4FF0000298BF0133C4F8A02099
:107C600098BF84F8A430204601F046FE31E0E38E50
:107C700018045CBF0133E386A36F53B3B4F9360035
:107C8000B4F94830984224DB02290AD0B4F94410F0
:107C9000B4F9463003EBE10369498A5C9340A4F8E8
:107CA00048300023B4F85220E386B4F85C30204614
:107CB0009A4228BF1A46238F52085B009A42A4F8C2
:107CC0005420B8BFA4F85430238FA4F8523001F0E8
:107CD00090FD002500E00125237C062B06D13168AC
:107CE000226B8A1A282A84BF0135EDB2227A02F06B
:107CF000080202F0FF074AB3042B01D0072B24D15E
:107D0000D4F89410D4F89870D4F89C00326800FB32
:107D10000710236BD31A4FF4FA72B0FBF2F08342D0
:107D200003D90135EDB2012710E094F8A50007FB57
:107D30000011B1FBF2F2934207D9204601F0B6FDE3
:107D400094F8A530013384F8A5300027237C032B59
:107D500007D13268236BD31A282B09D90135EDB22C
:107D600006E0092B04D13268236BD31AF02B00D81C
:107D700025B32046FFF72EFFE368B8F1000F02D0CD
:107D8000C8F80C3001E0C9F80030D4F890301BB1CD
:107D900060696FF0090198474FB1A38B22460093A9
:107DA000E38B0193A06D616A231D01F0DBFC21468A
:107DB0000120E768FFF7BEFB444618E094F8343032
:107DC00094F835200133DBB29A42E76884F8343006
:107DD0000DD8D4F88C3084F834501BB9204601F00B
:107DE00095FB04E06069214698470028F6D0A0463C
:107DF0003C4614E7134B1D689846C5B132682B6B9F
:107E0000D31AF02B11D92846FFF7E4FEEA680CB12B
:107E1000E26001E0C8F8002029460120EF68FFF782
:107E200089FB25462C463D46E7E7EF68FAE703B0B5
:107E3000BDE8F08334180010401800102123010021
:107E4000142301004418001010B503680C468B423F
:107E500002D1CB6803600CE0124A136043B1D968C9
:107E6000A14203D11360E268DA6002E00B46F5E755
:107E700013600023E3602046FFF7ACFE237C0A2B4F
:107E80000CD0012B0AD094F82030DA0706D543F045
:107E9000020384F82030204601F038FB00232374CD
:107EA00010BD00BF4818001013B50446037C00291C
:107EB00031D0012B2FD0C26F22B9018D40F668322C
:107EC000914228D0A38B22460093E38BA06D0193AF
:107ED000616A231D01F046FC2046FFF77BFE2F4A16
:107EE0001368A34201D1E3680BE02D4A136043B14C
:107EF000D968A14203D11360E268DA6002E00B4660
:107F0000F5E713600A232374264B1A681C60E260AD
:107F100001F076FD3DE0072B3BD8DFE803F0041CC1
:107F2000222B2B3A3A31A38BFBB11F4A1368A34291
:107F300001D1E3680BE01A4A136043B1D968A1424A
:107F400003D11360E268DA6002E00B46F5E71360E4
:107F50000023E36009E015482146FFF775FF022082
:107F600004E00E482146FFF76FFF01202146FFF78E
:107F7000E1FA0EE0204601F088FA58B9052304E042
:107F8000204601F082FA28B909232374204601F023
:107F9000BDFA002040B202B010BD00BF4018001072
:107FA00048180010441800104C1800103C1800101D
:107FB000037C012B05D090F8203043F0100380F8AB
:107FC00020300121FFF770BF10B50846144632B1CA
:107FD0001189FFF7BAFD2046FFF7F8FB04E01BB953
:107FE000BDE81040FFF7E4BF002010BD70B5164B90
:107FF0001C6844B3E26FE66892B1D4F8845025B1AE
:10800000606921460023A84704E0284621462B4604
:10801000FFF7DAFF08B9E06702E040B20A3010D09B
:1080200094F82030DA070CD543F0020384F82030AE
:10803000204601F06BFA94F8203023F0030384F813
:1080400020303446D5E770BD4018001008B5FFF762
:10805000CDFF064A13780133DBB21370DB0703D57B
:10806000BDE80840FFF7D0BD08BD00BF38180010BC
:1080700038B5037C0446012B15461ED059B1C06F9C
:1080800018B1FFF7A3FB0023E36794F8203043F017
:10809000100384F8203095B1227C033AD2B2042A2E
:1080A0000DD8012303FA02F212F0130209D0204680
:1080B0000021BDE83840FFF7F7BEF32002E00020C2
:1080C00000E0104640B238BD2DE9F04F037C85B08A
:1080D0000A2B04468A4608D121461D48FFF7B4FE04
:1080E00001202146FFF726FA2FE00368876D0393EE
:1080F0004368466AB0F81C90B0F81E80D0F89050E3
:10810000D0F814B0214613480293FFF79DFEA06FEC
:1081100008B1FFF745FD606F08B1FFF741FD012091
:108120002146FFF707FA1DB158466FF00901A8472D
:10813000BAF1000F09D0CDF80090CDF80480384690
:10814000314603AA02AB01F00DFB05B0BDE8F08F8C
:1081500044180010401800100121FFF7B5BF0000BF
:10816000034B044A10681A6810441860704700BF37
:108170007001001034180010F8B505460120FFF713
:10818000C3F93A4E0446002834D1394B31681B6894
:1081900043B11A6B8A1AA24234BF224618461446CB
:1081A000DB68F5E708B1FFF7D7FF0120FFF7ACF96F
:1081B0000446F8B92F4BD6F800E01B687F20224612
:1081C00073B1597CA94209D8814207D81F6BC7EB0C
:1081D0000E07A74202D308463C461A46DB68EFE783
:1081E00012B11046FFF7B8FF0120FFF78DF90446E2
:1081F000002839D00021A822204604F02BFA40F6AE
:108200006833A4F86E3023856385FF23A3724FF48F
:10821000067323870623A4F84830A4F846304FF6A7
:10822000FF736574E38600250123A4F85230A4F897
:1082300070506572A4F84450FFF792FF336860668F
:1082400023630D4BA065C4F884300C4BE064C4F884
:1082500094300B4BA066C4F89830092384F834504E
:10826000C4F89C3084F8A5502046F8BD341800109E
:108270004418001040180010C97F000000DD6D0098
:10828000F82401004020FFF777BF10B504460846E8
:10829000FDF724F930B1038E23B1283B9BB29C42F9
:1082A00028BF1C46204610BDF8B51F46037C044677
:1082B0000D46002B58D1002958D00B68C28343606B
:1082C000036833B90430FDF709F9002850D043683A
:1082D0002360A68B16B9FFF7FBFBA083FFF740FFD7
:1082E000A0650138002340F66832E064A0664FF4D0
:1082F00006706362E362294622856285A4F85C20E9
:108300002087FFF7C2FF0123208700EB8000984001
:10831000A4F85230A4F85400C4F888702046022112
:1083200001F068F828BB0223237496B1124A13683F
:10833000A34201D1E3680BE0104A136043B1D9684E
:10834000A14203D11360E268DA6002E00B46F5E770
:1083500013600B4B1A681C60E26001F051FB204671
:1083600001F0D4F8002004E0F72002E0FA2000E059
:10837000FC2040B2F8BD00BF4C1800104818001097
:10838000401800102DE9F041AE4B04461B78AE4D6D
:1083900013F0100F00F02581016E2B68B0F85C70AF
:1083A000426EC81A0028A94E0DDB994203D13168EC
:1083B000511A002907DB31688A4213D1A4490968A0
:1083C000C989B9420ED9A2490968C98923663368A7
:1083D000A4F85C10636629B194F8A43013B10023AB
:1083E00084F8A4303368E06C191A002930DC0021CD
:1083F000A4F86C1097490988002940F0B681B4F8B8
:108400005CC0616E3A446144914240F0AE81B4F97F
:108410003620002AC0F2A981984240F0A68194F843
:1084200050300133DBB2032B84F850300AD9B4F852
:108430005220238F13449BB2934240F2A580A4F8AC
:108440005230A1E040F0A080204601F004FA9BE009
:10845000A26D9A1A002A65DC94F82020500707D5EF
:1084600022F0040284F82020B4F85420A4F852200A
:10847000B4F94470B4F84600E36400EBE700A4F8F4
:108480004800237CB4F86E0089B20022A4F86C1076
:10849000032B014484F84A20A4F86E1084F850207D
:1084A0003CD9B4F85230B4F854209A42228F9CBF81
:1084B000524392FBF3F21A4492B29A422ED9A4F894
:1084C00052202BE03A695168938909BA5BBA326845
:1084D00013F00303C2EB0102398918BF01230B44D7
:1084E0001344002B00F345813B68A367B4F86C305C
:1084F00043B13A69928952BAD10744BF03F1FF33BD
:10850000A4F86C307868B4F87080FFF738FAC0EBE4
:108510000800A4F870003846FFF734FBA76F002F5F
:10852000D0D128E10023A4F86C302DE039693268FD
:1085300048688B8900BA5BBA111A13F003033889B3
:1085400018BF01230344CB1A002B20DBA36DD21AE2
:10855000002A1CDC3B686367B4F86C3043B13A69AD
:10856000928952BAD20744BF03F1FF33A4F86C30AA
:108570007868B4F87080FFF702FAC0EB0800A4F83E
:1085800070003846FFF7FEFA676F002FCED1E36B1D
:108590003BB3226C3168521A002A22DA2E4AB4F810
:1085A0004410126841F3CC00D21A121A92B293B25C
:1085B000180448BF53421144B4F8462048BF9BB248
:1085C00042F38D00121A89B213449BB2A4F84410EE
:1085D00041F3CC01A4F846300B44A4F84830002302
:1085E000E3631C4F636A38882A68002800F0AC8077
:1085F000991A012934D45E1CB61A301A00282FDCCF
:10860000164E0B46706842898A420DDA0189C91AF2
:1086100089B242899A4205DA9B1A0022018142817D
:108620000068F6E7594200E0494209B2FFF7A2F8B4
:108630002A683189636A0A44D21A328132692B600E
:10864000536016E060180010501800105C180010FD
:108650006418001058180010341800106C1800101E
:10866000D31A002B05DA94F8203043F0020384F883
:1086700020302B68626A991A002960DB208D591C12
:10868000891A091A00295ADC9A4258D13E4B1A69B4
:10869000938959BA3C4E11F00301B6F808E018BFAF
:1086A0000121714489B28142398022D959BAC9075E
:1086B00007D559BA01F03E0149BA23F47C530B4364
:1086C0009381238D3381928952BA900744BF03F17D
:1086D000FF33338170683189FFF72BF933699B8948
:1086E0005BBA294A13F00303128918BF012313440C
:1086F0003B803B882A6820461A446262228DD31A46
:108700002385FFF705FA73681A8922B11F4A13609F
:108710001D4B00225A6033699B895BBAD90704D587
:108720001B4B1A7842F020021A7094F82030DA07B6
:1087300002D523F0010312E043F0010311E02046CB
:10874000BDE8F04100F0B5BED11A002905DB0132C9
:10875000218DD31A5B1A002B14DD94F8203043F0DE
:10876000020384F82030BDE8F081002384F8503003
:108770000AE7002301E04FF6FF73E386002384F845
:10878000343001E7BDE8F0816C1800106818001063
:1087900061180010F0B51B4B1C68A3895ABAB2F5DA
:1087A000C04F2ED3143459BA090B0539890089B248
:1087B00000238B4225D2E25C012A05D021D3022A74
:1087C00004EB030202D017E0013318E05578042DC2
:1087D00017D1DD1C8D4214DA9578D27840F2B35669
:1087E00042EA0522571EBFB240F2B455B74288BFD5
:1087F0002A460280043302E0527812B113449BB23D
:10880000D7E7F0BD641800102DE9F04F8C4A43689B
:108810008BB0136005460F461A8851BAC1F3032185
:1088200003EB810387490B6051BAC1F3032189002F
:108830004942FEF79FFF834E10B92B89132B05D8B1
:1088400028460BB0BDE8F04FFEF7C0BF7E4C39465E
:108850002068FDF716F80028F2D1236803F0F00332
:10886000E02BEDD02B892846009378492246062339
:10887000FCF78AFD0028E3D133689B895BBAC3F318
:108880000733C3EB83339900284609B2FEF772FF22
:108890000028D5D1326813885BBA9BB20593138048
:1088A000518849BA56686A4B36BA1E609068694B5F
:1088B00000BA89B203901860518056609060D389E5
:1088C0005BBA9089D381079043BA634CDBB203F063
:1088D0003F0727702F8913F0030418BF0124DFF826
:1088E00080A13C441FFA84F8DFF85CB1DAF800405C
:1088F000DFF858910894DBF80040584FD9F8000091
:108900000694DFF84CB1089CA7F8008009904FF05E
:10891000000C002C00F05382B4F81E90059FB9455E
:1089200016D1B4F81C90894512D16068099FB842ED
:108930000ED12068069FB8420AD1BCF1000F0AD0C0
:10894000E3680898CCF80C30454BE0601C6002E00E
:10895000A446E468DDE7434928890A610881424E5C
:108960004248E26F00230B604D6003603370804625
:10897000CAB1D4F884C0BCF1000F03D060692146AD
:10898000E04704E0604621466346FFF71DFB08B957
:10899000E06708E040B20A303FF452AF2F4B1B882B
:1089A000002B7FF44DAF2C4D314A95F800901460A8
:1089B00019F0040F924615D0237C022B06D1254BCB
:1089C0001A68A36D9A4240F0C181B5E1204B1A6844
:1089D000636AD31A00F1BA81218D5B1A002B00F370
:1089E000B581A9E109F0020000F0FF0194F8202010
:1089F00040B1207C0238012804D942F0020284F8F8
:108A00002020A3E1D00602D41A4A12682263002271
:108A100084F8A52004F138000491FFF7BBFE227C06
:108A20000499023A072A00F29181DFE812F025004A
:108A30008C00D900E8001C01D9003701620100BF99
:108A400054180010641800100411001000110010D8
:108A5000501800105C180010601800105818001012
:108A6000401800106C1800106118001068180010F1
:108A7000801800103418001009F01202122A51D187
:108A8000A16FA44A09691268496809BA01318A428A
:108A900048D1B4F86E30E2640133A4F86E309E4AD7
:108AA000DBF800301268591C6162E162D289013B37
:108AB000236604232374E118A4F85C20208FFFF7B9
:108AC000E4FB00EB80035B00A4F85430B4F85230B0
:108AD0002087012B08BF4000B4F8703008BF80B277
:108AE000A4F85200013BA06FA4F870300368A3679C
:108AF0001BB94FF6FF73E38603E00023E38684F897
:108B00004A30FFF73FF8D4F8883023B994F8203082
:108B100043F0020318E160692146002298470A30B9
:108B2000F4D13DE119F0100F00F010817A4B7B4F2A
:108B30001B6839885888DBF8002000901B88019357
:108B4000744B186838E019F0100F3BD0714B18685F
:108B5000E36CDB43C34225D4A36DC31A002B21DC95
:108B600004232374A369002B00F007816069214668
:108B70000022984718B10A3000F01281FDE020462B
:108B8000B4F85270FFF7FEFBB4F86C3013B1013B40
:108B9000A4F86C30238F012F04BF5B009BB2A4F8B4
:108BA000523020E05C4B5D4A1B6811885F88DBF81F
:108BB000002000971B8801931144594B594A00F03B
:108BC000D1FDC3E0002900F0C180574A636A1268F2
:108BD000013B9A4240F0BA80204600F01EFEB5E00C
:108BE0002046FFF7CFFB33789A0640F1AF8094F828
:108BF000203043F0020384F82030072331E0204680
:108C0000FFF7C0FB337813F0200F2B7821D013F03F
:108C1000100F94F8203043F0020316D03D4A11683B
:108C2000A26D914211D184F820302046FEF7D2FF88
:108C30003E4A1368A34243D03D4A1360002B4ED0F6
:108C4000D968A14241D00B46F8E784F820300823C8
:108C500007E0DB067AD52F4B1A68A36D9A4275D1CF
:108C60000623237472E02046FFF78CFB33789F06BF
:108C70006CD594F82030204643F0020384F820306D
:108C8000FEF7A8FF294A1368A34219D0284A1360A7
:108C90002BB3D968A14218D00B46F9E72046FFF75D
:108CA00071FB2B78D80651D51A4B1A68A36D9A42DE
:108CB0004CD12046FEF78EFF1C4A1368A34201D117
:108CC000E3680CE01A4A136007E01360E268DA60B8
:108CD00006E0D968A142F8D00B46002BF9D1136009
:108CE0000A232374134B1A681C60E26000F088FEAC
:108CF0002CE02046FFF746FB2B78D90626D5054BFE
:108D00001A68A36D9A4221D1337843F0100333706F
:108D10001CE000BF5C180010641800105818001008
:108D2000001100100411001050180010401800101D
:108D30004818001044180010337843F008033370CB
:108D400094F8203023F0010384F8203033781A0798
:108D500017D4DA061CD4B4F86C20002A40F0F48052
:108D6000D8F80020002A00F0178194F82030DB06A4
:108D700040F1F6801046FEF729FD2046FFF7ECF99A
:108D80000EE0D4F890301BB160696FF00A0198478B
:108D900091482146FFF758F801202146FEF7CAFB0B
:108DA0008E4B00245868CAF80040C8F800400028DC
:108DB00000F00F81FEF70AFD884B5C6009E1884CEA
:108DC000D4F800C0BCF1000F3BD0BCF81E40059F9A
:108DD000BC4233D1BCF81C408C422FD1DCF804409B
:108DE000099884422AD1DCF80040069FBC4225D174
:108DF00058073FF525AD9A070ED5DCF82430F21A56
:108E0000002A0FDBBCF828201344F31A002B09DCDE
:108E100005980091019035E0DF0703D5714B1B6881
:108E2000CCF83030B8F1000F3FF40AAD9CF8203098
:108E3000604643F002038CF8203018E0DCF80CC0E8
:108E4000C0E7694CD4F8009064464F4697B1B7F834
:108E50001CC08C4507D1D7F800C00698844519D0AE
:108E6000BCF1000F16D03C46FF68EFE7304600F03B
:108E70004DFBE5E4079F7BBA58073FF5E1AC059C45
:108E800000910194039808EB0601584A584B00F0F2
:108E900069FCD5E42CB1F968E1605349C7F80C903E
:108EA0000F6003F0100101F0FF0431B1538800930B
:108EB0001388039A0193501CE5E79E077FF5C0AC29
:108EC000787CFFF759F9064600283FF4B9AC4748CB
:108ED000474A03683360BB8BB38313687360454BA9
:108EE0001A681388F38303233374DBF80030591CAA
:108EF0007162F162D289013BA6F85C20A6F8542089
:108F000033667B697361BB69B3613B7A23F073039A
:108F10003372DAF80030CAF80060F36000F070FDD8
:108F200006F13800FFF736FC311D308FFFF7ADF941
:108F300012213087304600F05DFA002896D0304686
:108F40002146FFF7C1F87BE4D4F88030002B3FF4D2
:108F500007AF6069214698470A307FF401AF1FE7E9
:108F60002B781F0703D5537B43F001035373D4F8C9
:108F7000845025B1606921460023A84704E02846B3
:108F800021462B46FFF720F843B20A333FF408AFDF
:108F900010B1D8F80030E36733789D0606D400237B
:108FA0002046CAF8003000F0B1FAF9E6238D40F609
:108FB00068329342D4F884501CBF01332385002DBE
:108FC000EDD00022606921461346A8470A30E6D159
:108FD000E6E60BB0BDE8F08F401800106C180010EA
:108FE00044180010341800103C1800100411001030
:108FF000001100106418001010B51488C90720442F
:1090000000EB104080B205D51978C1F1010119704B
:1090100040BA80B2108010BD2DE9F84F9DF828703D
:109020009B4617F0010F0CBF0023042317F0020F1B
:109030000CBF4FF000084FF00C08814603200D468E
:1090400092469844FEF760FA0026044618B928466E
:10905000FEF7BCFB33E04773066045602B891421A3
:10906000C8EB03030381468106732846FEF782FBA3
:1090700028B12046FEF786FD3046BDE8F88F6368CC
:109080005B682361B9F81C2052BA1A802369B9F8C9
:109090001E2052BA5A8023699BFA8BFB4FEA88281C
:1090A000C3F804B008F5A048236948EA0A0A9AFA06
:1090B0009AFAA3F80CA0236900229A74DA74204665
:1090C000BDE8F88F143138B589B204461546012041
:1090D0000022FEF7A8FBD0B14368A28B52BA1A80D7
:1090E000E28B52BA5A805D60626A12BA9A6045F2A7
:1090F000100252BA9A81628D52BADA8100221A7431
:109100005A749A74DA74628D636A1344E36238BDE8
:109110002DE9F04F8DB00893002304469146ADF839
:109120002C308DF82A300791D1B1037C072B03D066
:10913000023B022B00F28A80B9F1000F00F0898017
:10914000B4F86E304B4506D294F8203063F07F03BC
:1091500084F8203073E0B4F87030032B79D9F3E74A
:109160004FF0F20B6DE06A7B238F12F0010F0CBF02
:109170000020042012F0020F0CBF00210C212A89CC
:10918000B9F1000F00F085809B1A1B1A5B1A9BB285
:10919000002B00F08180002A7ED0089A4B45B4BF96
:1091A0009846C846D7074FF0030041465BD5324684
:1091B000FEF739FB0746002800F017810799424661
:1091C0004068FCF780F941460BAA0DF12A03FFF72E
:1091D00013FF3846FEF7D3FB059A2E46104480B2A3
:1091E0000590B3460026C2460996CA4580F0BB806A
:1091F000238FCAEB090292B29A4228BF1A46089BF3
:10920000002013F0010B0692ADF82E008DF82B0014
:1092100049D1584606990122FEF705FB034600286E
:1092200056D194F8203063F07F0384F8203017B1D2
:109230003846FEF7CBFA16B13046FEF7B1FC4FF0D8
:10924000FF0B4FFA8BF00DB0BDE8F08F4FF0F30B32
:10925000F7E7B4F87030656F059305B32E68002EFC
:1092600081D03546FAE70122FEF7DDFA07460028ED
:1092700000F0BB8041460798FCF704F9C0430DF1AC
:109280002A0380B241460BAAFFF7B6FE079B7B601C
:109290009FE7C8464F46A4E7B0463746A1E72E46AB
:1092A000A8462F469DE711460246FEF7BCFA8346C4
:1092B0000028B6D00799069A51444068FCF703F994
:1092C00006990DF12E020DF12B03FFF795FE1BE021
:1092D000079A06995244104604920393FCF7D2F879
:1092E000039B049AC0435A60ADF82E005946584675
:1092F0005A460393FEF797FA039B834608B918462C
:109300000CE01946FEF750FB5846FEF738FB059A6D
:10931000104480B20428059003D95846FEF756FA47
:109320007FE7A36E00225946009220465344FFF780
:1093300073FE834600283FF474AFBDF82E3043819E
:109340009DF82B300373437B43F00403437316B142
:10935000099B186000E00646069ACDF824B09244B6
:109360001FFA8AFA41E707B368683946FEF71CFB23
:109370003A892B8913442B81B8F1000F18D09DF83E
:109380002A3023B1BDF82C305BBAADF82C3005F192
:109390000C03BDF82C00414605F10A02FFF72CFE34
:1093A0006B7B43F004036B7302E00DB9666700E06A
:1093B0002E60A36E4B44A366B4F86E30C9EB03096C
:1093C000059BA4F86E90A4F87030BBF1000F3FF439
:1093D00038AFDBF8103053B1089A920707D408224F
:1093E00052BA99890A439A8101E0002719E74FF0A0
:1093F000000B26E773B5B0F870300446032B0D461A
:1094000013D8B0F86E30C1F34006B100002B38D04D
:1094100000200246FEF707FA014630B100962046CA
:109420002A46A36EFFF7F8FD30B994F8203063F0B8
:109430007F0384F8203024E0636F0BB9606704E099
:109440001A680AB11346FBE71860AA0707D0A36E93
:109450000133A366B4F86E30013BA4F86E30EB071D
:1094600005D594F8203043F0200384F8203040687C
:10947000B4F87050FEF783FA2844A4F87000002076
:1094800000E0FF2040B202B070BD436F43B11A68E4
:109490000AB11346FBE71B699A8951BA490702D002
:1094A0000121FFF7A7BF012149BA0A439A81002091
:1094B0007047F7B5826D002112BA0446FFF702FE2D
:1094C0000546F0B194F82030476823F0030384F890
:1094D00020300389261D0093214632460623FBF7E0
:1094E00053FF3882627AA37A0092062201922146C3
:1094F00032462846FCF7A9F92846FEF767F900200E
:1095000000E0FE2040B203B0F0BD00002DE9F341C1
:10951000914B04461B68834200F01A81B0F8523028
:10952000B0F85C80456F984528BF984690F8203089
:1095300099070FD545B12B6929895A68C36C12BAAE
:10954000CB1A1344434505D9204602B0BDE8F0418B
:10955000FFF7AFBFA66F002E00F0A8803368002B86
:1095600000F0A4801E46F9E72B692A895968E36C4C
:1095700009BAD21A0A44424500F2D880A36F002BE0
:1095800040F098802B686367237C022B0BD02B69FB
:10959000102252BA99890A439A8194F8203023F014
:1095A000030384F82030626A2B6912BA9A602B692F
:1095B000628D52BADA81628D636A27461344E36290
:1095C0006A7B2B69D20744BF644A5A61B4F93630CA
:1095D000013304BF0023E38657F8043B002B7BD004
:1095E000E36B33B95E4B1B68E3632B695B681BBAA3
:1095F00023646B6829695A688A1A598992B2891A50
:1096000059816B6819898A1A1A816B682A695A60AC
:109610002B6900221A745A742B693A4668689B8930
:109620005BBA1B0B01899B009BB200910193214601
:109630000623FBF7E1FE2B7B23B16B895BBA6B81C1
:1096400000232B736B892146DB439BB218442B69A3
:1096500000EB10401882627AA37A009206220192EF
:1096600068683A46FCF7F1F82A695168928909BAA4
:1096700052BA288912F0030318BF0123A26D0344D4
:109680000B44D21A002AB8BFA3652A6993895BBA32
:1096900013F00303298918BF0123D9423DD00023C9
:1096A0002B60A36F03BBA5672E46656F002D7FF46B
:1096B0005BAF47E094F8201011F0440F7FF462AFE5
:1096C000636F002B2ED0186800287FF45BAF1889D9
:1096D000238F984226D355E73846FBF7FFFE002834
:1096E000C2D0436823607BE7336951685B6809BA7D
:1096F0001BBACB1A002B0EDA04F1780213683BB1C7
:109700001869406800BA401A002801DA1A46F5E7DD
:109710002B60156004E03560C6E72846FEF732FA94
:109720003546C1E711F0A00F7FF42CAF94F8A430B8
:1097300043B9B4F85C108A4204D9C4F8A0300123BC
:1097400084F8A43094F8203003F07F0384F82030AC
:10975000002002B0BDE8F08180180010020405B4BA
:10976000341800102DE9F74F81460E46904601202F
:10977000142100221F46BDF830B0BDF834A0FEF71A
:1097800052F8054690B344689BFA9BFBA4F800B0DE
:109790009AFA9AFA99FA89F936BAA4F802A0C4F8A2
:1097A0000490A66045F214035BBAA3810B23002644
:1097B000A3736823E37326746674A674E67403893E
:1097C000414600933A460623FBF7DEFD062320823E
:1097D00041460193009628463A46FF23FCF735F8A8
:1097E000284603B0BDE8F04FFDF7F0BF03B0BDE879
:1097F000F08F826F82B113680BB11A46FBE7416F9D
:109800001160826FC363426790F84A208367013218
:1098100080F84A20FFF77ABE7047836F30B5CBB12E
:109820001A6800F1740182670A6852B114696568A8
:109830001C692DBA646824BA2C1B002C01DA11466D
:10984000F2E71A600B6090F84A30013380F84A3032
:109850000023C36330BD836F10B504462BB390F86B
:1098600020305B0721D4FFF7D8FFB4F85230B4F8AA
:109870005C2093428BBF52085B08A4F85420A4F8E4
:109880005430228FB4F8541053009942B8BFA4F852
:109890005430B4F8541013440B44A4F8523094F8E4
:1098A000203043F0040384F8203010BDF7B5826DFA
:1098B0000021013A12BA0446FFF704FC0546C8B17C
:1098C0000389261D47682146009332460623FBF78D
:1098D0005BFD0021388206228DE80600A37A284627
:1098E00021463246FBF7B1FF284603B0BDE8F04001
:1098F000FDF76CBF03B0F0BD2DE9F341866F044660
:1099000016B9466F002E4CD03369B3F80C8098FA24
:1099100098F818F0010806D0B6F80880D8F10108C8
:1099200038BF4FF000085FFA88F8204688F0010140
:109930005A68FFF7C7FB0546002832D04768B8F1E0
:10994000000F07D0112252BABB8923F47C53134372
:10995000BB810CE0706843689E8976BA4FF6FC7351
:10996000B60A07F1140101223340FEF780F82B8973
:10997000261D00932146324628460623FBF704FDA8
:109980000021388206228DE80600A37A2846214667
:109990003246FBF75AFF284602B0BDE8F041FDF71A
:1099A00015BF02B0BDE8F08170B504460B200D462E
:1099B0001646FDF7A9FD0346F8B11049002280E8DC
:1099C00074000A682AB15068A04208D9041B546088
:1099D0001A600B6070BD4C68844208D80A46516812
:1099E0005868401A586011680029F4D101E0201A23
:1099F000486011681960136070BD70BD8818001050
:109A0000084B1A6862B9084A126812B9074A126804
:109A100032B101221A60FA2005490022FFF7C4BFC3
:109A2000704700BF84180010401800104418001040
:109A3000359A000008B5FEF709FB084B1B6813B9FF
:109A4000074B1B6833B1FA2006490022BDE80840E5
:109A5000FFF7AABF044A136008BD00BF40180010FA
:109A600044180010359A00008418001008B54FF40F
:109A70007A7011490022FFF797FF41F288300F49B1
:109A80000022FFF791FF4EF660200D490022FFF7FC
:109A90008BFF4FF4FA700B490022FFF785FF64201B
:109AA00009490022FFF780FFBDE808404FF47A70B3
:109AB00006490022FFF778BF599B00003D9B00003C
:109AC000219B0000059B0000ED9A0000D19A000048
:109AD00008B5FDF7E1FABDE808404FF47A70024995
:109AE0000022FFF761BF00BFD19A000008B5FBF765
:109AF00035FCBDE80840642001490022FFF754BF4F
:109B0000ED9A000008B5FDF777F8BDE808404FF47E
:109B1000FA7002490022FFF747BF00BF059B000013
:109B200008B5FCF7E9FFBDE808404EF660200249A1
:109B30000022FFF739BF00BF219B000008B5FAF7EC
:109B4000F5FFBDE8084041F2883002490022FFF7E6
:109B50002BBF00BF3D9B000008B5FCF715F8BDE822
:109B600008404FF47A7002490022FFF71DBF00BF82
:109B7000599B000030B5114A13681546E3B1002225
:109B80009C68844213D1DC688C4210D119680AB9F0
:109B9000296000E011601A681AB1506859680144E0
:109BA00051600B201946BDE83040FDF7C3BC1C686E
:109BB00014B11A462346E3E730BD00BF88180010F1
:109BC000F8B505460E46134C22682AB92846314698
:109BD000BDE8F84001F04CBF526862B921680B2023
:109BE0000A68CF6822608C68FDF7A4FC002CEAD0DC
:109BF0003846A047E7E72846314601F039FF431CC5
:109C0000ECD023685968884234BFC0EB01020022BF
:109C10005A60F8BD881800102DE9F04FD0F804A064
:109C200087B004468846BAF8003059BA0289C1F3B1
:109C300003210231B2EB810F07D359BAC1F30321DB
:109C400089004942FDF796FD28B1204607B0BDE8DE
:109C5000F04FFDF7BBBD564B41461868D4F8049051
:109C6000FBF70FFEB9F8007006467FBABFB2B9F82D
:109C7000021049BA89B24429039111D1432F4BD123
:109C8000D8F82830002B47D05B68002B44D05A68A6
:109C9000002A00F08A80474909688A423CD184E062
:109CA000454B00251868424B2A46D3F800C0414B6B
:109CB0000CF0F0011B680491059303465BB3B3F805
:109CC00012B003998B4523D1D3F800B016B9BBF17C
:109CD000000F0AD0E34508D00499E02905D0BEB1B1
:109CE00093F808B01BF0200F12D02DB993F810B0E4
:109CF0001BF0040F08BF1D46B3F814B0BB4507D1D5
:109D0000D3F804B0BBF1000F49D005998B4546D07C
:109D10001A46DB68D2E735B9254BD8F804201B6812
:109D20009A4292D10025B9F806304BB123892046DA
:109D3000009320491E4A1123FBF726FB002884D1FB
:109D400020466FF00701FDF715FD00287FF47DAF79
:109D500065B1EE69002E3FF478AF0097286A294676
:109D60002246144BB04707B0BDE8F08F002E7FF4B9
:109D70006CAF0F4B1B6803F0F003E02B3FF465AFB3
:109D8000BAF8001049BAC1F3032102312046890014
:109D9000FDF7F0FC20460321FBF798F955E722B1C7
:109DA000D968D160044AD86013601D46BBE700BF84
:109DB00004110010001100108C180010F0B51A4D9D
:109DC00000242B689BB198420ED05E8A96420CD13B
:109DD0001F680FB9F82025E00029FBD00E68002E7F
:109DE000F8D0B74201D1F5E70124DB68EAE701B119
:109DF0000968016082B929684FF440420B465BB1A3
:109E00004FF6FF76B242E5D05E8A964203BF01323A
:109E100092B20B46DB68F2E7428214B92B682860E5
:109E2000C360002040B2F0BD8C1800102DE9FF4740
:109E30009A46037A0E46990605469046DDF830901C
:109E400002D56A8A3AB10CE010684946FBF719FD61
:109E50000028F6D03FE028462946FFF7AFFF00284C
:109E60007AD130460821FDF785FC08B934460CE06C
:109E7000012008210022FDF7D6FC0446002868D006
:109E8000338913B13146FDF7A0FD67686B8A5BBA71
:109E90003B809AFA9AFA0023A7F802A0BB71FB71E3
:109EA000D8F8003003F0F003E02B06D12B7C1A0722
:109EB00003D5637B43F0040363732B6813B909F183
:109EC000040A0BE0D9F80420934206D0B44202D031
:109ED0002046FDF77BFCFA203EE0AA4623895BBAC8
:109EE000BB802B7CDB0721D423899DF83420009391
:109EF00082B1082301932046112351464246FBF7C5
:109F00007BFABDF83830DB439BB2184400EB1040BD
:109F100080B205E02046514642461123FBF734FA51
:109F20004FF6FF73002808BF1846F8806A7AAB7AAC
:109F3000009211220192CDF80890204651464246E7
:109F4000FBF772FCB442054605D02046FDF73EFC07
:109F500001E0FF2000E0284640B204B0BDE8F087F1
:109F6000F0B514461268054602F0F002E02A85B00A
:109F70000CBF183020460F461E46FBF7AFFA68B1FB
:109F80009DF8283000900193BDF82C3028460293AC
:109F9000394622463346FFF749FF00E0FC2040B235
:109FA00005B0F0BD37B5858A8DE80C00021D2B4643
:109FB000FFF7D6FF03B030BD13B500240094019421
:109FC000FFF7CEFF02B010BD1FB5069C0094002421
:109FD00001940294FFF72AFF04B010BD70B5164635
:109FE000428A04460D4612B13DB12D6805E0014696
:109FF000FFF7E4FE0028F7D011E0237C094A43F084
:10A000000403237413686560A682184618B184425D
:10A0100004D0C068FAE7E360146000E0002040B2BA
:10A0200070BD00BF8C180010C16102627047000053
:10A03000094A01461368834209D1C368136008E0E6
:10A04000DA681AB18A4204BFCA68DA60DB68002B9A
:10A05000F6D10020FDF76EBA8C18001010B5002064
:10A06000FDF752FA044628B10021242202F0F2FA48
:10A07000FF23A372204610BD30B5044687B098B1C7
:10A080000B4B68468DE818008DF80C1001F008FCA9
:10A09000054601F0ABFD94F908300933A8BF2572DD
:10A0A00001F0B6FD284600E0F22040B207B030BD16
:10A0B000C1AC000030B5002389B0044601930D46C1
:10A0C00009B9F22055E00B600028FAD0C369002BD3
:10A0D0004ED0007A43B209334BDB04F11C0001A9D6
:10A0E000D4F8982001F0C4FC01300BD101F07EFDC2
:10A0F00094F908300933A4BFFD23237201F088FDD1
:10A10000FD2036E02378102B019B25D194F89C206C
:10A11000120700D553B9184A039402920BB11B8958
:10A1200000E0012302A8059301F0BAFB019A8AB965
:10A13000D4F8A83013B120460121984701F056FD0C
:10A1400094F908300933A4BFF423237201F060FDB1
:10A15000F4200EE0128901E01B681A89D4F8A830B7
:10A1600013B1204601219847019B00202B6000E09D
:10A17000F32040B209B030BDE3AB000030B50D466E
:10A1800087B0114600F0E0FB0446A0B10C4B0190F3
:10A19000684600938DF80C5001F082FB68B104F121
:10A1A0000C0001F0D8FC04F11C0001F031FC072088
:10A1B0002146FDF7BFF9002000E0204607B030BD82
:10A1C000E1A8000010B5044686B040B1054B6846D2
:10A1D0008DE8180001F064FB204600F0F4FB00203D
:10A1E00006B010BD67AA000030B5044687B0B8B10C
:10A1F000B1B1AAB10C4803918DE8110068460492F0
:10A200008DF8143001F04CFB054601F0EFFC94F999
:10A2100008300933A8BF257201F0FAFC284600E097
:10A22000F22040B207B030BD63AC000030B5044648
:10A2300087B0A0B10C4B68468DE818000391ADF8CB
:10A24000102001F02DFB054601F0D0FC94F90830F8
:10A250000933A8BF257201F0DBFC284600E0F2209C
:10A2600040B207B030BD00BFF1AA000020B10378B2
:10A27000102B01D1FFF71EBF6FF00D00704773B5B3
:10A2800005460E4609B9F22032E000230B60002893
:10A29000F9D0C2695AB30278102A25D10620019359
:10A2A000FDF732F9044658B901F0A0FC95F90830E1
:10A2B0000933A4BFFF232B7201F0AAFCFF2017E093
:10A2C000284601A9FFF7F6FE054620B106202146E3
:10A2D000FDF730F906E0019BA0812360019BA0609F
:10A2E00063603460284603E0FFF7E4FE00E0F320FB
:10A2F00040B202B070BD00007FB568B10378102B8A
:10A300000AD190F89C301B0706D5054B0190684692
:10A310000093039101F0C4FA07B05DF804FB00BF9D
:10A32000E3AB000030B5044687B090B10B4B6846F4
:10A330008DE81800039101F0B3FA054601F056FCD0
:10A3400094F908300933A8BF257201F061FC284652
:10A3500000E0F22040B207B030BD00BF81AB00008A
:10A3600030B5044687B0C8B10078102818D1CAB1FA
:10A370000E4803918DE8110068468DF81430049260
:10A3800001F08EFA054601F031FC94F908300933EA
:10A39000A8BF257201F03CFC284604E0F22002E050
:10A3A000FA2000E0104640B207B030BD21AC0000FA
:10A3B000002A0CBF0023022300290CBF194643F0DA
:10A3C0000101FFF759BE0000F0B50E468BB00746FD
:10A3D000F0B1E9B106AC2046002101F07DFB054655
:10A3E0008DF80700A8B90DF10703012202A90A4858
:10A3F000059302970396049401F028FA2946204613
:10A4000001F084FB204601F0A6FB9DF8070000E068
:10A41000F22040B20BB0F0BD19AD0000D36811B905
:10A42000FA21197004E00020187053680968196057
:10A43000906801F086BB2DE9F04116461F46BDF835
:10A440001880054608B1C36923B93046BDE8F0411C
:10A45000FDF7BCB90620FDF757F804460028F4D0F4
:10A460000660466007B13F68A760A4F80C802146EB
:10A4700005F11C00368901F0F1FA014620B12046B1
:10A48000BDE8F04100F05EBCD5F8A83013B1284615
:10A4900032469847BDE8F08110B544680146204631
:10A4A000FDF786FB20460949FDF784FB2046084955
:10A4B000FDF783FB204607490422FDF786FB204673
:10A4C0000549BDE81040FDF77BBB00BF77A8000041
:10A4D00027A80000D5A70000DDA40000F8B50025DE
:10A4E00004460E46456001F081FB267201F090FBA8
:10A4F000D4F8A830677865701BB1204604212A463D
:10A500009847D4F8A8301BB1002120460A46984746
:10A51000D4F8A8301BB12046022100229847E369F5
:10A5200023B104F11C00002101F098FAA36D23B1BE
:10A5300004F15800002101F091FA012F02D0033FED
:10A54000012F15D894F89C3023F0040203F0040383
:10A5500084F89C2003F0FF0253B9D4F8A43004F12E
:10A560000C001E71C4F8A420BDE8F84001F0E9BA5F
:10A57000F8BD38B5044680B3D0F8A43003B11A71E1
:10A580002378102B03D112B92046FFF785FF94F8EA
:10A590009C3083F0040523F0040384F89C30C5F359
:10A5A00080050023C4F8A430637045B901F01EFB98
:10A5B00094F908300933A8BF257201F029FBD4F8BB
:10A5C000A8301BB120460221002298473DB104F17A
:10A5D0000C0001F0B6FA002002E0FA2000E0284664
:10A5E00040B238BDF8B590F89C30D0F8A42013F0F4
:10A5F000020F08BF177C137CD0F8A0609168D26866
:10A60000044640683144C6EB02060CBFC7F380071E
:10A610000127B0F86E50B6F5803F32BFB6B24FF6A4
:10A62000FF7643F00203FFB2B5423CBF43F00203A2
:10A630002E4687B196420ED294F89C3043F0100318
:10A6400084F89C30D4F8A8301BB120460321324650
:10A650009847F9250AE03246FEF75AFD05460FB144
:10A660006A1CE9D06B1CDBB2012B0BD9D4F8A430E7
:10A6700004F10C001D710023C4F8A430637001F0D4
:10A6800060FA2AE0636840F2B452B3F86E10914267
:10A6900003D9B3F87030012B06D9D4F8A8301BB118
:10A6A000204603213246984795B9D4F8A030606817
:10A6B0001E44D4F8A430C4F8A060DB689E4206BFF4
:10A6C000C4F8A05001262E46FEF720FF2EB1CDE79C
:10A6D0006B1CCBD16068FEF719FF0020F8BD0000AD
:10A6E000F8B5D0F8A43004461D7AEB1E05F002063A
:10A6F00005F001075D425D41F6B21DB140680021E1
:10A70000FDF756FA6068037C012B03D10021FDF7A9
:10A710005AFA16E037B10021FDF74CFA60680021C3
:10A72000FDF751FA1EB160680021FDF746FA6DB1E0
:10A73000606800210422FDF748FA60680021FDF7F7
:10A740003FFA1DB16068FDF733FC04E060683946EC
:10A750003246FDF78DFC024618BBD4F8A4301871C0
:10A76000C4F8A400607060602DB1D4F8A83013B1B3
:10A7700020460421984737B1D4F8A8301BB10021F6
:10A7800020460A46984736B1D4F8A8301BB1204677
:10A7900002210022984704F10C00BDE8F84001F0C6
:10A7A000D0B960680849FDF708FA606807490422D3
:10A7B000FDF70BFA60680649FDF702FA606821466A
:10A7C000BDE8F840FDF7F4B927A80000D5A70000C0
:10A7D000DDA4000010B543780446012B02D1FFF739
:10A7E00001FF03E0042B01D1FFF77AFF94F89C20CE
:10A7F000D30616D56368A3B1B3F86E0040F2B45126
:10A8000088420ED9B3F87030012B0AD8D4F8A8309A
:10A8100022F0100284F89C201BB120460221002265
:10A820009847002010BD38B543780446012B1546E3
:10A8300002D1FFF7D7FE03E0042B01D1FFF750FF51
:10A840006368B3B1B3F86E1040F2B452914210D9BC
:10A85000B3F87030012B0CD894F89C3023F010031F
:10A8600084F89C30D4F8A8301BB1204602212A4637
:10A870009847002038BDF8B515461F46064648B330
:10A88000C46954B90AB9002427E008461189FDF7C4
:10A890005CF92846FCF79AFF1FE001F0A7F996F94A
:10A8A00008300933A8BF377201F0B2F90DB12F8912
:10A8B00000E02F4606F11C00294601F0CFF80446BF
:10A8C00050B9D6F8A830002BDDD0304621463A46A4
:10A8D000984702E0FA2400E0FF2460B2F8BD0000CF
:10A8E00038B50023056803716B68044623BB2B78D9
:10A8F00003F0F003102B12D0202B1BD1FFF7AEFB7F
:10A9000068602268536883B112780E49222A04BF16
:10A9100001221A7422685068FFF786FB0CE0FDF7ED
:10A92000B1FC6860206843680BB9FF2303E0FFF7C0
:10A93000B3FD01E0FA2323712068BDE838400C30F4
:10A9400001F0FFB837A400002DE9F04106460720CA
:10A950008846FCF7D9FD0025044688B300F10C07B2
:10A960000670057245602946384601F0B5F806467E
:10A9700030B107202146FCF7DDFD2846BDE8F08117
:10A9800004F11C00082101F023F848B1384601F019
:10A99000E2F807202146FCF7CDFD3046BDE8F08106
:10A9A0004FF0FF32A0656070C4F89420C4F8A8800E
:10A9B000C4F8A400C4F8A000C4F8980084F89C006F
:10A9C0002046BDE8F08110B504460C3001F0C3F814
:10A9D0000023E36021460720BDE81040FCF7AABD34
:10A9E00037B5C3690446FBB104F11C05284601A92B
:10A9F00001F060F8013012D02378102B0BD1019DAB
:10AA0000002DF1D0606810B12989FDF79EF8284625
:10AA1000FCF7DCFEE8E7019800F094F9E4E728464B
:10AA200000F0F6FF0023E361A36DD3B104F15805F4
:10AA3000284601A901F03EF801300DD0019D2846BD
:10AA4000FFF7CEFF686818B1FDF786FB00236B6047
:10AA50002846FFF7B8FFE9E7284600F0D9FF0023B2
:10AA6000A36503B030BD10B50446006843782BB130
:10AA7000023B012B02D9FB2323712FE0FFF7B0FF2C
:10AA800023685A68E2B1197801F0F001102908D062
:10AA9000202912D10023136223685868FFF7C8FAEF
:10AAA0000BE004225A70032323722368C3F8A440E6
:10AAB0002068BDE81040FFF713BE236800225A60EB
:10AAC0002068D0F8A83013B100210A4698472068C2
:10AAD000D0F8A83013B10221002298472068C3683B
:10AAE00023B10C30BDE8104001F02BB810BD0000C0
:10AAF00010B503680446586808B9F42336E01A789C
:10AB000002F0F002102A07D0202A2ED1A168A289D3
:10AB1000FFF764FA20712AE05A780AB1F72325E09A
:10AB20001846FFF7B9FC2368A1685868A289134B3F
:10AB3000FDF7BAFB2071D0B92368032193F89C205C
:10AB40005970236812F0020F93F89C2005D042F050
:10AB5000040283F89C20FB2308E022F0040283F81F
:10AB60009C202368C3F8A44010BDFA2323712068F9
:10AB7000BDE810400C3000F0E4BF00BF73A500003A
:10AB800073B5036805461A7A51B2093101DA0271C8
:10AB900020E0F32202715868E0B11B7803F0F00363
:10ABA000202B17D1AC6814F10802A67B01D0A36852
:10ABB00033B9216806F00202238AFFF7F3F908E0AF
:10ABC00006F00206A3890096218A01912168FFF709
:10ABD000C7F9287128680C3002B0BDE8704000F059
:10ABE000B0BF70B500230371036804465A682AB9E0
:10ABF0002068BDE870400C3000F0A3BF1B78102B1C
:10AC0000F6D18568B5F5803F236834BFAEB24FF604
:10AC1000FF7658683146FCF798FFAD1BF2D1E7E7A5
:10AC200003681A7A51B2093116DB1A78102A12D148
:10AC30005A780AB1FB220FE0596851B101215970CD
:10AC40000368C3F8A4000368C3F8A0200068FFF7F6
:10AC5000C9BCF32200E0FA22027103F10C0000F0FB
:10AC600070BF03685B682BB3017C826809B11B6805
:10AC700000E05B6813600023037103681A7802F038
:10AC8000F002102A0DD0202A16D1027C5B6812B186
:10AC9000C2685B8A0CE01A7C52070BD5C2689B8A9B
:10ACA00006E0017CC2685B6809B19B8B00E0DB8B2E
:10ACB000138001E0F323037100680C3000F041BF02
:10ACC00010B504460068427812F0FD0F01D0FB2356
:10ACD0001BE04368C3B10378102B15D1237A032BF3
:10ACE00003D0022A01D1F3230FE0DB0701D5FFF7E0
:10ACF00077FE236804225A702368C3F8A4402068B2
:10AD0000BDE81040FFF7ECBCFA2323710C30BDE81E
:10AD1000104000F016BF000038B50446C568234651
:10AD200003C8074AFCF7CEF92870E36893F90030AE
:10AD3000053304D0A068BDE8384000F002BF38BD3C
:10AD40001DA4000010B5044660B1006820B1FCF7F6
:10AD50003DFD00236360236021460620BDE81040CE
:10AD6000FCF7E8BB10BD10B5044630B1006808B16F
:10AD7000FCF72CFD00236360236010BD70B50E4608
:10AD800015460446A8B1006808B1FCF71FFD002075
:10AD900001460222FCF747FD206010B96060FF20E9
:10ADA00008E04660236800201D815D8123686360A0
:10ADB00000E0F22040B270BD13B501A90446FFF7D0
:10ADC00003FB20B10B4BD2221A6000200FE00A4B8C
:10ADD000019A0A491A600A4A13600A4B5060596086
:10ADE0000221996004211C60D9601A61184602B0E2
:10ADF00010BD00BFB0180010A4180010B418001047
:10AE0000A818001090180010032808D818234343EE
:10AE1000044AD018D358002B08BF002070470020E8
:10AE2000704700BFBC1800102DE9F84380468946E2
:10AE3000002400F0DBFE18236343144E9D59E5B94E
:10AE4000F71846F8038000F0E3FE7D603D817D81C8
:10AE500098F80030102B04D119F1000118BF01211E
:10AE600000E00121182303FB04660023B181F38174
:10AE7000336173612046BDE8F883013400F0C8FEF9
:10AE8000042CD6D14FF0FF30BDE8F883BC18001079
:10AE90002DE9F84F0F46044600287DD0D0F8945095
:10AEA000002D0EDA00F0A2FED4F894500346002DD7
:10AEB00005DA17B9013DC4F89450184668E000F06F
:10AEC000A7FE2846FFF7A0FF0446002864D000F044
:10AED0008DFE0646042F12D8DFE807F003060A0CA1
:10AEE0000F006389013301E06389013B638106E060
:10AEF000012300E00023A38101E00123E3816369D2
:10AF0000002B44D005F007084FF0010909FA08F9B1
:10AF1000EF10224B1D68002D39D06B693BBBB4F993
:10AF20000A20002A06DDAB6823B1DB5D43FA08F393
:10AF300003F00103A2894AB13BB9EA6832B1D35D9B
:10AF400043FA08F303F0010300E00123E2893AB178
:10AF50003BB92B695BB1DB5D13EA090F01D106E058
:10AF60002BB101236B6105F1180000F0EAFDDFF859
:10AF700030A03046DAF800B000F04AFE00F036FEAD
:10AF8000DAF8003006469B45C3D12D68C3E730464A
:10AF9000BDE8F84F00F03CBEBDE8F88FB8180010CF
:10AFA0001C1900102DE9F04F002689B0454F039081
:10AFB000894692469B468DF814608DF818608DF88E
:10AFC0001C603446039B9C426BDA00F00FFE032C9E
:10AFD00008D857F8045C35B13A68FB88B7F80880A0
:10AFE0007D8903E00025A8462B462A46029201935C
:10AFF00000F00EFE029A019BB9F1000F1AD0082052
:10B0000094FBF0F019F800C004F007014CFA01FCC1
:10B010001CF0010F0ED012B91BB2002B0ADD08ABD9
:10B020001844012303FA01F110F80C3C01361943CE
:10B0300000F80C1CBAF1000F17D0082394FBF3F3AF
:10B040001AF8031004F007021141C8070DD5B8F132
:10B05000000F0AD008A90B44012101FA02F213F8EB
:10B06000081C01360A4303F8082CBBF1000F15D069
:10B07000082394FBF3F31BF8031004F007021141BB
:10B08000C9070BD555B108A90B44012101FA02F2F9
:10B0900013F8041C01360A4303F8042C0134183752
:10B0A00090E79DF81420129B30461A709DF81820E6
:10B0B000139B1A709DF81C20149B1A7009B0BDE8F0
:10B0C000F08F00BFC01800107047F8B5FFF79CFE66
:10B0D0000446F8B1006828B10778B7F110035F4261
:10B0E0005F4100E007460025FFF76CF866682581A0
:10B0F0006560256100F07AFD256000F089FD30462D
:10B100005EB11FB1FCF762FB2846F8BDFFF71AFEDF
:10B110003846F8BD4FF0FF30F8BDF8BD73B50D46A9
:10B120001646FFF771FE0446E8B1102E16D16B7873
:10B13000022B13D1AB0711D16B6802A941F8043D72
:10B140006A8852BA006892B2FFF770F848B140427C
:10B150000F2803D8064B53F8203000E00523236165
:10B1600001E0206101E04FF0FF3002B070BD00BF90
:10B17000282301002DE9F04F00258BB001911746DF
:10B1800098460495FFF740FEDDF8549004460028E9
:10B1900000F0908063680BB104932EE018F0080F64
:10B1A00004D1236893F89C30990708D5B4F90A3084
:10B1B000002B04DC002D75D10B2323617AE020687D
:10B1C00004A90378102B02D1FFF750F801E0FFF734
:10B1D00056F880B1002D65D140B243420F2B96BF87
:10B1E000514A052352F8233010F10C0518BF0125F0
:10B1F0002361684295E0049B6360236801991B7892
:10B200002944102B049B14BFD3F800B09B46BBF815
:10B2100008A023895846C3EB0A0A1FFA8AFA574541
:10B2200094BFBEB256463246FCF721FC2068354436
:10B230000378102B0CD1BF1B0AD09BF80D20D2072E
:10B2400006D4B4F90A20002A02DD18F0010B06D05A
:10B25000149A12B1B9F1000F2FD14FF0010B18F071
:10B26000010F1AD123681A78102A0AD1C6EB0A0AEC
:10B27000BAF1000F05DD049B636023891E4426811B
:10B280000BE00022626022811B780498102B02D10F
:10B29000FCF79CFA01E0FFF755FDBBF1000F3FF40E
:10B2A00079AF1DB120682946FFF726F800232361F6
:10B2B000284636E04FF0FF3033E0102B08D105A9C7
:10B2C0000DF10E020023FEF78FFF0DF1140B05E0C8
:10B2D000049B03F1080B9B89ADF80E3010231A462E
:10B2E00006A80021009301F0B5F9009B8DF81830F5
:10B2F00002238DF81930BDF80E305BBAADF81A3064
:10B30000DBF8003014980793D9F8003006A9102B09
:10B3100084BF1023C9F80030D9F8002000F039FBB1
:10B320009BE70BB0BDE8F08F2823010013B5002484
:10B3300000940194FFF71EFF02B010BD2DE9F04705
:10B3400086B08146884616469A46FFF75DFD0E9CFC
:10B350000F9F0546B0B102681378102B06D14846FE
:10B3600041463246534600F041F839E0B6B204B9DE
:10B370005FB1102F04D16378022B01D1A30704D051
:10B3800005232B614FF0FF302AE000230293019345
:10B390008DF8123034B16368039363885BBAADF8FB
:10B3A000103002E00394ADF8104001A84146324647
:10B3B000FFF7E4FC044620B9286801A9FEF7B2FFB4
:10B3C000044601A8FFF7CFFC63B25B420F2B96BF88
:10B3D000054A052352F823302B61002CD2D1304688
:10B3E00006B0BDE8F08700BF282301002DE9F34136
:10B3F00080460F4614461E46FFF706FD0546D0B1AF
:10B4000000680378102B09D0002300930193404675
:10B41000394622463346FFF791FF28E016F008012F
:10B4200003D190F89C309B0708D540F668339C42C6
:10B4300004D95A232B614FF0FF3018E016F0100F9B
:10B440000CBF0123032300290CBF0026042622463B
:10B4500033433946FEF784FF43420F2B96BF054A1C
:10B46000052352F823302B610028E4D1204602B096
:10B47000BDE8F08128230100022938B507D003294F
:10B4800002D001292AD10DE04020D1B204E0882A5F
:10B4900014BF202021200021124AFEF76FFE04462F
:10B4A00068B91BE0102000210E4AFEF767FE044633
:10B4B000A0B190F89C3043F0080380F89C302046FF
:10B4C0000021FFF7B1FC431C054618BFC4F89400E7
:10B4D00002D12046FEF776FE284638BD4FF0FF30F9
:10B4E00038BD00BF91AE00002DE9F04F95B008AF18
:10B4F00001970DF11C0A09AFCDF800A00297804614
:10B500000E4615461C46FFF74DFD8146002840F0CB
:10B51000EE801E9F2FB13B681BB97B68002B00F0AB
:10B52000E680002110A80A910B910C960D950E94BF
:10B530000F910DF1280B00F0CFFA002840F0E480C5
:10B5400000F054FB744A13680A930BB1C3F804B0BB
:10B55000724BC2F800B01A684FF0000901321A604D
:10B5600000F056FBC14538DA4EB1082299FBF2F2E1
:10B57000B15C09F0070241FA02F2D20715D44DB1CD
:10B58000082299FBF2F2A95C09F0070241FA02F2E3
:10B59000D3070AD4F4B1082299FBF2F2A15C09F0B6
:10B5A000070241FA02F2D70714D5B9F1030F07D801
:10B5B000182101FB09F15A480A5812B1421800E05B
:10B5C0000022059200F012FB059A51690131516188
:10B5D00000F01EFB09F10109C4E708AA09AB0192BA
:10B5E0000293CDF800A0404631462A462346FFF795
:10B5F000D9FC8146A8B91E9F6FB179684FF47A7360
:10B60000386801F5FA7191FBF3F103FB0011002991
:10B6100008BF012100E0014610A800F077FA0746B4
:10B6200000E00027002343453DDA4EB1082193FB9B
:10B63000F1F1705C03F0070140FA01F1C80715D47D
:10B640004DB1082193FBF1F1685C03F0070140FA6A
:10B6500001F1C9070AD424B3082193FBF1F1605C1E
:10B6600003F0070140FA01F1CA071AD5032B0AD8E3
:10B670004FF0180C0CFB03FC29485CF8001021B1BA
:10B6800000EB0C0202E0002200E00A46049305925F
:10B6900000F0ACFA059A51690139516100F0B8FA2D
:10B6A000049B0133BFE700F0A1FA0A9B0BB10B9991
:10B6B000596019490A685A4518BF0B990B60174B16
:10B6C00019680131196000F0A3FA10A800F043FADC
:10B6D00001370CD008AB09AF0193CDF800A0029759
:10B6E000404631462A462346FFF75CFC814616B1A8
:10B6F0009DF81C30337015B19DF820302B7034B19B
:10B700009DF82430237002E04FF0FF3000E04846FF
:10B7100015B0BDE8F08F00BFB81800101C1900105C
:10B72000BC18001038B50D46FFF76EFB044638B361
:10B73000006820B10378102B03D05F2007E06B2056
:10B7400005E035B1012D07D0022D08D0162020616B
:10B7500038BD2A46012104E02A46002101E00122E9
:10B760001146FEF725FE43420F2B96BF064A0523DE
:10B7700052F82330003018BF01202361404238BD09
:10B780004FF0FF3038BD00BF2823010007B51C4B28
:10B790001B6813B11B4A106898471B4801A9FEF7A4
:10B7A0000FFA019B1A78042AF7D8DFE802F00307A2
:10B7B000191F1500986803680430EDE7D968986888
:10B7C00091F8392012F0600F02D0F9F7F3FA01E096
:10B7D000F9F7A4FE09200EE09A68D868904709E0BE
:10B7E00003F1080007C8FEF7DFF803E0D86819691D
:10B7F000FEF7C0F908200199FBF79CFECDE700BFDA
:10B80000601900105C19001020190010F8B50E4DD9
:10B8100006462B680F4693B10920FBF775FE0446D8
:10B8200078B1012303708660C7602146284600F086
:10B8300015F938B109202146FBF77CFE01E0FA201A
:10B8400000E0FF2040B2F8BD201900102DE9F041C2
:10B85000124D06462B680F469046CBB10820FBF7E9
:10B8600053FE0446B0B1042303708660C7602146CE
:10B870002846B8F1000F03D000F0E0F800200AE0FD
:10B8800000F0ECF838B108202146FBF753FE01E048
:10B89000FA2000E0FF2040B2BDE8F081201900103E
:10B8A00030B504460A4887B003686BB1002501A98A
:10B8B0008DF80450039400F0C1F8606829460C30FC
:10B8C00000F024F9207A00E0FA2040B207B030BD41
:10B8D0002019001037B504460D46FBF783FC094BD1
:10B8E00008211C60084B09481D6000F071F8002217
:10B8F000009207494FF48063064800F099F903B0BD
:10B9000030BD00BF601900105C1900102019001034
:10B910008DB700006823010010B5002210F001036C
:10B9200004D0A1B310F8012B1202013910F0030466
:10B9300005D002291ADB30F8024B12190239082906
:10B940000BDB50F8044B121942F1000250F8044B83
:10B95000121942F100020839F1E7022906DB30F83A
:10B96000024B121942F100020239F6E719B10478CC
:10B97000121942F10002C2F30F44C2F30F0212196E
:10B98000C2F30F44C2F30F02121903B152BA1046A8
:10B9900010BD130911D051F804CB40F804CB51F875
:10B9A00004CB40F804CB51F804CB40F804CB51F859
:10B9B00004CB40F804CB013BEDD112F00F0305D0CE
:10B9C00011F801CB00F801CB013BF9D17047000021
:10B9D000082970B504460D4602DD0C48F6F7A2F9B9
:10B9E00004F10C0630223046002100F033FE2046E0
:10B9F000A660002140F8045FF7F75AFC2060D0F100
:10BA0000010038BF0020404270BD00BF7523010017
:10BA10001FB50346196801A80022F7F783FC019BB4
:10BA2000102B05D1044805B05DF804EBF6F77AB9A0
:10BA300005B05DF804FB00BF8E23010008B54FF090
:10BA4000FF320068F7F74EFC20B10348BDE808401C
:10BA5000F6F768B908BD00BFA323010008B50022AE
:10BA60000068F7F73FFC003018BF0120404208BDD6
:10BA7000F0B585B0144607460E46F6F71BF8002CC5
:10BA800014BF22464FF0FF320546396801A8F7F788
:10BA900049FC019B102B18BF4FF0FF3008D1029BCF
:10BAA0003360F6F707F84FF47A73401BB0FBF3F0FE
:10BAB00005B0F0BD1FB503460C4601A81968002269
:10BAC000F7F730FC019B102B05BF029B00204FF0C5
:10BAD000FF30236004B010BD70B500F108050446C6
:10BAE0000E4608220021284600F0B4FD204640F80A
:10BAF000045F3146F7F7F4FA206010B90248F6F710
:10BB000011F9002070BD00BFB823010070B50C46CC
:10BB10000646F5F7CFFF002C14BF21464FF0FF314A
:10BB200005463068F7F7F6FA002807DDF5F7C2FF9B
:10BB30004FF47A73401BB0FBF3F070BD4FF0FF3051
:10BB400070BD08B50068F7F7F3FA18B1BDE8084012
:10BB5000F6F7AEB808BD704738B500F108050446E1
:10BB600000210C22284600F075FD204640F8045FB5
:10BB7000F7F72EFA2060D0F1010038BF00204042D4
:10BB800038BD000008B54FF0FF310068F7F73AFA0A
:10BB900020B10348BDE80840F6F7C4B808BD00BFAF
:10BBA000D223010008B50068F7F738FA20B103483E
:10BBB000BDE80840F6F7B6B808BD00BFE8230100AD
:10BBC00008B5F5F777FF0648F7F702FA054B186056
:10BBD00020B90548BDE80840F6F7A4B808BD00BF85
:10BBE00078010010241B00100024010008B5064B4A
:10BBF0004FF0FF311868F7F705FA10B10348F6F770
:10BC000091F8012008BD00BF241B00101024010082
:10BC100008B5054B1868F7F701FA20B10348BDE8ED
:10BC20000840F6F77FB808BD241B00102824010047
:10BC30002DE9F0471F46164B91461A688A46052A99
:10BC4000984602DD1348F6F76DF8D8F8003048251D
:10BC50005D43114E0133C8F80030089B7419C4F8D5
:10BC600004A02381E760384600F0B2FC206110B9DF
:10BC70000A48F6F757F8201D4946F7F701F87051C2
:10BC800010B90748F6F74EF82046BDE8F08700BF28
:10BC90006419001042240100681900105F2401009B
:10BCA00081240100704710B5002104461022143091
:10BCB00000F0D0FC0023237010BD10B50446FFF740
:10BCC000F2FF204610BD00007FB50D460446164623
:10BCD000FFF7E9FF0DF10A0300930DF10B03019348
:10BCE00028460E4902AA0DF1090300F073FE04284C
:10BCF00006D02846FFF760F858B103691B6800E0DA
:10BD000002AB1B68A3610223637576BA0020E6824A
:10BD100001E04FF0FF3004B070BD00BF9E24010071
:10BD20004FF0FF3202600122027140F2DC52826069
:10BD3000704701718260704710B503680446013393
:10BD400002D04FF0FF3010BD02200022FFF794FB1D
:10BD50000028F6DB2060002010BDF0B50646006824
:10BD600085B0082590FBF5F40DF1100C644400F04B
:10BD700007004FF0010C0CFA00F000270DF10C0E3B
:10BD8000BA4214BF72463A46BB428DF80C703B462D
:10BD900004F8040C00914FF00400114614BF7246E1
:10BDA0003A46FFF7A1FBB8420FDD326804A992FBC7
:10BDB000F5F30B4413F8040C02F00702104100F0F5
:10BDC000010080F00100404201E04FF0FF3005B07B
:10BDD000F0BD01220023FFF7C0BF00220123FFF7BF
:10BDE000BCBF10B50446006800280BDB11B102216E
:10BDF000FFF798FC2068FFF768F94FF0FF332360E6
:10BE0000002010BD4FF0FF3010BD10B501210446D9
:10BE1000FFF7E7FF204610BD30B54FF47A72044DAE
:10BE2000B1FBF2F405FB04114A430460426030BDEB
:10BE300018FCFFFF10B50446FFF772FF04F10C0079
:10BE4000FFF73BFF002384F83030204610BD70B56B
:10BE50000D46012104461646FFF76EFF002813DB4E
:10BE6000294604F10C003246FFF72EFF054658B96B
:10BE7000206804F120011022FFF750F9002806DAAB
:10BE800020460121FFF7ADFF4FF0FF3502E001230F
:10BE900084F83030284670BD73B503680446002B23
:10BEA0000D46164619DB90F83030B3B1037943B92B
:10BEB000A1686846FFF7B0FF20466946FFF78DFF8F
:10BEC00058B90023206829463246FFF78FFA031C31
:10BED00018BF012384F8303001E04FF0FF3002B08A
:10BEE00070BD73B503680446002B0D46164619DB7A
:10BEF00090F83030B3B1037943B9A1686846FFF7D1
:10BF00008BFF20466946FFF764FF58B9002320687D
:10BF100029463246FFF70AFA031C18BF012384F8AA
:10BF2000303001E04FF0FF3002B070BD00B589B095
:10BF300006A8F5F749FF9DF819209DF818300092E2
:10BF40009DF81A20132101929DF81B2006480292A9
:10BF50009DF81C2003929DF81D200492034A00F0D6
:10BF6000E3FC09B05DF804FB481B0010AE2401009F
:10BF7000F0B5164C85B007460E461548002115460B
:10BF8000FFF7A8FC4FF0FF311248F8F77BF8204686
:10BF90000021442200F05EFB002300930E4B394643
:10BFA00001930E4B3246029320462B46FBF712FBC1
:10BFB0002046FBF749FB20460949FBF7ADFB094941
:10BFC000204605B0BDE8F040FBF772BB5C1B0010DB
:10BFD000FDBF0000281B0010154500000DB8000033
:10BFE000E9BF000009C0000090F83930DB0602D537
:10BFF0000148F8F74AB87047D41B00100148F8F719
:10C0000044B800BF281B001010B590F83930044622
:10C01000DB071BD50430F9F727FD01460C4800F07B
:10C0200052FD04F10C00F9F71FFD0146094800F02C
:10C030004AFD04F10800F9F717FD0146064800F033
:10C0400042FDBDE810400548F8F71FB810BD00BF1D
:10C05000A01B0010B11B0010C21B0010381B0010E9
:10C0600008B5064B01221A70FFF760FF0020014659
:10C070000246FFF77DFF002008BD00BF5B1B0010DC
:10C0800010B50446F8F74AFB094B0A481B781BB168
:10C09000FAF71AFE084802E0FBF7DCFA07482146E7
:10C0A000F7F7F0FF0028CCBF00200120404210BD70
:10C0B0005B1B00105C1B0010381B0010D41B001011
:10C0C00070B5114E114D124C30460021F7F7C7FFE5
:10C0D0003046104E2246294600F020F83046002116
:10C0E000F7F7BDFF30460C4E2246294600F016F801
:10C0F00030460021F7F7B3FF304629462246BDE817
:10C10000704000F00BB800BF281B001091400000E9
:10C11000C8000010D41B0010381B0010034608464E
:10C12000194600F007B8014600200246034602F017
:10C1300015BA000070B5064C06460D4613462CB1E4
:10C1400031462A46022002F009FA70BD204670BD31
:10C150005DE50000014B1868704700BFDC0100106E
:10C1600008B5074B044613B1002102F053FA054B02
:10C170001868836A03B198472046F5F759FF00BF56
:10C1800015E60000302501008A892DE9F0410546B9
:10C1900010070C4657D44B68002B02DC0B6C002BAD
:10C1A00018DDE66AB6B102F48052002392B22F681D
:10C1B0002B600AB1626D10E0216A28460123B04766
:10C1C000411C024609D12B683BB11D2B01D0162B17
:10C1D00046D12F600020BDE8F081A3895B0705D51B
:10C1E0006368D21A636B0BB1236CD21AE66A2846D5
:10C1F000216A0023B047461CA28905D12B681BB1D8
:10C200001D2B01D0162B19D1002363602369D104A3
:10C21000236004D5421C01D12B6803B96065616BB2
:10C220002F600029D6D004F14403994202D0284659
:10C2300000F018FA00206063BDE8F08142F040028F
:10C24000A281BDE8F0810E69002EC3D00B680E609C
:10C25000C6EB030893070CBF4B6900238B6012E009
:10C26000A3894FF0FF3043F04003A381BDE8F08184
:10C27000A76A2846216A32464346B8470028EFDDC0
:10C280000644C0EB0808B8F1000FF1DCA2E700009B
:10C2900038B50B6905460C46DBB118B183690BB99B
:10C2A00000F086F80C4B9C4201D16C6808E00B4B07
:10C2B0009C4201D1AC6803E0094B9C4208BFEC688A
:10C2C000B4F90C302BB128462146BDE83840FFF7C1
:10C2D0005BBF002038BD00BFCC240100EC2401006E
:10C2E0000C250100014620B9044B0549186800F0EF
:10C2F000DFB8044B1868FFF7CBBF00BF3025010043
:10C3000091C20000DC010010F8B5074600F14804B6
:10C3100094B1A5686668013E0CD4AB89012B07D99E
:10C32000B5F90E30013303D038462946FFF7B0FF88
:10C330006835F0E72468EBE7F8BD0000002310B58E
:10C34000044603604360836081814366C281036168
:10C350004361836119465C30082200F07BF9054B8C
:10C3600024626362044BA362044BE362044B2363C5
:10C3700010BD00BF29CA00004FCA000087CA0000D4
:10C38000ABCA000070B54B1E68255D430E4605F133
:10C39000740100F0ABF9044640B1002180E842008E
:10C3A0000C30A06005F1680200F054F9204670BD21
:10C3B000836910B5044633BB8364C3640365124BC1
:10C3C000124A1B688262984204BF0123836100F015
:10C3D0001FF86060204600F01BF8A060204600F0C7
:10C3E00017F80421E06000226068FFF7A7FFA0684B
:10C3F00009210122FFF7A2FFE06812210222FFF7C4
:10C400009DFF0123A36110BD3025010009C3000079
:10C41000F8B51B4B07461E68B36913B93046FFF7E2
:10C42000C7FF4836B4687368013B04D4B4F90C50B4
:10C4300075B16834F8E733682BB938460421FFF743
:10C44000A1FF306008B13668ECE70C233B60F8BD13
:10C450004FF6FF73E3810123A38165662560A56024
:10C46000656025616561A56104F15C0029460822CB
:10C4700000F0F0F86563A563A564E5642046F8BDA7
:10C480003025010038B5084D084C641BA41005EB9D
:10C49000840524B155F8043D013C9847F9E7BDE80F
:10C4A000384005F0A5BC00BF280200102C02001087
:10C4B0002DE9F8438046894600F14804002694B1EE
:10C4C000A5686768013F0CD4AB89012B07D9B5F982
:10C4D0000E30013303D040462946C847064368352D
:10C4E000F0E72468EBE73046BDE8F88370B50E4B03
:10C4F0000E4D0024ED1AAD101E46AC4204D056F885
:10C50000242090470134F8E705F06CFC084D094BF6
:10C510000024ED1AAD101E46AC4204D056F824207B
:10C5200090470134F8E770BD1C0200101C02001097
:10C53000280200101C020010F0B58B8991B09E07F4
:10C5400005460C4625D4B1F90E10002908DAA38956
:10C55000002713F0800F14BF40264FF480660DE0D3
:10C5600001AA02F01DFF0028F1DB029F4FF4806654
:10C5700007F47047B7F500514F424F412846314606
:10C5800000F0B4F860B9A3899A051DD443F0020302
:10C59000A38104F14703236023610123636113E056
:10C5A0000A4BAB62A389206043F08003A381206122
:10C5B00066614FB12846B4F90E1002F003FF18B1BE
:10C5C000A38943F00103A38111B0F0BD09C30000AA
:10C5D000024B0146186800F089B800BFDC0100106A
:10C5E000024B0146186800F03DB800BFDC010010A6
:10C5F00010B5C9B202449042034605D01C78013000
:10C600008C42F8D1184610BD002010BD10B5002393
:10C61000934203D0CC5CC4540133F9E710BD81428E
:10C6200070B501D300230EE08C18A042FAD2851811
:10C63000134613F1FF3305D351426618F65C2944C3
:10C64000CE54F6E770BD934203D0CC5CC4540133A2
:10C65000F9E770BD02440346934202D003F8011B80
:10C66000FAE7704730B500293CD051F8042C0B1F75
:10C670001D49002AB8BF9B180A680C4612B95A60B7
:10C680000B6030BD93420DD219685818904203D107
:10C690005A581144426819605A60236030BD99426B
:10C6A00003D80A4651680029F9D1146815199D422A
:10C6B0000AD11B682344D0188842136012D108683D
:10C6C000034413604B680CE002D90C23036030BDB7
:10C6D00018681C188C4203D10C6849682044186003
:10C6E0005960536030BD00BFE81B001070B5CD1C11
:10C6F00025F0030508350C2D38BF0C25002D064606
:10C700003FDB8D423DD3214B1C6818462146A1B129
:10C710000B685B1B0ED40B2B03D90B60CC18CD50D0
:10C720001FE08C4202D1626802601AE04B686360CD
:10C730000C4616E00C464968E9E7154C23681BB91E
:10C74000304600F0E1F820602946304600F0DCF881
:10C75000431C014615D0C41C24F0030484420AD1B2
:10C76000256004F10B00231D20F00700C31A0BD035
:10C770005A42E25070BD3046611A00F0C5F80130EF
:10C78000EED10C233360002070BD00BFE81B001009
:10C79000E41B00100FB40A4B13B51C6824B1A36945
:10C7A00013B92046FFF704FE05AB2046A168049AA2
:10C7B000019300F083FD02B0BDE8104004B0704763
:10C7C000DC01001070B50E46054618B183690BB93F
:10C7D000FFF7EEFDAC68A389190701D5236983B97A
:10C7E0002846214601F04CFE58B14FF0FF3070BD95
:10C7F000002B0EDB236816F8012C1A702368013316
:10C800002360A36816F8012B013BA360002AEFD137
:10C8100017E0A269934209DB236816F8012C1A700D
:10C82000236819780A29EAD1284602E016F8011C83
:10C830002846224601F0BEFDB0F1FF325042504181
:10C84000D2E7002B16DAA269934208DB23680A229A
:10C850001A7023681978914210D1284601E02846C1
:10C860000A21224601F0A6FDB0F1FF33584258419B
:10C8700030B1BAE723680A221A70236801332360B3
:10C880000A2070BD024B01461868FFF79BBF00BF2E
:10C89000DC010010194B10B51C68A36BD3B918202C
:10C8A000FFF796FE43F20E33A06303804AF6CD33C2
:10C8B000438041F2342383804EF26D63C3804DF692
:10C8C000EC630381052343810B2383810122002331
:10C8D000C0E90423A16B0A4C0A6948695443094B17
:10C8E00003FB0040A2FB03230132034443F1000396
:10C8F000C1E9042323F0004010BD00BFDC0100109B
:10C900002DF451582D7F954C38B5064C0023054623
:10C9100008462360F5F776FB431C02D1236803B178
:10C920002B6038BD7C1C00100CB430B5164B0C1EAF
:10C930009DB01D6804DA8B232B604FF0FF301EE0A2
:10C940004FF40273ADF8143014BF04F1FF332346E3
:10C95000049307934FF6FF7302900690ADF81630DC
:10C96000284621AB02A9209A019300F0B1F9431C9B
:10C97000BCBF8B232B6014B1029B00221A701DB028
:10C98000BDE8304002B07047DC0100100EB400B5C5
:10C990004FF402719CB0ADF814106FF00041049197
:10C9A00007914FF6FF711DABADF81610084953F80B
:10C9B000042B02900690086802A9019300F088F900
:10C9C000029B00221A701CB05DF804EB03B07047A4
:10C9D000DC0100100EB430B59CB01FAC4FF40172F6
:10C9E00054F8045BADF814200290069000F073F840
:10C9F0000B4B03900B9300230F9314934FF6FF738D
:10CA0000ADF81630074B079002A918682A4623464E
:10CA1000019400F0A3FA1CB0BDE8304003B07047A9
:10CA20004BCA0000DC01001010B50C46B1F90E1025
:10CA300003F020F9002803DB636D0344636510BD38
:10CA4000A38923F48053A38110BD002070472DE9F2
:10CA5000F0411D468B890746DB050C46164605D579
:10CA6000B1F90E100022022302F0C0FCA38938465F
:10CA700023F48053A381B4F90E1032462B46BDE84F
:10CA8000F04101F0EBBC10B50C46B1F90E1002F00C
:10CA9000ADFC431CA38903D123F48053A38110BDB3
:10CAA00043F48053A381606510BDB1F90E1001F00D
:10CAB00015BE10F8012B11F8013B012A28BF9A423C
:10CAC000F7D0D01A7047034611F8012B03F8012B59
:10CAD000002AF9D17047034613F8012B002AFBD135
:10CAE000181A0138704770B58AB10B4605461C7894
:10CAF00010F8016B0131B44201D1012A03D1287829
:10CB00001B78C01A70BD013A002CEED1F7E7104631
:10CB100070BD000084463F482DE9F04FD0F80080FA
:10CB20000E46344614F8015B08EB0500407800F02F
:10CB3000080000F0FF0708B12646F2E72D2D03D1CB
:10CB4000B41C7578012703E02B2D04BF7578B41C45
:10CB500033F010000DD1302D08D1207800F0DF0027
:10CB6000582851D165781023023402E0002B08BF09
:10CB70000A23002F0CBF6FF0004A4FF0004ABAFBA7
:10CB8000F3F903FB19AA0026304608EB050B9BF8C6
:10CB900001B01BF0040F01D0303D0BE01BF0030B84
:10CBA0001BD0BBF1010F14BF4FF0570B4FF0370BE9
:10CBB000CBEB05059D4210DAB6F1FF3F0AD04845A0
:10CBC00006D801D1554503DC03FB0050012601E0E6
:10CBD0004FF0FF3614F8015BD7E7731C0CD1002F20
:10CBE0004FF022030CBF6FF000404FF00040CCF834
:10CBF00000302AB9BDE8F08F07B1404242B106B11A
:10CC0000611E1160BDE8F08F002B08BF0823B0E75C
:10CC1000BDE8F08FE00100102DE9F0478D688146F6
:10CC2000AB420C4692461F4643D38B8913F4906F58
:10CC30003DD0266809690222C1EB0608666906EB49
:10CC4000460696FBF2F608F101023A44964238BFD6
:10CC500016465B050FD53146FFF748FD054698B1EE
:10CC600021694246FFF7D2FCA38923F4906343F085
:10CC70008003A38113E0324602F0D5FF054670B968
:10CC800048462169FFF7EEFC0C23C9F80030A38960
:10CC90004FF0FF3043F04003A381BDE8F0872561EA
:10CCA00066614544C8EB06062560A6603D46AF4276
:10CCB00000D23D462A4620685146FFF7B0FCA368E3
:10CCC00000205B1BA36023681D442560BDE8F0873E
:10CCD0002DE9F0439DB003938B8907461C060D4652
:10CCE00016460CD50B6953B94021FFF7FFFC2860AD
:10CCF000286110B90C233B60C7E040236B6100231F
:10CD0000099320238DF8293030238DF82A303346BB
:10CD10001C4613F8012B1AB9B4EB06090FD002E038
:10CD2000252AF5D1F8E73846294632464B46FFF723
:10CD300073FF013000F0A480099B4B4409932378D2
:10CD4000002B00F09D8000234FF0FF3204930793E7
:10CD5000059206938DF853301A9304F101094D4E54
:10CD60004C46304621780522FFF742FC09F10109C3
:10CD7000049B28B1861B0120B04003430493EEE7D7
:10CD8000D90644BF20228DF853201A0744BF2B2216
:10CD90008DF8532022782A2A02D0079B21460EE0E4
:10CDA000039A111D12680391002A01DB079204E027
:10CDB000524243F002030792049301340AE00C4606
:10CDC00022780131303A092A03D80A2000FB0323D4
:10CDD000F5E7079323782E2B19D163782A2B09D1F5
:10CDE000039B02341A1D1B680392002BB8BF4FF03F
:10CDF000FF330BE0611C00230C4622780131303AEE
:10CE0000092A03D80A2000FB0323F5E70593224EE5
:10CE1000217830460322FFF7EBFB30B1861B402020
:10CE2000B040049B01340343049321781B4806223D
:10CE3000661C8DF82810FFF7DBFB88B1184B33B95F
:10CE4000039B073323F007030833039314E003AB7A
:10CE50000093384604A92A46124B00F0D5FB07E0A0
:10CE600003AB0093384604A92A460E4B00F04CFE53
:10CE7000B0F1FF3F804603D0099B4344099346E746
:10CE8000AB895B0601D4099801E04FF0FF301DB07B
:10CE9000BDE8F083342501003A2501003E2501005C
:10CEA00009D6000019CC000038B54B1C144602D13D
:10CEB0004FF0FF3038BD9389CDB223F0200393812A
:10CEC000536B526883B1A36B9A4207DA23685A1EE8
:10CED000226003F8015C636801331FE0214600F023
:10CEE0008BF90028F2D0E3E72169236851B18B4226
:10CEF00008D913F8010CA84204D1013B0132236088
:10CF0000626038BDE36304F1440363630323A363F6
:10CF10002346226403F8465F2360012363602846AA
:10CF200038BD10B50C46496B69B104F14403994210
:10CF300001D0FFF797FB236C00206063636013B19F
:10CF4000E36B236010BD23694FF0FF3023600023A3
:10CF50006360A38943F02003A38110BD2DE9F0474E
:10CF6000ADF5247D01930023469347939D4B0DF12E
:10CF70000C09A2939C4B07460C469046CDF8209195
:10CF8000A39398F80050002D00F0248197490B6876
:10CF90008A462B445A7802F0080202F0FF03EAB1F5
:10CFA0006368002B10DD2368DAF8002019780A4442
:10CFB000527815070ED5479A0133013247926268BD
:10CFC0002360013A6260EBE7A39B3846214698470D
:10CFD0000028E8D008F10106B046D2E7252D08F177
:10CFE00001064FD14593439398F801302A2B03D182
:10CFF0001023439308F1020631783546A1F130033E
:10D00000092B06F1010606D8459B0A2202FB0313F1
:10D01000303B4593F0E7DFF8DC8103224046FFF721
:10D02000E7FA40B1C8EB0008012000FA08F0439B82
:10D030003546034343936E1C2D78672D0FD8652D1D
:10D0400078D25B2D54D005D8002D00F0C580252D59
:10D0500018D071E0632D57D0642D3FD06CE0702D57
:10D0600032D007D86E2D55D03AD8692D64D100231F
:10D07000449339E0752D31D0782D29D0732D5BD1B3
:10D0800002233FE06368002B0DDD23681A78AA4273
:10D0900040F0A080013362682360479B013A01336E
:10D0A0006260479398E7A39B38462146984700283B
:10D0B000EBD04698002800F08F80A38913F0400F32
:10D0C00018BF4FF0FF3089E0439B43F020034393A8
:10D0D000439B43F400734393102302E00A2300E0D0
:10D0E00008236E2D449301DC03230BE0042309E0A5
:10D0F0003146484602F0F2FD439B064643F04003AA
:10D100004393012349931BE0439B43F04003439324
:10D110000023F7E7439AD0063FF55EAF12F0010F08
:10D12000019A479B02F104010191126814BF138018
:10D13000136051E70523E5E7032349930A2344934A
:10D140006368002B03DD439B590611D518E0A39BB0
:10D150003846214698470028F5D0AAE7479A013279
:10D1600047926268013A002A626013DD013323604E
:10D170002368DAF8002019780A4452781207EDD4AF
:10D18000499B022B0DDC384643A9224601AB00F037
:10D19000BBFF19E0A39B3846214698470028E7D0FB
:10D1A00087E7042B06DC384643A9224601AB01F091
:10D1B0000BF809E00E4B002B3FF40EAF384643A9A5
:10D1C000224601AB00F0B4FD012803D002287FF411
:10D1D00003AF6EE7469801E04FF0FF300DF5247D78
:10D1E000BDE8F087A9CE000023CF0000E0010010C9
:10D1F00031DD00003A2501002DE9F0410C46496B74
:10D2000004F1440399421AD14FF48061FFF76EFA9A
:10D2100018B94FF0FF30BDE8F0814FF48063A3638D
:10D2200094F84630606380F8FF3394F8453000F29C
:10D23000FD30437094F844300370206012E0A66B18
:10D2400077003A4602F0EFFC05460028E1D000EBFB
:10D250000608404629463246FFF7D8F9C4F8008050
:10D260006563A7630020BDE8F081936810B5013BBA
:10D27000002B936005DA9469A34208DBCBB20A2B3A
:10D2800005D01368581C10601970C8B210BDBDE8F5
:10D29000104001F08FB8F8B505460E461446D71871
:10D2A000BC4208D0284614F8011B3246FFF7DDFFC8
:10D2B000431CF5D100E00020F8BD00002DE9F0434B
:10D2C0009DB00D4617460393064618B183690BB906
:10D2D000FFF76EF8734B9D4201D1756808E0724B01
:10D2E0009D4201D1B56803E0704B9D4208BFF568CF
:10D2F000AB8918070AD52B6943B100230993202372
:10D300008DF8293030238DF82A3038E03046294610
:10D3100001F0B6F80028F0D04FF0FF30BEE0039ADD
:10D32000111D12680391002A70DB079201342378E3
:10D330002E2B7DD05E4F217838460322FFF758F917
:10D3400030B1C71B4020B840049B01340343049311
:10D35000217858480622671C8DF82810FFF748F9F5
:10D36000002800F08980544B002B7CD1039B0733AD
:10D3700023F0070308330393099B434409933B4677
:10D380001C4613F8012B1AB9B4EB07090ED002E0C2
:10D39000252AF5D1F8E7304629463A464B46FFF7AD
:10D3A0007AFF013075D0099B4B4409932378002BF9
:10D3B0006FD000234FF0FF3204930793059206933A
:10D3C0008DF853301A9304F101093C4F4C4638460E
:10D3D00021780522FFF70CF909F10109049B28B116
:10D3E000C71B0120B84003430493EEE7D90644BFAE
:10D3F00020228DF853201A0744BF2B228DF853208A
:10D4000022782A2A8BD0079B214605E0524243F01E
:10D4100002030792049389E70C4622780131303ADF
:10D42000092A03D80A2000FB0323F5E707937EE7C8
:10D4300063782A2B09D1039B02341A1D1B680392BF
:10D44000002BB8BF4FF0FF330BE0611C00230C46EC
:10D4500022780131303A092A03D80A2000FB03233D
:10D46000F5E7059366E703AB0093304604A92A4627
:10D47000134B00F0C9F807E003AB0093304604A952
:10D480002A460F4B00F040FBB0F1FF3F80467FF48F
:10D4900073AFAB895B063FF53FAF09981DB0BDE8A0
:10D4A000F08300BFCC240100EC2401000C25010016
:10D4B0003A2501003E25010009D60000342501006F
:10D4C00097D2000030B51346044A05460C46106852
:10D4D00029462246BDE83040FFF7F0BEDC010010CF
:10D4E0002DE9F047002B88B014461D46109E129976
:10D4F000139F05DA05F100431D4614462D2300E075
:10D5000000230B70149B23F0200ABAF1460F04D0BD
:10D51000BAF1450F03D1013601E0032300E00223F5
:10D520008DE8C80006AB039307AB049322462B4655
:10D5300001F076F9BAF1470F804602D1119BDB0763
:10D5400025D5BAF1460F08EB06090FD198F800303F
:10D55000302B09D1204629460022002304F002FA8C
:10D5600010B9C6F101063E603B6899442046294641
:10D570000022002304F0F6F908B1CDF81C90079BB7
:10D580004B4504D25A1C079230221A70F7E7079BCA
:10D590004046C8EB0302159B1A6008B0BDE8F0874F
:10D5A00073B50346002903F8022B03DA49421A46F1
:10D5B0002D2401E01A462B24092944701BDD0DF1AE
:10D5C00006040A2691FBF6F506FB1511092D01F15B
:10D5D0003001234604F801192946F2DC05F1300137
:10D5E00003F8011D0DF107018B420AD213F8011B4C
:10D5F00002F8011BF6E730241A46214402F8024BD8
:10D600005970101A02B070BD2DE9F04F8FB00C4662
:10D6100016461F46DDF86090054601F0E3FED0F89F
:10D6200000A05046FFF757FA00230C93D9F80030BA
:10D630000990073323F0070303F10802D3E900013F
:10D6400094F81880C9F80020C4E9120102F024FB04
:10D650000128D4E9120117D10022002304F08CF92B
:10D6600010B12D2384F84330904B914AB8F1470F05
:10D670008CBF9146994603232361236823F004035A
:10D6800023604FF0000B86E002F006FB236848B9E8
:10D69000884A8949B8F1470F8CBF894691460322D1
:10D6A0002261EBE7626828F0200B511C01D10622B1
:10D6B00004E0BBF1470F02D10AB901226260606841
:10D6C00043F480618DE80300D4E912230DF12B00AF
:10D6D00002900BA803900CA80590002021600690F2
:10D6E000CDF810802846FFF7FBFEBBF1470F8146BF
:10D6F0000B9909D1C81C02DB6368994230DDA8F19F
:10D7000002085FFA88F802E0B8F1650F12D8013913
:10D71000424604F150000B91FFF742FF0C9A8346FA
:10D720008318012A236102DC2268D2072DD5013338
:10D7300023612AE0B8F1660F14D10029636807DD80
:10D74000216113B92268D0071CD501330B4418E0BE
:10D7500013B92268D20701D5023312E0012310E089
:10D760004FF067080C9A914205DB23682161D807C6
:10D7700008D54B1C05E00029D4BFC1F102030123E9
:10D7800013442361A1654FF0000B9DF82B3013B1BA
:10D790002D2384F843300097284621460DAA3346AE
:10D7A00000F040F9013002D14FF0FF3036E123683C
:10D7B0005A0504D4284631464A46236908E1B8F19F
:10D7C000650F40F2CB80D4E912010022002304F05F
:10D7D000C9F800282AD028463146384A0123B847DC
:10D7E0000130E1D00C9B0B9A9A4207DB2368D807E3
:10D7F00004D423689B0700F1F880FDE028463146F9
:10D800005246099BB8470130CED04FF000080C9B20
:10D81000013B9845EDDA2846314604F11A0201230E
:10D82000B8470130C0D008F10108F0E70B9B002B8E
:10D8300028DC28463146214A0123B8470130B3D0BD
:10D840000B9B23B90C9B13B92368D907D1D5284664
:10D8500031465246099BB8470130A5D04FF0000829
:10D860000B9B28465B429845314608DA04F11A02C0
:10D870000123B847013097D008F10108F0E74A4684
:10D880000C9BA5E0A36D0C9A9A42B4BF93469B46AD
:10D89000BBF1000F02DC4FF000081CE028463146C7
:10D8A0004A465B46B8470130F5D17DE74525010082
:10D8B000492501004D250100512501009E2501004B
:10D8C0002846314604F11A020123B84701303FF4DB
:10D8D0006BAF08F10108A36D2BEAEB729A1A904521
:10D8E000EEDB09EB03080B9A0C9B9A420FDB2368D3
:10D8F000DA070CD40C9B0B9A9944C8EB09099B1AC4
:10D900009945A8BF9946B9F1000F08DC0FE02846F9
:10D9100031465246099BB8470130EBD144E72846CF
:10D92000314642464B46B84701303FF43DAF4FF0D9
:10D9300000080AE02846314604F11A020123B847DC
:10D9400001303FF431AF08F101080B9B0C9A29EA32
:10D95000E971D31A5B1A9845ECDB4AE70C9A012A65
:10D9600001DCDB0739D5284631464A460123B84752
:10D9700001303FF419AF284631465246099BB8475B
:10D9800001303FF411AFD4E912010022002303F06B
:10D99000E9FF10B14FF0000811E00C9B284631461A
:10D9A00009F10102013B1CE02846314604F11A024C
:10D9B0000123B84701303FF4F7AE08F101080C9B92
:10D9C000013B9845F0DB2846314604F150025B46A6
:10D9D000B84701307FF40DAFE6E6284631464A46A7
:10D9E0000123B8470130EED1DEE64FF00008E268CF
:10D9F0000D9BD31A984505DBE0680D9B9842B8BF94
:10DA000018460BE02846314604F119020123B847B5
:10DA100001303FF4C9AE08F10108E8E70FB0BDE8F6
:10DA2000F08F00BF2DE9F84315461F468A680B6941
:10DA300006469A42A8BF13462B6091F843200C4635
:10DA4000DDF820800AB101332B602368990602D5E6
:10DA50002B6802332B60236813F006091DD094F85D
:10DA600043302268003318BF012392061FD5E11806
:10DA7000302081F843005A1C94F8451022440233A8
:10DA800082F8431013E03046394604F119020123AD
:10DA9000C047013007D009F10109E2682B68D31AA9
:10DAA0009945F0DBDBE74FF0FF30BDE8F883304607
:10DAB000394604F14302C0470130F4D023682A6894
:10DAC00003F00603E168042B08BFC2EB01052369DC
:10DAD000A2680CBF25EAE57500259A42C4BFC3EBD6
:10DAE0000203ED184FF00009A9450ADA304639461D
:10DAF00004F11A020123C0470130D4D009F1010911
:10DB0000F2E70020BDE8F8832DE9FF470E7E80464E
:10DB10006E2E0C4691469A460C9D01F1430000F092
:10DB2000A58011D8632E22D009D8002E00F0AF8036
:10DB3000582E40F0BF8081F845607B4A4FE0642E4C
:10DB40001ED0692E1CD0B5E0732E00F0A48009D839
:10DB50006F2E2BD0702E40F0AD800B6843F0200369
:10DB60000B6038E0752E21D0782E34D0A2E02B68DF
:10DB700001F142071A1D1B682A6081F842309DE0BE
:10DB800022682B6812F0800F03D01A1D2A601D68CE
:10DB900005E05106F9D51A1D2A60B3F90050002D91
:10DBA00039DA2D236D4284F8433034E022682B6843
:10DBB00012F0800F03D01A1D2A601D6804E052067F
:10DBC000F9D51A1D2A601D88237E574A6F2B14BF72
:10DBD0000A2308231BE07823544A84F8453023683D
:10DBE000296813F0800F01F104062E6001D00D6842
:10DBF00002E05F06FBD50D88DE0744BF43F020033B
:10DC000023601DB9236823F0200323601023002123
:10DC100084F8431001E0444A0A236668002EA66097
:10DC200003DB216821F00401216005B96EB104F124
:10DC30004201B5FBF3F603FB1655555D0F4601F89F
:10DC400001593546002EF4D100E00746082B0AD1D1
:10DC50002368DD0707D5626823699A4203DC302315
:10DC600007F8013C013FC01B20612CE009682B68CC
:10DC700011F0800F626904D0191D29601B681A60B9
:10DC800005E04906F8D5191D29601B681A80002394
:10DC90002361074617E02B681A1D2A601F68384663
:10DCA000FEF719FF63682061984288BF23612369EA
:10DCB000636005E004F1420784F8426001232361B8
:10DCC000002384F84330CDF800A04046214603AA43
:10DCD0004B46FFF7A7FE013002D14FF0FF301FE0A7
:10DCE000404649463A462369D0470130F5D023687B
:10DCF0009B0705D4E068039B9842B8BF18460FE025
:10DD00000025E268039BD31A9D42F3DA4046494658
:10DD100004F119020123D0470130DED00135F0E7CC
:10DD200004B0BDE8F08700BF55250100662501005D
:10DD30002DE9F04F16468A6887B00293531EB3F55B
:10DD4000AE7F07460C4606D96FF4AE731A4440F214
:10DD50005D138B6000E000222368A04643F4F0636B
:10DD60004FF0000B48F81C3B4546DA46CDF814B09E
:10DD7000CDF810B0D946CDF80CB0A168002900F05C
:10DD8000E98033681B78492B75D016D8392B0DD80C
:10DD9000312B3ED22D2B45D002D82B2B42D0D9E0AF
:10DDA0002E2B00F09780302B23D0D3E0452B00F0B2
:10DDB0009A80462B7CD0412B0CE0652B00F09380A1
:10DDC0000AD8542B7AD002D84E2B33D0C2E0592B2C
:10DDD0007AD0612B49D0BDE06E2B2BD004D8662BB6
:10DDE00066D0692B47D0B5E0742B67D0792B6BD008
:10DDF000B0E0206810F4807F0BD020F0800020601D
:10DE000009F10109002A00F08C800131013AA1607A
:10DE100087E00AEB0B01002940F09C80216821F487
:10DE2000C07105E02168080640F1948021F080016E
:10DE3000216074E0BAF1000F0ED1B9F1000F0ED1DC
:10DE4000216801F4E060B0F5E06F08D121F4F061E1
:10DE500021604FF0010A62E0BAF1020F5DD0BBF120
:10DE6000010F20D0BBF1040F1CE0BAF1010F71D1FA
:10DE70004FF0020A53E0BBF1000F0ED1B9F1000FD1
:10DE80006BD1216801F4E060B0F5E06F69D121F455
:10DE9000F06121604FF0010B41E0BBF1030F02D0B4
:10DEA000BBF1050F56D10BF1010B5FFA8BFB36E08E
:10DEB000BBF1020F4ED14FF0030B30E0BBF1060F68
:10DEC00048D14FF0070B2AE0BBF1070F42D14FF0CA
:10DED000080B24E0216888053CD521F420712160DD
:10DEE000CDF80C901BE0216801F4A060B0F5806FC4
:10DEF00004D048052ED5B9F1000F32D0880504D4DE
:10DF000003980595C0EB0900049021F4F06141F4F9
:10DF1000C07121604FF0000901E04FF0030A2B703F
:10DF20000135A368013BA360236901332361736852
:10DF3000013B002B736003DD3368013333601CE762
:10DF40000192D4F88031384631469847019A00282A
:10DF50003FF413AFB9F1000F03D0236823F48073AB
:10DF600023600AF1FF3ABAF1010F10D845452A465D
:10DF70000BD9D4F87C3112F8011C38463246984748
:10DF80002369013D013B2361F0E70126B5E00BF178
:10DF9000FF33062B2CD8BBF1020F1AD9ABF1030BC0
:10DFA0005FFA8BFBAA46CBEB050CE2450ED0D4F80A
:10DFB0007C311AF8011D3846CDF804C03246984726
:10DFC0002369DDF804C0013B2361EEE7CBEB0505D7
:10DFD0000EE045452A46D8D9D4F87C3112F8011C08
:10DFE0003846324698472369013D013B2361F0E7FB
:10DFF0002368DA052ED55B050ED545452A46C4D9DA
:10E00000D4F87C3112F8011C38463246984723690F
:10E01000013D013B2361F0E715F8011C23696529E7
:10E0200003F1FF3305F1FF3A23610DD045290BD0F1
:10E03000D4F87C31384632469847236915F8021CDB
:10E04000013BA5F1020A2361D4F87C3138463246FF
:10E0500098475546266816F010064DD12E70236855
:10E0600003F4C063B3F5806F05D10399C1EB0903D5
:10E070005A4263B915E0049D9DB1059D3246691C65
:10E0800038460A23FEF746FD049D421B059D04F217
:10E090006F139D4228BF04F5B77528461949FEF74E
:10E0A00075FC41460022384601F082FE2268029D3E
:10E0B00012F0020F804689462B6802D01A1D2A6092
:10E0C00006E0029D12F0040F03F104022A6003D05F
:10E0D0001B68C3E900890BE01D6801F0DDFD10B984
:10E0E00001F02EFE03E04046494603F0B5FC2860EF
:10E0F000E3680133E36000E00026304607B0BDE886
:10E10000F08F00BF772501002DE9F04115468A68A0
:10E1100080460C4632B98A69002A14BF4FF0FF329C
:10E1200001228A602268D10603D41A68111D196081
:10E1300017680026A069E0B923680136DA0604D41E
:10E140002B6801371B7807F8013C2A686B6801329D
:10E150002A60A268013B013A6B60A26012B3002BF7
:10E16000E8DCD4F880314046294698470028E1D0C1
:10E1700018E0012807D12A6811786269525C002AE8
:10E18000DAD1EEB10EE0022801D04EB10AE02A68E1
:10E190000C49127809680A4452781307CCD5F4E781
:10E1A00001280DD0236813F0100305D1E268013275
:10E1B000E260A26902B13B70236900201E4426611F
:10E1C000BDE8F081E00100102DE9F04F89B00C4668
:10E1D000984605A9734B02918146164693E80700BD
:10E1E000029B83E80700A3696F4A7049032B08BFAD
:10E1F0001146A36803915A1EB2F5AE7F07D96FF49A
:10E20000AE7503EB050A40F25D13A36001E04FF029
:10E21000000A236804F11C0743F450632360BB46E3
:10E220000023326805A951F82300117802220193D6
:10E23000FEF7DEF9019B002835D0012B0BD1626877
:10E240002AB908226260226842F4007222602268C1
:10E2500022F4A0620BE0022B0AD1226802F4C06112
:10E26000B1F5007F1FD11021616042F480722260FD
:10E27000A268511EA160B2B132680BF10105511CB8
:10E28000316012788BF800207268013A002A7260BF
:10E2900008DC0193D4F88021484631469047019B21
:10E2A000002841D1AB460133032BBAD163680BB9C7
:10E2B0000A23636063683E496069C91A01F00EFD74
:10E2C0005D464FF0000BA368002B2FD032686069C9
:10E2D0001178405C50B3302921680BD1080509D56D
:10E2E0000BF1010BBAF1000F0BD001330AF1FF3A29
:10E2F000A36006E021F4106121601378013505F870
:10E30000013C7368013B002B736003DD336801330C
:10E31000336005E0D4F8803148463146984728B943
:10E32000A368013BA360CEE74FF0000B2368D9053B
:10E330000DD5BD4209D915F8011CD4F87C314846E9
:10E340003246984705F1FF3A5546BD4226D022682D
:10E3500012F010021BD12A70636848463946039EAA
:10E36000B0472268D8F8003012F0200F07D1D2074A
:10E3700005D51A1DC8F800201B68188004E01A1D76
:10E38000C8F800201B681860E3680133E360236964
:10E39000ED1BAB445B442361002000E0012009B089
:10E3A000BDE8F08F7C25010015CB0000E9090100D4
:10E3B0009825010070B50E461446054618B18369CC
:10E3C0000BB9FDF7F5FF224B9C4201D16C6808E0C8
:10E3D000204B9C4201D1AC6803E01F4B9C4208BF1C
:10E3E000EC68A369A360A3891A0709D523693BB127
:10E3F00023692068F6B2C01A636998420FDB08E00F
:10E400002846214600F03CF80028F1D04FF0FF30BC
:10E4100070BD28462146FDF73BFF0028F6D1A368D2
:10E420000130013BA36023685A1C22601E7063699F
:10E43000984204D0A389DB0707D50A2E05D12846C8
:10E440002146FDF725FF0028E0D1304670BD00BF12
:10E45000CC240100EC2401000C25010038B5074C48
:10E46000054600202060084611461A46F3F748FD8D
:10E47000431C02D1236803B12B6038BD7C1C001003
:10E48000324B70B51D6806460C4625B1AB6913B911
:10E490002846FDF78DFF2E4B9C4201D16C6808E0A9
:10E4A0002C4B9C4201D1AC6803E02B4B9C4208BF33
:10E4B000EC68A28993B2190720D4DD0605D409239C
:10E4C00042F040023360A2813BE0580712D5616BF5
:10E4D00041B104F14403994202D03046FEF7C2F83C
:10E4E00000236363A38923F02403A38100236360D3
:10E4F00023692360A38943F00803A38123694BB9EF
:10E50000A38903F42073B3F5007F03D0304621467E
:10E51000FEF712F8A38913F0010205D00022A260D1
:10E5200062695242A26103E0990758BF6269A26022
:10E5300022694AB903F0800080B230B143F0400351
:10E54000A3814FF0FF3070BD002070BDDC010010D2
:10E55000CC240100EC2401000C2501002DE9F84336
:10E56000294D06462C680F46914698460CB9274C13
:10E570002C6063681F2B12DD254B1BB94FF0FF3059
:10E58000BDE8F8838C20FEF723F804460028F5D078
:10E590002A680023026043602860C0F888304EB3C8
:10E5A000D4F8880078B91A4B002BE7D04FF4847068
:10E5B000FEF70EF80028E1D00023C0F80031C0F8C3
:10E5C0000431C4F888006568012340F8259000EB09
:10E5D000850203FA05F5D0F80031022E43EA05035F
:10E5E000C0F80031C2F8808004D1D0F804311D4356
:10E5F000C0F80451636800205A1C0233626044F87A
:10E600002370BDE8F88300BF781C0010EC1B0010DD
:10E61000D1C500002DE9F74F824689462D4F3C6851
:10E62000002C54D06268D4F8885002F10208561EBB
:10E6300005EB820B04EB8808002E36DBB9F1000FE6
:10E6400004D065B3DBF87C204A4528D1616858F8CE
:10E65000042C01398E4216BF0021666048F8041C64
:10E66000EAB1636801932DB10121B140D5F80001F1
:10E67000014201D190470BE0D5F80401014204D1D9
:10E6800050465BF8041C904702E05BF8040C90478E
:10E690006268019B9342C1D13A68A242BED1013E59
:10E6A000ABF1040BA8F10408C6E70B4B7BB1626821
:10E6B00023684AB943B13B6015B12846FDF790FF86
:10E6C0002046FDF78DFFAAE727461C46A8E703B0C2
:10E6D000BDE8F08F781C0010E1C5000038B5064C8D
:10E6E0000023054608462360F3F7F2FB431C02D1E2
:10E6F000236803B12B6038BD7C1C00102DE9F74F57
:10E7000003690C698046A342C0F28380013CA200E9
:10E7100001F1140700F114059146009257F82460A6
:10E720002A44019255F824200136B2FBF6F6B9448A
:10E73000002E3BD04FF0000E3A462846F34652F8E2
:10E7400004CB03681FFA8CFA4FEA1C4C0AFB06EA5A
:10E750000CFB06FC0CEB1A4C1FFA8AFACAEB0B0BEB
:10E760004FEA1C4E1FFA83FA1FFA8CFCDA44CCEBFA
:10E77000134C0CEB2A4C1FFA8AFA4AEA0C4A4A4517
:10E780004FEA2C4B40F804ABD9D9009AAB586BB97F
:10E79000019A131FAB421A4602D8C8F8104005E090
:10E7A0001268043B002AF8D1013CF3E7404601F02F
:10E7B00086F800282BDB01362B46002057F804CBC7
:10E7C0001A681FFA8CF1411A1FFA82FA4FEA1C4CA0
:10E7D0005144CCEB124202EB214289B210144F4556
:10E7E00041EA024243F8042BE8D955F8242005EB0E
:10E7F000840362B9043BAB421A4602D8C8F8104001
:10E8000005E01268043B002AF8D1013CF3E73046EA
:10E8100000E0002003B0BDE8F08F00000000000021
:10E820002DE9F04F456A9BB08246279CCDE9042331
:10E8300045B91020FDF7CCFECAF82400456085607C
:10E840000560C560DAF82430196861B15B6801229F
:10E850004B6002FA03F350468B6000F00EFEDAF8CC
:10E86000243000221A600598002805DA012320F0E0
:10E8700000412360059101E000232360059F9C4A2D
:10E8800027F000431B0D1B0593421DD1269A42F22F
:10E890000F731360049B43B9964B974AC7F3130059
:10E8A00000280CBF1046184600E09248289F002F11
:10E8B00000F07185C37813B100F1080300E0C31CB8
:10E8C000289F3B6000F067BDDDE90445002220463B
:10E8D0002946002303F046F8804658B1269F0123BD
:10E8E0003B60289F002F00F0538584483860013832
:10E8F00000F051BD19AB009318AB0193504622466E
:10E900002B4601F0CEF8C7F30A5683465EB1C5F335
:10E91000130343F07F51204641F44011A6F2FF3625
:10E92000CDF854801CE0199B189E1E446FF482633E
:10E930009E4209DB04991F3306F212409B1B21FA09
:10E9400000F09F40384304E06D48049A801B02FAAF
:10E9500000F002F029FD0127A1F1F871013E1597A1
:10E960000022684B02F0E2FB5BA3D3E9002302F034
:10E9700091FD5BA3D3E9002302F0DAFB04463046A5
:10E980000D4602F021FD58A3D3E9002302F082FDD9
:10E9900002460B462046294602F0CAFB04460D46B5
:10E9A00003F012F82946814600222046002302F097
:10E9B000E3FF58B1484602F007FD02460B462046E9
:10E9C000294602F0CFFF08B909F1FF39B9F1160F56
:10E9D0000DD84D4B03EBC903D3E90001DDE9042356
:10E9E00002F0E8FF30B109F1FF39002700E001270C
:10E9F000149700E01490189B9E1B013E099604D5C5
:10EA0000774208970027099701E000270897B9F196
:10EA1000000F07DB099FCDF844904F44099700276A
:10EA20000E9708E0089FC9EB07070897C9F1000790
:10EA30000E9700271197249F092F29D8052FC4BFAF
:10EA4000043F2497249FC8BF0025A7F10203D8BF25
:10EA50000125032B21D8DFE803F0060F020401276C
:10EA600002E0012709E000270F97259F002F1EDDF8
:10EA70000B9707973B461FE000270F97259F4F44B2
:10EA80000B9701373B460797012BB8BF012313E0D3
:10EA90000125002724970F9501E001270F974FF0DC
:10EAA000FF370B97079700271223259704E00127CC
:10EAB0000B9707973B462597DAF8244000226260BF
:10EAC000042101F114029A4220D8626849000132FF
:10EAD0006260F6E7AFF3008061436F63A787D23FC0
:10EAE000B3C8608B288AC63FFB799F501344D33F3D
:10EAF0000000F07FAD260100A42601009F25010043
:10EB0000EEFBFFFF0000F83FB826010050466168A9
:10EB100000F07EFCDAF824302060079F1B680E2F7F
:10EB20000A9300F26B81002D00F06881B9F1000FAB
:10EB3000DDE90401CDE9120131DD814A09F00F035D
:10EB400002EBC3034FEA2914D3E90001CDE90C011C
:10EB5000E0060CD5DDE912017A4B04F00F04D3E98D
:10EB6000082302F0C1FD0327CDE9040100E00227DC
:10EB7000744D6CB1E10708D5DDE90C01D5E900233E
:10EB800002F088FCCDE90C01013764100835F0E78C
:10EB9000DDE90401DDE90C2302F0A6FD1BE0C9F16B
:10EBA0000004DCB1664B04F00F0203EBC203DDE9A5
:10EBB0001201D3E9002302F06DFC624D24110227FB
:10EBC0004CB1E20704D5D5E90023013702F062FC1D
:10EBD00064100835F4E7CDE9040100E00227149938
:10EBE000E9B1DDE90445002220462946564B02F0F2
:10EBF000C3FEC8B1079AE2B10B9B002B40F3FA8029
:10EC000009F1FF3010902946204600224F4B02F0B8
:10EC100041FCCDE904010B9901370C910DE0079AF5
:10EC2000CDF840900C9208E0079BCDF840900C93F3
:10EC300003E00798CDF840900C90384602F0C4FBF2
:10EC4000DDE9042302F026FC0022414B02F070FAB9
:10EC50000C9F0446A1F15075CFB900223D4BDDE970
:10EC6000040102F063FA22462B4606460F4602F0E4
:10EC7000A1FE002840F05382224605F100433046B1
:10EC8000394602F079FE002840F03F82B2E00C9F46
:10EC90002B4B7A1E0F9F03EBC203002F5ED0D3E9EC
:10ECA000002300202C4902F01FFD22462B4602F0D3
:10ECB0003DFADDE90467DDF8288004460D46394653
:10ECC000304602F081FE029002F07EFB02460B46C7
:10ECD0003046394602F02AFADDF808C022460CF127
:10ECE000300308F8013B2B4606460F4602F044FE6F
:10ECF000002840F03B8332463B460020124902F098
:10ED000015FA22462B4602F037FE002840F0D58047
:10ED10000A980C99C0EB08038B426BDA204629460F
:10ED200000220A4B02F0B6FB002204460D46304694
:10ED30003946064B02F0AEFB06460F46BFE700BF62
:10ED4000B8260100802701000000F03F00002440A9
:10ED500000001C40000014400000E03F2246D3E9C0
:10ED600000012B4602F096FBDDE90467DDF8288000
:10ED70000C9ACDE916010A9C90443946304602F0BF
:10ED800023FE054602F020FB02460B46304639467C
:10ED900002F0CCF9303504F8015B444506460F46D5
:10EDA00021D10022874BDDE9160102F0C1F90246AC
:10EDB0000B463046394602F0FDFD00287DD1DDE9E5
:10EDC000162300207F4902F0B1F902460B46304677
:10EDD000394602F0D1FD68B1A04618F8013C013C6B
:10EDE000302BF9D0C2E20022774B02F053FB0646EB
:10EDF0000F46C2E7DDE91201CDE90401199B002BA2
:10EE00007CDBB9F10E0F79DC704B259F03EBC90356
:10EE1000002FD3E9004514DA079F002F11DC40F0E2
:10EE20007681204629460022694B02F033FBDDE95A
:10EE3000042302F0B5FD079D2C46002840F06981AF
:10EE400071E1DDF82880DDE9046722462B46304673
:10EE5000394602F049FC02F0B7FD049002F0B4FA22
:10EE600022462B4602F016FB02460B463046394638
:10EE700002F05CF9049F024607F130060A9F08F889
:10EE8000016BC7EB0806079F0B46BE4229D102F073
:10EE90004FF922462B4606460F4602F08BFD70B90D
:10EEA0003046394622462B4602F05CFD002800F031
:10EEB0005F82049FFB0702D45AE2DDF8409043468C
:10EEC000984618F8012C013B392A06D10A9F9F4227
:10EED000F6D1302209F101093A701A7801321A701C
:10EEE00046E20022384B02F0D5FA00220023064603
:10EEF0000F4602F037FD0028A7D039E20F9F002F00
:10EF000030D0249F012F0ADC159F17B103F2334341
:10EF100002E0189BC3F136030E9D089E16E0079F82
:10EF20007D1E0E9FAF4201DB7D1B06E00E9F0E95FE
:10EF3000EB1B119F00251F441197079F002F03DA39
:10EF400008980023C61B01E0089E079B089F5046B7
:10EF50001F440897099F01211F44099700F06DFB8A
:10EF6000044602E00E9D089E0F9C6EB1099F002F83
:10EF70000ADD3B46089FB342A8BF3346FF1A0897F5
:10EF8000099FF61AFF1A09970E9F002F28DD0F9F81
:10EF900007B3002D10DD21462A46504600F0EEFB57
:10EFA00004465A462146504600F050FB5946074653
:10EFB000504600F062FABB460E9F7A1B10D05046B6
:10EFC00059460AE00000E03F00002440B826010056
:10EFD000000014400E9A5046594600F0CFFB83467D
:10EFE0005046012100F029FB119F0546002F05DD49
:10EFF000294650463A4600F0C1FB0546249F012FA2
:10F0000012DC049880B90599C1F3130373B921F098
:10F0100000473F0D3F0557B1089F01370897099FEB
:10F0200001370997012702E0002700E0049F1198AB
:10F0300040B12B6905EB8303186900F0B1FAC0F108
:10F04000200000E00120099B034413F01F030FD0B0
:10F05000C3F12002042A09DD0899099AC3F11C03AF
:10F0600019441A4408911E44099209E008D0134635
:10F07000089809991C331844194408901E440991B2
:10F08000089A002A04DD5946504600F0C5FB834625
:10F09000099B002B05DD294650461A4600F0BCFBB3
:10F0A00005461498E0B15846294600F008FC0028AF
:10F0B00016DA594650460A22002300F0F5F90F9956
:10F0C00009F1FF39834649B121460A2250460023FF
:10F0D00000F0EAF90B9A0446079201E00B9B0793B4
:10F0E0000798002829DC2499022926DD88B92946B9
:10F0F0000522079B504600F0D7F905462946584699
:10F1000000F0DDFB00280EDC03E00C9D00E0002594
:10F110002C46259FDDF828806FEA07090AE00C9D40
:10F12000DDF840902C460A9F312307F101083B701F
:10F1300009F101092746002407E10F98002800F093
:10F14000BB80002E05DD21465046324600F064FBB0
:10F1500004469FB16168504600F05AF9226906469C
:10F16000023204F10C0192000C30FDF74FFA5046C8
:10F170003146012200F050FB074600E027460A9E78
:10F1800029465846FFF7BAFA214600F1300C80466E
:10F190005846CDF808C000F092FB3A460890294640
:10F1A000504600F0A9FBC3680246DDF808C04BB921
:10F1B00011465846039200F082FB039A0346DDF89D
:10F1C00008C000E00123504611460393CDF808C063
:10F1D00000F053F9039BDDF808C063B9249951B9D5
:10F1E000049800F0010232B9BCF1390F35D0089B08
:10F1F000002B24DC25E00898002802DA002B08DC2C
:10F200001FE023D1249909BB049800F00102EAB958
:10F21000F4E7594601225046CDF808C000F0FCFA48
:10F220002946834600F04BFB0028DDF808C003DCCC
:10F2300007D11CF0010F04D0BCF1390F0DD008F13B
:10F24000310C06F1010886F800C07EE0002B06F1C3
:10F25000010809DDBCF1390F03D1392333700136C0
:10F260005BE00CF1010368E00A99079AC1EB08031F
:10F270004646934206F801CC3CD059460A22002368
:10F28000504600F011F9BC428346214650464FF0EB
:10F290000A024FF0000304D100F006F904460746C5
:10F2A0006EE700F001F9394604460A225046002371
:10F2B00000F0FAF8074663E70F9E58462946FFF725
:10F2C0001DFA0A9F00F1300C07F806C0079F0136AF
:10F2D000BE4207DB0A9E012FACBFF6190136274656
:10F2E000002407E0594650460A22002300F0DCF8CB
:10F2F0008346E2E7594601225046CDF808C000F0A7
:10F300008BFA2946834600F0DAFA0028DDF808C0B7
:10F3100003DC14D11CF0010F11D016F8013CB046EB
:10F32000392B06F1FF3607D10A98B042F5D13123C7
:10F3300009F10109037008E00133337005E0B046BC
:10F3400018F8013C013E302BF9D05046294600F018
:10F3500094F86FB12CB1BC4203D05046214600F066
:10F360008CF85046394600F088F801E0DDF840900E
:10F370005046594600F081F80023269F88F8003057
:10F3800009F101033B60289F27B1C7F8008001E025
:10F39000024800E00A981BB0BDE8F08F9E250100EE
:10F3A00038B5074C00230546084611462360F2F79E
:10F3B00019FE431C02D1236803B12B6038BD00BF86
:10F3C0007C1C001038B5064C002305460846236017
:10F3D000F2F7E0FD431C02D1236803B12B6038BD76
:10F3E0007C1C001000487047E401001038B5074C41
:10F3F000054600202060084611461A46F2F7DEFD59
:10F40000431C02D1236803B12B6038BD7C1C001063
:10F4100070B5456A04460E463DB91020FDF7D8F890
:10F420006062456085600560C560656AEB6843B1F0
:10F43000636ADA6852F8260078B1016842F826104B
:10F4400017E020460421212200F0DFFB636AE86018
:10F45000DB68002BECD1002070BD012101FA06F51C
:10F460006A1D2046920000F0D0FB0028F3D04660D1
:10F47000856000220261C26070BD70B5446A0646B4
:10F480000D463CB91020FDF7A3F87062446084601B
:10F490000460C4603DB1736A6A68DB6853F8221087
:10F4A000296043F8225070BD2DE9F0410C461E46FC
:10F4B0000D69074614310023086801331FFA80FCE8
:10F4C000000C02FB0C6C504300EB1C401FFA8CFC40
:10F4D000060CAB420CEB004041F8040BECDBD6B160
:10F4E000A3689D4212DB616838460131FFF790FF47
:10F4F000226904F10C010232804692000C30FDF7C3
:10F5000085F821463846FFF7B8FF444604EB8503EB
:10F5100001355E6125612046BDE8F0812DE9F843A3
:10F520001446984603F1080209230D4692FBF3F2B4
:10F530000646012300219A4202DD5B000131FAE711
:10F540003046FFF765FF089B092C43614FF001032C
:10F550000146036111DD05F109094F46254417F8FD
:10F56000013B30460A22303BFFF79EFFAF42014687
:10F57000F5D109EB0407083F02E005F10A07092469
:10F580002546454509DA3B1B5B5D30460A22303B88
:10F59000FFF78AFF01350146F3E70846BDE8F88327
:10F5A000030C1B0413B90004102300E0002310F027
:10F5B0007F4F04BF0002083310F0704F04BF0001FA
:10F5C000043310F0404F04BF80000233002803DBF7
:10F5D000420003D5581C70471846704720207047DA
:10F5E000036813F007020BD0D90722D49A0703D57A
:10F5F0005B080360012070479B080360022070478E
:10F6000099B209B91B0C102213F0FF0F04BF1B0A9B
:10F610000832190704BF1B090432990704BF9B086D
:10F620000232D90702D45B0805D0013203601046CC
:10F630007047002070472020704710B50C4601210C
:10F64000FFF7E6FE01224461026110BD2DE9F04F93
:10F65000164633690A6985B09A420D4601DA354685
:10F660000E46D5F810803769AB68696808EB070467
:10F670009C42C8BF0131FFF7CBFE00F1140303EB3E
:10F68000840101911A46DDF804A0524503D20021FD
:10F6900042F8041BF7E705F1140106F1140201EB2F
:10F6A000880802EB8707CDF808800397039E15466C
:10F6B000B24256D2B5F800C00432BCF1000F25D0DA
:10F6C0000F461D46002657F8049BD5F800801FFA08
:10F6D00089FB1FFA88FA0CFB0BAA4FEA19494FEA7B
:10F6E00018480CFB0988B24408EB1A481FFA8AFA3A
:10F6F0004AEA084A4FEA1846DDF80880AB46B845A2
:10F700004BF804AB01D95D46DDE76E6032F8028C40
:10F71000B8F1000F23D01E680F461D464FF00009B8
:10F72000B7F800A0B5F802C0B6B208FB0ACCE144B5
:10F7300046EA0946AC464CF8046B57F8046BB5F83A
:10F7400004A0360C08FB06A6DDF808A006EB194657
:10F7500057454FEA164901D26546E1E76E6004332A
:10F76000A4E7019B002C03DC046105B0BDE8F08F29
:10F7700053F8042D002AF7D1013CF3E712F00303FC
:10F780002DE9F04105460E46174607D0214A013BB8
:10F7900052F823200023FFF787FE0646BF1035D01E
:10F7A0006C6A3CB91020FCF713FF68624460846007
:10F7B0000460C460D5F82480D8F808407CB9284695
:10F7C00040F27121FFF739FF0023C8F80800044612
:10F7D000036004E07F1019D0206870B10446FB0775
:10F7E000F8D5314622462846FFF730FF314680469D
:10F7F0002846FFF742FE4646ECE7284621462246C9
:10F80000FFF724FF002320600360E7E73046BDE8F0
:10F81000F08100BFA82701002DE9F0470C462369BD
:10F820004FEA621A0AEB03094968A3688046154645
:10F8300009F101079F4202DD01315B00FAE7404612
:10F84000FFF7E6FD0023064600F11402534504DAF3
:10F85000002142F823100133F8E720692AEAEA710F
:10F8600004F1140315F01F0C02EB810103EB800E71
:10F8700016D0CCF1200A002518680A4600FA0CF0D0
:10F88000054342F8045B53F8045B734525FA0AF517
:10F8900001D21146F0E74D6045B109F1020705E0DC
:10F8A00053F8042B734541F8042BF9D3013F40462C
:10F8B00037612146FFF7E1FD3046BDE8F087026978
:10F8C0000B6910B5D21A13D19C00143001F1140247
:10F8D0000319224453F8044D52F8041D8C4203D0FE
:10F8E00008D24FF0FF3010BD9842F3D3002010BD76
:10F8F000104610BD012010BD2DE9F04706460C460C
:10F90000084611461546FFF7DAFF071E08D13046B4
:10F910003946FFF77DFD012303614761BDE8F087AC
:10F9200001DB002703E0234601272C461D466168C2
:10F930003046FFF76DFD22692B69143405F114067A
:10F9400006EB830AC76004EB820C00F1140300216C
:10F9500054F8047B56F8049B1FFA87F81FFA89F5C0
:10F9600041444FEA1949C5EB0108C9EB174707EBBA
:10F9700028471FFA88F83914B24548EA0747254650
:10F9800043F8047BE4D865450DD255F8044BA6B284
:10F990000E44240C04EB2644B6B2211446EA044477
:10F9A00043F8044BEFE753F8041D09B9013AFAE7AD
:10F9B0000261BDE8F08700000F4B0B40A3F15073CC
:10F9C000002B01DD194609E05B421B15132B4FF09C
:10F9D000000105DC4FF4002242FA03F100207047D9
:10F9E000322B4FF00102DABFC3F1330302FA03F303
:10F9F00013461846704700BF0000F07F2DE9F04124
:10FA0000066900F1140707EB860656F8044C884691
:10FA10002046FFF7C5FDC0F120030A28A6F1040522
:10FA2000C8F8003014DCBD42C0F10B0188BF56F8A5
:10FA3000085C24FA01FC98BF0025153025FA01F175
:10FA400084404CF07F5343F4401341EA040224E025
:10FA5000BD4286BFA6F1080556F8081C0021B0F18A
:10FA60000B0615D0B440C0F12B0021FA00FC44F085
:10FA70007F5444F44014BD4244EA0C038CBF55F853
:10FA8000044C002424FA00F0B14040EA010204E0F2
:10FA900044F07F5343F440130A4610461946BDE82C
:10FAA000F0812DE9F74301211D46DDF82890DDF8AE
:10FAB0002C801446FFF7ACFCC5F30A570646C5F385
:10FAC00013030FB143F480130193D4B102A840F89B
:10FAD000084D6846FFF784FD009B48B1019AC0F1CC
:10FAE000200102FA01F1C2400B437361019200E070
:10FAF0007361019B002B0CBF01240224B3613461AC
:10FB000007E001A8FFF76CFD019B012473613461DC
:10FB100020303FB1A7F233470744C9F80070C0F165
:10FB200035000AE0A0F2324006EB8403C9F8000079
:10FB30001869FFF735FDC0EB4410C8F800003046E7
:10FB400003B0BDE8F0832DE9F3410E4669468046D7
:10FB5000FFF754FF0D46044601A93046FFF74EFF5C
:10FB6000009F0B46019902467F1AD8F810003169B0
:10FB7000411A07EB41110029CCBF05EB0155A3EB5E
:10FB800001532046294601F0AFFD02B0BDE8F081E7
:10FB900010B5013902F1140349111269013100EB6A
:10FBA000810103EB8202934204D253F8044B40F8E4
:10FBB000044BF8E7884203D2002340F8043BF9E7FE
:10FBC00010BD00F1140200694B11834210B50CDC2A
:10FBD0000CDA11F01F0109D052F8230020FA01F4C9
:10FBE00004FA01F181420ED100E0034602EB8303E7
:10FBF0009342194605D951F8041C043B0029F7D05B
:10FC000001E0002010BD012010BD38B502FB01F459
:10FC10002146FCF76BFD054618B100212246FCF792
:10FC200019FD284638BDF8B5064614460D4621B9DB
:10FC30001146BDE8F840FCF759BD1AB9FCF712FDB2
:10FC40002046F8BD01F064FAA0420ED230462146AB
:10FC5000FCF74CFD074650B129462246FCF7D6FC7E
:10FC600030462946FCF7FEFC01E02846F8BD384640
:10FC7000F8BD000038B5074C054600202060084656
:10FC800011461A46F2F764F9431C02D1236803B106
:10FC90002B6038BD7C1C001031F0004310B500D142
:10FCA00078B10C4AA3F5801494420CD9B3F5801FA7
:10FCB0000BD3094A93420AD1D0F1010038BF00208A
:10FCC00010BD022010BD042010BD032010BD002077
:10FCD00010BD00BFFFFFDF7F0000F07FF0B50B78A5
:10FCE0005E2B02D04C1C002102E08C1C4B780121C1
:10FCF000002281540132B2F5807FFAD10BB9651E22
:10FD00001BE0C1F10107FEB2C654621C12F8011CCF
:10FD1000551E2D29144604D05D290DD069B10B461E
:10FD2000F1E715785D2DFAD09D42F8DB0133AB4247
:10FD3000C654FBDB0232E9E715462846F0BD000059
:10FD4000004870470000C07F30B5026811F8015BC1
:10FD5000541C55B153782246A3F14104192C98BF85
:10FD60002033AB42F2D0002030BD0460012030BD12
:10FD70002DE9F0410D469046FFF71EFE06460F4660
:10FD8000B8F1000F0FD0C5F30A53C3F16B03002B7A
:10FD900009DD1C0504F17F5303F54013002201F037
:10FDA00079FBBDE8F08130463946BDE8F0810000BE
:10FDB0002DE9F04F00239FB08146049115921A93CC
:10FDC0004FF0000A4FF0000B1991199A13780D2B80
:10FDD00005D8092B14D2002B00F0B18113E02B2B96
:10FDE00007D02D2B02D0202B0DD109E0012609963A
:10FDF00001E000270997531C199353782BB99EE112
:10FE000001321992E1E700260996199C2378302BDC
:10FE10005AD16378582B01D0782B49D1099F1AAB5E
:10FE200000930197484619A99C4A1BAB00F09EFE1F
:10FE300010F00706054600F0AD85062E02D101340C
:10FE400019947EE11A9A3AB11CA83521FFF7A0FE59
:10FE500048461A99FFF711FB1B9A062E21D8DFE8B6
:10FE600006F0040D08171C0D04004FF0000BDA46D5
:10FE700017E0DDF870A0DDF874B012E01D9B02F20F
:10FE8000334223F48013DDF870A043EA025B08E0FC
:10FE9000DFF80CB24FF0000A03E06FF0004B4FF0B8
:10FEA000FF3A2B0740F176854BF0004B00F072BD16
:10FEB000199B5A1C19925B78302BF9D0002B00F05B
:10FEC00069850123059301E000260596199F4FF0EF
:10FED00000080797CDF80C804446199E3578A5F1A7
:10FEE0003003DAB2092A10D8082CD8BF039F4FF08C
:10FEF0000A02D8BF02FB073706F10106D4BF0397F9
:10FF000002FB083801341996E7E74846FFF76AFA1A
:10FF100007684846FFF766FA0068FCF7DCFD3946DB
:10FF200002463046FCF7DFFD064628B100232A468C
:10FF3000194625460A935FE04846199DFFF752FA95
:10FF40000068FCF7C8FD2B1819932A5C002C45D1DA
:10FF50002346302A05D1199A0133511C1991527840
:10FF6000F7E7A2F13101082942D8199E194600236A
:10FF700007961D46303A03F1010029D001446E1C5A
:10FF8000771B874210DA771E082F06DC039F4FF09D
:10FF90000A0C0CFB07F7039704E0102EDCBF0A27BE
:10FFA00007FB08F80136EBE7002BACBFEB182B1C66
:10FFB000082B03F1010505DC039E0A2303FB06263B
:10FFC000039604E0102DDCBF0A2303FB0828002061
:10FFD000199B5A1C19925A78034602E0254633466B
:10FFE0003146A2F130000928C4D901270A9703E05D
:10FFF0000025012029460A9022F02006452E53D1E3
:020000021000EC
:1000000025B91BB9059E002E00F09980199F7A1C16
:1000100019927A7804972B2A04D02D2A05D000262D
:100020000F9608E000200F9001E001270F97049E33
:10003000B21C1992B278A2F13007092F32D8302AB7
:1000400004D1199A571C19975278F8E7A2F1310791
:10005000082F29D81998A2F130070690199A561C32
:10006000199652780E96A2F13006092E05D84FF057
:100070000A0C0CFB0727303FF0E70E98069EC6EBF4
:10008000000CBCF1080F44F61F6C02DC6745B8BFDA
:10009000BC460F9F57B1CCF1000C07E0B42701001C
:1000A0000000F07F049E19964FF0000C002D4CD1FB
:1000B000002B40F06F84059F002F40F06B840A985E
:1000C00000283CD14E2A1BD002DC492A05D036E05C
:1000D000692A02D06E2A13D031E019A8AC49FFF783
:1000E00033FE60B3199B19A8013BAA491993FFF786
:1000F0002BFE10B9199B01331993DFF8B4B21AE043
:1001000019A8A549FFF720FEC8B1199B1B78282B19
:100110000FD119A8A1491CAA00F06AFF052808D12F
:100120001D9BDDF870A043F0FF4B4BF4E00B00F09B
:1001300031BCDFF880B24FF0000A00F02BBC049B0A
:1001400019930026099600F025BCC1EB0C01039819
:10015000102DB4BFAC464FF0100CCDF808C006917E
:1001600001F022F9DDF808C0002C08BF2C46BCF1D4
:10017000090F82468B4615DD894B03EBCC0353E90F
:10018000122301F087F9064640460F4601F00CF9AC
:1001900002460B463046394600F0CAFFDDF808C07B
:1001A00082468B460F2D37DC069F002F00F0F2832E
:1001B00023DD162F07DC7A49524601EBC701D1E94E
:1001C00000015B4614E0069EC5F125039E4223DC38
:1001D000734CC5F10F0504EBC503751BD3E9000192
:1001E00052465B4604EBC50401F054F9D4E9002300
:1001F00001F050F982468B46CCE3069F16370BDBA5
:10020000DDF818C0664F5046A7EBCC075946D7E932
:10021000002301F069FAEDE7069ECCEB0508B04437
:10022000B8F1000F61DD18F00F030AD05C4A02EB51
:10023000C303D3E9000152465B4601F02BF9824625
:100240008B4638F00F0800F0C880B8F59A7F13DDB0
:100250004FF00008CDF80C80CDF81C80CDF814804C
:10026000079F2223C9F80030DFF844B14FF0000A9D
:10027000002F40F07B838DE34FEA28185046594603
:100280000026B8F1010F0DDD18F0010F06D0454B27
:1002900003EBC603D3E9002301F0FCF801364FEA73
:1002A0006808EEE73F4B8246A1F1547B03EBC6069C
:1002B00052465B46D6E9000101F0ECF821F000431C
:1002C0008B461B0D38491B058B428246C0D8A1F5D1
:1002D00080118B4206D90026DFF8DCB04FF0FF3AE0
:1002E00004967CE00BF1547B77E076D0C8F10008EF
:1002F00018F00F030AD02A4A504602EBC3035946AE
:10030000D3E9002301F0F0F982468B465FEA281812
:1003100063D0B8F11F0F08DD4FF00008CDF80C8056
:10032000CDF81C80CDF814801EE118F0100F14BF1A
:100330006A26002604961D4E50465946B8F1000F15
:100340000ADD18F0010F03D0D6E9002301F0A2F86E
:100350004FEA68080836F1E7049F82468B469FB350
:10036000C1F30A53C3F16B03002B2DDD1F2B25DDD9
:10037000342B4FF0000A02DD4FF05C7B24E0203B81
:100380004FF0FF3101FA03F303EA0B0B1CE000BF4F
:100390004A250100A726010052250100F02701008F
:1003A000B8260100802701000000A07CC8270100BA
:1003B0000000F07F0000F8FFFFFFEF7F4FF0FF32FB
:1003C00002FA03F303EA000A5046594600220023CA
:1003D00001F0C8FA00289FD101E000270497039E8E
:1003E00048460096079922462B46FFF797F8079054
:1003F00000283FF42DAF069F4FF000087B42002FEE
:10040000A8BF00230E93CDF80C80079E4846716864
:10041000FEF7FEFF059000283FF422AF326906F197
:100420000C01023292000C30FCF7F0F81BAB009389
:100430001CAB0193484652465B46CDE90AABFFF739
:1004400030FB1A9000283FF40BAF48460121FFF71C
:10045000F4F8039000283FF403AF1B9BDDF818C0AD
:10046000002B2CEAEC77C0F28B800E9C3A461C44A1
:10047000049E1C9D9B1B59196FF47F739942C5F113
:10048000360580F287805B1A1F2BC3EB05054FF002
:10049000010078DC9840002314900F9304986619AB
:1004A0001544A642B4BF334623460544AB42A8BF19
:1004B0002B46002B02DDF61AED1AE41A0E990029DC
:1004C0006FD1002E00F38780002F40F08E80002D2A
:1004D00000F39580002C00F39C8048461A99059AF9
:1004E000FFF70AFA804600283FF4BAAEC668002338
:1004F000C36003990896FFF7E2F9002880F298801C
:10050000002E40F02082BAF1000F40F01C82CBF3A5
:100510001303002B40F017822BF000431B0D1B052B
:10052000B3F1D66F40F20F82D8F81430002B7AD096
:10053000414601224846FFF76FF903998046FFF7CD
:10054000BEF9002840F3FF812BF00043049F1B0DF0
:100550001B05002F00F09C80B3F1D66F00F298804D
:10056000B3F15C7F00F2F181079E22234FF0000A75
:100570004FF0000BC9F80030002E40F0F78109E27F
:10058000FA1A0E9C74E7844E1490761A00FA06F656
:100590000F9683E700264FF0010C0F96CDF850C060
:1005A0007CE7484603990E9AFFF7E8F80390002885
:1005B0003FF456AE484603991A9AFFF747F80346A8
:1005C00000283FF44DAE48461A990293FEF755FFB6
:1005D000029B1A9375E748461A993246FFF71CF9B1
:1005E0001A9000287FF470AF3AE6484605993A46DB
:1005F000FFF7C4F8059000287FF469AF30E648465D
:1006000005992A46FFF708F9059000287FF462AFA4
:1006100026E6484603992246FFF7FEF80390002895
:100620007FF45BAF1CE6D8F81030012B80DC8AE148
:1006300063D1089FCBF313032FB358495A468B421B
:100640002FD1049E51466EB1554B0BEA0303B3F113
:10065000D46F07D81B0DC3F16B034FF0FF3000FAC6
:1006600003F301E04FF0FF3399421AD14D4B9A4208
:1006700002D101313FF4F4AD494B4FF0000A134071
:1006800003F5801B5FE163B9BAF1000F09D15BE7A5
:10069000A3F580136FEA135B6FEA0B5B4FF0FF3A31
:1006A00051E10F9B13B113EA0B0F02E0149E16EAFF
:1006B0000A0F00F04881089F50465946049A57B1E6
:1006C000FFF756FB02460B46DDE90A0100F030FD5C
:1006D00082468B4637E1FFF74BFB02460B46DDE9CE
:1006E0000A0100F023FD0022002382468B4601F020
:1006F00039F900287FF438AF25E140460399FFF728
:1007000022FA00224FF0804304460D4601F03EF9E4
:10071000002832D0089E26B1234F002634463D469D
:100720004CE0BAF1000F03D1CBF313033BB90BE05C
:10073000BAF1010F03D1BBF1000F3FF415AF002652
:100740001A4F0024184D39E0204629460022164B46
:1007500001F012F940B9204629460022144B00F05E
:1007600099FE04460D4601E0114D002405F10047B5
:1007700016941797DDE9166720E0204629460022E7
:100780000B4B00F087FE089E04460D4696B901F11A
:100790000047109011970FE0E3FBFFFFFFFF0F00F2
:1007A0000000F07FFFFFEF7F0000F03F0000F0BF90
:1007B0000000E03FCDE91045DDE910672BF0004C6B
:1007C0004FEA1C5C844B4FEA0C5C9C4531D1DDE95F
:1007D0000A01ABF1547BCDE90C0150465946CDF8E6
:1007E00008C0FFF7E9F802460B463046394600F0EC
:1007F00051FE02460B465046594600F099FC21F046
:1008000000431B0D754A1B0593428246DDF808C064
:100810000CD9734B0D99994203D10C9A01323FF4D4
:100820001FADDFF8BCB14FF0FF3A7BE001F1547B24
:1008300042E0049B53B3BCF1D46F27D85EA3D3E945
:10084000002320462946CDF808C001F09FF8DDF8C6
:1008500008C0B8B12946204601F0DEF8002808BFDC
:10086000012000F0A1FD089E04460D46DDF808C0F9
:1008700026B901F100471290139701E0CDE9124526
:10088000DDE9126707F1D663CCEB0307DDE90A0166
:10089000CDF808C0FFF790F802460B4630463946BF
:1008A00000F0F8FD02460B46DDE90A0100F040FCCD
:1008B000DDF808C082468B46049F002F32D12BF012
:1008C00000431B0D1B059C452CD12946204601F0F9
:1008D0007BF800F079FD02460B462046294600F0E1
:1008E00025FC089F04460D462FB9BAF1000F02D12E
:1008F000CBF3130686B12046294631A3D3E9002362
:1009000001F03AF8002831D1204629462EA3D3E938
:10091000002301F04FF804E02DA3D3E9002301F0F8
:100920002BF818BB48461A99FEF7A7FD48460599CB
:10093000FEF7A3FD48460399FEF79FFD4846414652
:10094000FEF79BFD61E5049E86B1264F00200C90CA
:100950000D9750465946DDE90C2300F09BFD824679
:100960008B4619B910B92223C9F8003048461A99A4
:10097000FEF783FD48460599FEF77FFD484603993B
:10098000FEF77BFD48460799FEF777FD484641464E
:10099000FEF773FD159E0EB1199B3360099F1FB1C1
:1009A00050460BF1004101E0504659461FB0BDE8EA
:1009B000F08F00BFAFF300800000C0FFFFFFDF41FA
:1009C0009535A094FFFFDF3F35E5AF350000E03FF0
:1009D0009535A094FFFFCF3F0000E07FFFFF9F7C95
:1009E000FFFFEF7F0000503984463A482DE9F04F71
:1009F000D0F800800E46344614F8015B08EB050081
:100A0000407800F0080000F0FF0708B12646F2E742
:100A10002D2D03D1B41C7578012703E02B2D04BFC5
:100A20007578B41C33F010000DD1302D08D120782A
:100A300000F0DF00582847D165781023023402E027
:100A4000002B08BF0A234FF0FF39B9FBF3F903FB72
:100A500009FA00266FEA0A0A304608EB050B9BF8F4
:100A600001B01BF0040F01D0303D0BE01BF0030B75
:100A70001AD0BBF1010F14BF4FF0570B4FF0370BDB
:100A8000CBEB05059D420FDA002E08DB484506D862
:100A900001D1554503DC03FB0050012601E04FF076
:100AA000FF3614F8015BD8E7002E05DA2223CCF8D4
:100AB00000304FF0FF3001E007B1404242B106B1D3
:100AC000611E1160BDE8F08F002B08BF0823BAE754
:100AD000BDE8F08FE0010010F0B506694B11B3429C
:100AE00000F1140226DA11F01F0102EB860602EB78
:100AF000830401D1134616E052F82350C1F1200CB3
:100B0000CD4004341346B44209D2276807FA0CF7E3
:100B10003D4343F8045B54F8045BCD40F3E71D60AC
:100B20004DB1043307E0B44205D254F8041B43F836
:100B3000041BF8E713469B1A9B10036103B943613A
:100B4000F0BDA0F13003092B01D820380AE0A0F154
:100B50006103052B01D8473804E0A0F14103052BC0
:100B600002D82738C0B27047002070472DE9F04FF7
:100B700089B00591069390460390FEF733FC006818
:100B80004FF0000B0490FBF7A6FF049B059903446C
:100B900013F8013C029007930B6802331F4613F8C9
:100BA000010B302802D10BF1010BF7E7FFF7C9FF6A
:100BB0000646F8B938460499029AFBF794FF0028D4
:100BC00039D1029B029DF85C3D44FFF7BAFF002833
:100BD00033D02B4618781F46302803F10103F9D093
:100BE000FFF7AFFFD0F1010438BF00242E464FF0CD
:100BF000010B01E000242646B9464D46287809F14C
:100C00000109FFF79EFF0028F7D128460499029AB0
:100C1000FBF769FF58B95EB9029E2E44B1464D46B6
:100C2000287809F10109FFF78CFF0028F7D136B1C8
:100C3000761BB60003E03D4600E0064601242B7813
:100C4000502B01D0702B34D16B782B2B05D02D2B52
:100C500005D005F10109002104E0002100E0012197
:100C600005F1020999F800000191FFF76AFF431EA0
:100C7000DBB2182B01991CD8A0F1100A09F101036D
:100C8000994699F80000013301910093FFF759FF4D
:100C9000421ED2B2182A0199009B05D80A2202FBF3
:100CA0000A0AAAF1100AEBE709B1CAF1000A564490
:100CB00000E0A9460599C1F800902CB1BBF1000FE6
:100CC0000CBF062000207DE1EB1B013B2146072BDA
:100CD00002DD01315B10FAE70398FEF799FB4FF054
:100CE000000900F1140A04465346CB46BD4233D9ED
:100CF0006A1E0592079915F8012C8A4209D0BBF1AA
:100D0000200F17D1C3F800904FF000090433CB46F1
:100D100010E0029A0599C2F1010C8C44BC45EED357
:100D2000604604998DE80810FBF7DDFE9DE8081089
:100D300080B1E4E715F8010C0093FFF702FF00F023
:100D40000F0000FA0BF0DDF814C0009B49EA00091F
:100D50000BF1040B6546C9E743F8049BCAEB030398
:100D60009B10236148465F01FEF71AFCD8F800503B
:100D7000381AA84226DD471B39462046FEF721FFD8
:100D8000C8B17B1E03F01F014FF0010909FA01F100
:100D90005A115AF8222011420ED04B4502DC4FF076
:100DA000020909E02046B91EFEF70BFF0028F6D025
:100DB0004FF0030900E0814620463946FFF78CFEDC
:100DC0003E440CE009DA2F1A214603983A46FEF712
:100DD00023FDF61B044600F1140A4FF00009D8F871
:100DE00008309E4208DD03982146FEF746FB129A22
:100DF00000231360A320E5E0D8F804309E4254DAC3
:100E00009E1BAE422EDBD8F80C30022B1AD0032BDF
:100E10001CD0012B1DD1AE421BD1012D0BDCD8F80B
:100E20000430069962200B6001232361CAF8003068
:100E3000129B1C60C6E02046691EFEF7C2FE002819
:100E4000EDD106E0139B002BE9D002E0139B002BB1
:100E5000E5D103982146FEF710FB129900230B60A1
:100E60005020AFE0771EB9F1000F07D1002F07DD4A
:100E700020463946FEF7A5FE814601E04FF0010904
:100E80007B11012207F01F0702FA07F75AF82330F7
:100E900031461F42204618BF49F00209AD1BFFF73B
:100EA0001BFE0227D8F8046000E00127B9F1000F0B
:100EB00000F08380D8F80C30022B0ED0032B10D01A
:100EC000012B78D119F0020F75D0DAF8003049EA19
:100ED000030919F0010F07D16DE0139BC3F1010362
:100EE0001393139B002B66D0D4F8109004F11403D5
:100EF0004FEA890A03EB0A01184653F8042BB2F1B2
:100F0000FF3F02D00132026021E000228B4243F811
:100F1000042CF1D3A368994512DB61680398013171
:100F2000FEF776FA226904F10C0102328346920040
:100F30000C30FBF76BFB21460398FEF79EFA5C46EC
:100F400023695A1C226104EB830301225A61022F98
:100F500004F1140311D1D8F80020013A954227D1A9
:100F60006A11012105F01F0501FA05F553F8223039
:100F70001D420CBF02270F461AE022694A450ADDCE
:100F800020460121FFF7A8FDD8F8083001369E421F
:100F90003FF729AF0BE015F01F0508D0534453F875
:100FA000040CFEF7FDFAC5F12005A842E8DB012795
:100FB00047F0200701E047F01007129B38461C60FD
:100FC000069B1E6009B0BDE8F08FC2F108029200D6
:100FD00070B5C2F12004056850F8043F03FA04F626
:100FE000D3403543884240F8045C0360F3D370BDBE
:100FF0002DE9F04F0B6885B05E11039013F01F03CD
:1010000002EB86060293039B18BF0436A6F1040880
:101010001546D3F80090002246F8042C4746444673
:101020009246934699F8011000293AD008468DE877
:101030000600FFF786FD9DE80600D8B9202912D8E2
:10104000DA452BDABC4205D2072A03DC20463946B2
:10105000FFF7BBFFAC4220D9271F002244F8042C25
:10106000DA463C461AE029294CD1039B09F10201DA
:10107000196016E00132082A0BF1010B06DDAC42C3
:101080000CD9002244F8042C043C0122216800F011
:101090000F0040EA0111216000E0082209F1010976
:1010A000C0E7BBF1000F2DD0BC4205D2072A03DCFC
:1010B00020463946FFF789FFAC420CD92B4654F83D
:1010C000042B444543F8042BF9D9002243F8042BA0
:1010D0004345FAD90DE0029B5BB1C3F120094FF003
:1010E000FF3323FA09F956F8043C03EA090346F8EA
:1010F000043C56F8043C043E33B9B542F9D101230F
:101100002B6001E0042000E0052005B0BDE8F08F71
:1011100051F8040C002802DA04390B58184404383A
:101120007047000081F0004102E000BF83F00043FF
:1011300030B54FEA41044FEA430594EA050F08BF72
:1011400090EA020F1FBF54EA000C55EA020C7FEA36
:10115000645C7FEA655C00F0E2804FEA5454D4EBB3
:101160005555B8BF6D420CDD2C4480EA020281EA7D
:10117000030382EA000083EA010180EA020281EAB5
:101180000303362D88BF30BD11F0004F4FEA013107
:101190004FF4801C4CEA113102D0404261EB410116
:1011A00013F0004F4FEA03334CEA133302D052429C
:1011B00063EB430394EA050F00F0A780A4F1010458
:1011C000D5F1200E0DDB02FA0EFC22FA05F2801892
:1011D00041F1000103FA0EF2801843FA05F3594178
:1011E0000EE0A5F120050EF1200E012A03FA0EFCF7
:1011F00028BF4CF0020C43FA05F3C01851EBE37121
:1012000001F0004507D54FF0000EDCF1000C7EEB3D
:1012100000006EEB0101B1F5801F1BD3B1F5001F7B
:101220000CD349085FEA30004FEA3C0C04F101049A
:101230004FEA445212F5800F80F09A80BCF1004FC3
:1012400008BF5FEA500C50F1000041EB045141EA45
:10125000050130BD5FEA4C0C404141EB010111F446
:10126000801FA4F10104E9D191F0000F04BF0146F1
:101270000020B1FA81F308BF2033A3F10B03B3F1CF
:1012800020020CDA0C3208DD02F1140CC2F10C025F
:1012900001FA0CF021FA02F10CE002F11402D8BFBD
:1012A000C2F1200C01FA02F120FA0CFCDCBF41EA89
:1012B0000C019040E41AA2BF01EB0451294330BD58
:1012C0006FEA04041F3C1CDA0C340EDC04F1140435
:1012D000C4F1200220FA04F001FA02F340EA03000C
:1012E00021FA04F345EA030130BDC4F10C04C4F152
:1012F000200220FA02F001FA04F340EA0300294632
:1013000030BD21FA04F0294630BD94F0000F83F47B
:10131000801306BF81F480110134013D4EE77FEA5E
:10132000645C18BF7FEA655C29D094EA050F08BFAA
:1013300090EA020F05D054EA000C04BF194610468B
:1013400030BD91EA030F1EBF0021002030BD5FEACF
:10135000545C05D14000494128BF41F0004130BDF7
:1013600014F580043CBF01F5801130BD01F000454B
:1013700045F0FE4141F470014FF0000030BD7FEABE
:10138000645C1ABF194610467FEA655C1CBF0B46B9
:10139000024650EA013406BF52EA033591EA030FD0
:1013A00041F4002130BD00BF90F0000F04BF0021C8
:1013B000704730B54FF4806404F132044FF00005FB
:1013C0004FF0000150E700BF90F0000F04BF002174
:1013D000704730B54FF4806404F1320410F00045DA
:1013E00048BF40424FF000013EE700BF42004FEAD5
:1013F000E2014FEA31014FEA02701FBF12F07F4352
:1014000093F07F4F81F06051704792F0000F14BF4E
:1014100093F07F4F704730B54FF4607401F0004592
:1014200021F0004120E700BF50EA010208BF7047E9
:1014300030B54FF000050AE050EA010208BF7047DE
:1014400030B511F0004502D5404261EB41014FF447
:10145000806404F132045FEA915C3FF4DCAE4FF04B
:1014600003025FEADC0C18BF03325FEADC0C18BF32
:10147000033202EBDC02C2F1200300FA03FC20FA83
:1014800002F001FA03FE40EA0E0021FA02F11444D0
:10149000C1E600BF70B54FF0FF0C4CF4E06C1CEAE5
:1014A00011541DBF1CEA135594EA0C0F95EA0C0F5A
:1014B00000F0DEF82C4481EA030621EA4C5123EACD
:1014C0004C5350EA013518BF52EA033541F48011FC
:1014D00043F4801338D0A0FB02CE4FF00005E1FBAF
:1014E00002E506F00042E0FB03E54FF00006E1FBF9
:1014F00003569CF0000F18BF4EF0010EA4F1FF043C
:10150000B6F5007F64F5407404D25FEA4E0E6D417B
:1015100046EB060642EAC62141EA55514FEAC5208C
:1015200040EA5E504FEACE2EB4F1FD0C88BFBCF508
:10153000E06F1ED8BEF1004F08BF5FEA500E50F1B9
:10154000000041EB045170BD06F0004646EA01017F
:1015500040EA020081EA0301B4EB5C04C2BFD4EBB1
:101560000C0541EA045170BD41F480114FF0000EAA
:10157000013C00F3AB8014F1360FDEBF002001F018
:10158000004170BDC4F10004203C35DA0C341BDC92
:1015900004F11404C4F1200500FA05F320FA04F064
:1015A00001FA05F240EA020001F0004221F0004198
:1015B00010EBD37021FA04F642EB06015EEA430E0B
:1015C00008BF20EAD37070BDC4F10C04C4F120053B
:1015D00000FA04F320FA05F001FA04F240EA0200EE
:1015E00001F0004110EBD37041F100015EEA430EBF
:1015F00008BF20EAD37070BDC4F1200500FA05F2DF
:101600004EEA020E20FA04F301FA05F243EA02035D
:1016100021FA04F001F0004121FA04F220EA02006C
:1016200000EBD3705EEA430E08BF20EAD37070BDB2
:1016300094F0000F0FD101F00046400041EB010192
:1016400011F4801F08BF013CF7D041EA060195F074
:10165000000F18BF704703F00046520043EB03032E
:1016600013F4801F08BF013DF7D043EA060370471B
:1016700094EA0C0F0CEA135518BF95EA0C0F0CD026
:1016800050EA410618BF52EA4306D1D181EA03016C
:1016900001F000414FF0000070BD50EA410606BF66
:1016A0001046194652EA430619D094EA0C0F02D1AB
:1016B00050EA013613D195EA0C0F05D152EA0336F0
:1016C0001CBF104619460AD181EA030101F000410E
:1016D00041F0FE4141F470014FF0000070BD41F057
:1016E000FE4141F4780170BD70B54FF0FF0C4CF431
:1016F000E06C1CEA11541DBF1CEA135594EA0C0F50
:1017000095EA0C0F00F0A7F8A4EB050481EA030E9C
:1017100052EA03354FEA013100F088804FEA033383
:101720004FF0805545EA131343EA12634FEA022251
:1017300045EA111545EA10654FEA00260EF0004112
:101740009D4208BF964244F1FD0404F5407402D264
:101750005B084FEA3202B61A65EB03055B084FEAF5
:1017600032024FF480104FF4002CB6EB020E75EBF2
:10177000030E22BFB61A754640EA0C005B084FEA1A
:101780003202B6EB020E75EB030E22BFB61A754697
:1017900040EA5C005B084FEA3202B6EB020E75EBE2
:1017A000030E22BFB61A754640EA9C005B084FEA5A
:1017B0003202B6EB020E75EB030E22BFB61A754667
:1017C00040EADC0055EA060E18D04FEA051545EA56
:1017D00016754FEA06164FEAC30343EA52734FEAFF
:1017E000C2025FEA1C1CC0D111F4801F0BD141EA78
:1017F00000014FF000004FF0004CB6E711F4801FDD
:1018000004BF01430020B4F1FD0C88BFBCF5E06FBC
:101810003FF6AFAEB5EB030C04BFB6EB020C5FEACC
:10182000500C50F1000041EB045170BD0EF0004E21
:101830004EEA113114EB5C04C2BFD4EB0C0541EA53
:10184000045170BD41F480114FF0000E013C90E650
:1018500045EA060E8DE60CEA135594EA0C0F08BF14
:1018600095EA0C0F3FF43BAF94EA0C0F0AD150EA13
:1018700001347FF434AF95EA0C0F7FF425AF1046A6
:1018800019462CE795EA0C0F06D152EA03353FF4CE
:10189000FDAE1046194622E750EA410618BF52EA4B
:1018A00043067FF4C5AE50EA41047FF40DAF52EA1F
:1018B00043057FF4EBAE12E74FF0FF3C06E000BFBC
:1018C0004FF0010C02E000BF4FF0010C4DF804CDC9
:1018D0004FEA410C7FEA6C5C4FEA430C18BF7FEA89
:1018E0006C5C1BD001B050EA410C0CBF52EA430CB7
:1018F00091EA030F02BF90EA020F0020704710F137
:10190000000F91EA030F58BF994208BF90422CBFC5
:10191000D8176FEAE37040F0010070474FEA410CBE
:101920007FEA6C5C02D150EA013C07D14FEA430CDC
:101930007FEA6C5CD6D152EA033CD3D05DF8040B4D
:10194000704700BF8446104662468C46194663467F
:1019500000E000BF01B5FFF7B7FF002848BF10F156
:10196000000F01BD4DF808EDFFF7F4FF0CBF01209B
:1019700000205DF808FB00BF4DF808EDFFF7EAFF17
:1019800034BF012000205DF808FB00BF4DF808EDD2
:10199000FFF7E0FF94BF012000205DF808FB00BFC7
:1019A0004DF808EDFFF7CEFF94BF012000205DF851
:1019B00008FB00BF4DF808EDFFF7C4FF34BF01205E
:1019C00000205DF808FB00BF4FEA410212F500124B
:1019D00015D211D56FF47873B3EB625212D94FEA76
:1019E000C12343F0004343EA505311F0004F23FA60
:1019F00002F018BF404270474FF00000704750EAB5
:101A0000013005D111F0004008BF6FF00040704771
:101A10004FF00000704700BF4A0011D212F50012CB
:101A200011D20DD56FF47873B3EB62520ED44FEA36
:101A3000C12343F0004343EA505323FA02F07047B6
:101A40004FF00000704750EA013002D14FF0FF30F4
:101A500070474FF0000070474FEA4102B2F1E04397
:101A600024BFB3F5001CDCF1FE5C0DD901F0004C85
:101A70004FEAC0024CEA5070B2F1004F40EB8300D5
:101A800008BF20F00100704711F0804F21D113F101
:101A90003872BCBF01F00040704741F480114FEA3A
:101AA0005252C2F11802C2F1200C10FA0CF320FAC3
:101AB00002F018BF40F001004FEAC1234FEAD323E0
:101AC00003FA0CFC40EA0C0023FA02F34FEA43034A
:101AD000CCE77FEA625307D150EA01331EBF4FF0D3
:101AE000FE4040F44000704701F0004040F0FE40EE
:101AF00040F40000704700BF4FF0FF0C1CEAD052CA
:101B00001EBF1CEAD15392EA0C0F93EA0C0F6FD060
:101B10001A4480EA010C400218BF5FEA41211ED03E
:101B20004FF0006343EA501043EA5111A0FB01312A
:101B30000CF00040B1F5000F3EBF490041EAD371FF
:101B40005B0040EA010062F17F02FD2A1DD8B3F17B
:101B5000004F40EBC25008BF20F00100704790F0EA
:101B6000000F0CF0004C08BF49024CEA502040EA3C
:101B700051207F3AC2BFD2F1FF0340EAC250704702
:101B800040F400004FF00003013A5DDC12F1190F40
:101B9000DCBF00F000407047C2F10002410021FAB2
:101BA00002F1C2F1200200FA02FC5FEA310040F1CA
:101BB000000053EA4C0308BF20EADC70704792F043
:101BC000000F00F0004C02BF400010F4000F013A7B
:101BD000F9D040EA0C0093F0000F01F0004C02BF76
:101BE000490011F4000F013BF9D041EA0C018FE7E5
:101BF0000CEAD15392EA0C0F18BF93EA0C0F0AD0EB
:101C000030F0004C18BF31F0004CD8D180EA010010
